:100000000C945A3A0C94F93A0C94F93A0C94F93A43
:100010000C94F93A0C94F93A0C94F93A0C94F93A94
:100020000C94F93A0C94F93A0C94F93A0C94F93A84
:100030000C94F93A0C94B23E0C94F93A0C94F93AB7
:100040000C94F93A0C94F93A0C94F93A0C94F93A64
:100050000C94F93A0C94F93A0C94F93A0C94F93A54
:100060000C94F93A0C94F93A0C94F93A0C94F93A44
:100070000A461846EB46C64AB04A1B462A46394647
:10008000964A47465546DADADADADADADADADADAE4
:10009000DADADADADADADADADADADADADADADADAC0
:1000A000DADADADADADADADADADADADADADADADAB0
:1000B000DADADADADADADADADADADADADADADADAA0
:1000C000DADADADADADA919191919191919191916A
:1000D0009191919191919191919191919191919110
:1000E0009191919191919191919191919191919100
:1000F00091919191919191919191919191919191F0
:10010000919191919191DADADADADADADADADADA05
:10011000DADADADADADADADADADADADADADADADA3F
:10012000DAFFDADADADADADADADADADADADADADA0A
:10013000DADADADADADADADADADADADADADADADA1F
:10014000DADADADADADADADADADADADADADADADA0F
:10015000DA5D5DDADADADA5D6FB76F665DDA5D6F48
:100160005E00FF5E6F5D665EFF00FFFF5E66665EBF
:10017000FFFF00FF5E665D6F5EFFFF5E6F5DDA5D35
:10018000666F6F665DDADADADADADADADADADADA0A
:10019000DADADADADADA3F3F3FDA3F3F3FDADA3FFC
:1001A0003F3F3F3FDADADADA3F3F3FDADADADA3F87
:1001B0003F3F3F3FDADA3F3F3FDA3F3F3FDADADAAD
:1001C000DADADADADADA13AD5B5B64125C65AE5C5C
:1001D0005C6554AE65AE5D5C5CA65C5C145C5C5CAE
:1001E0006553135C14145C130A135C5C13130A5CF0
:1001F0005C130A0A130A0A1365AE6D5C0A0213B790
:100200006EB7B66E0A0A6EB7B6B7B7B76E02B7B7B3
:10021000B6B76E6EB70A5C1CB76EB66EAE1313B788
:100220006EAEAE6E6E521313AEB6AE65135CDA0BE5
:100230000B0A530B6DDADADADADADADADADADADA80
:10024000DADADADADADA0A5C1B131B131313121385
:100250001C1C1C13131C131B130A0A0A0A135C0A26
:1002600064645C5C1309135C645C5C131309131B0A
:100270005C1B13130A0A0A131313130A0A0A09133D
:1002800012131309120A13120A0A1309130A120A83
:10029000130A091313130A0A5B130A13120A13131E
:1002A00064120A1B5C131C121B0A0A1B1B13131378
:1002B000130A0A131B13090A12120A12120A0A0B52
:1002C0000A0B0A0A4B0A121213131B1B13131B13DC
:1002D000131312131C131B0A0A0A1313131C1213F1
:1002E000131C0A0A0B1C13131C13131313131313DD
:1002F000130A131313130A130A0A13130A130A0B0C
:100300000A0A0A0A09130A135C13131313120A13B5
:1003100013130A0A5C5C130A0A0A09125C641312BA
:10032000130A0A135C5C1B130A130A135C1B1313D6
:10033000130A0A131B1B121313130B0A0A130A12B4
:100340000A1252090A0ADADA116B236B1A23DADA73
:100350000A0911111111DA23232A11232212121072
:1003600010231123221810100910115B1111101AFB
:10037000111810101111101011100A09101110107D
:10038000DA090A13130ADADADA1313131313DADAAF
:10039000DADA0A1C0A1CDADADADA0A0A1B0ADADA08
:1003A000DADA13120A0ADADADADA1212DA51DADAF5
:1003B000DADADA0ADADADADADADADADADADADADA6D
:1003C000DADADADADADA231A6B236B11DADA1111F4
:1003D0001111090ADADA122223112A2323DA182248
:1003E00023112310101211115B111009101011119B
:1003F000101018111A101110090A101110100A13F8
:10040000130A09DA10101313131313DADADA1C0AB9
:100410001C0ADADADADA0A1B0A0ADADADADA0A0A99
:100420001213DADADADA51DA1212DADADADADADAD4
:100430000ADADADADADADADADADADADADADADADAEC
:10044000DADADADADADA23747423231223231A23AA
:1004500023222323111811181810101022221A1009
:10046000101010101010101A12101010100909108E
:10047000101009090A0A130A0A0A13130A1C0A0AA5
:100480000A655C1B09132223222323231A741011EB
:100490001111111111181B222222231122230910DC
:1004A0001011181122231A111010111111231110FB
:1004B0001010111810100A5C131218111009655C45
:1004C0001B13090913131C13135C1B1B0A130A0AC1
:1004D0000A1313130A130A0A0A13130A0A0A64DA1C
:1004E000DA090A4B5BDADADADADADADADADADADA1B
:1004F000DADADADADADADADADADADADADADADADA5C
:10050000DADADADADADA13130A5C13131313120ADB
:10051000135C121C0A1C130A131B130A1313121266
:10052000090A0B0A0A13DADADADA09DADA09DADAA4
:10053000DADADADADADADADADADADADADADADADA1B
:10054000DADADADADADA131213131B1B1313DA13FB
:10055000131312131C13DA0A0A0A1313131CDA12E8
:10056000131C0A0A0B1CDADA1C1313131313DADA3E
:10057000130A13131313DADADA0A13130A13DADA83
:10058000DA0A0A0A09130A135C1313130A4B0A1333
:1005900013130A0A5CDA130A0A0A09125CDA131244
:1005A000130A0A135CDA1B130A130A13DADA131399
:1005B000130A0A13DADA121313130BDADADA0A124D
:1005C0000A1252DADADADADADADADADADADADA90F5
:1005D000DADADA90DADADA98DADADA98DADADA988B
:1005E000DADADA98DADADAEADADADAEADADA98F2B7
:1005F00098DA98F298DAEAF2EADAEAF2EADAEAF271
:10060000EADAEAF2EADAF2E1E1F2E190EAEAF2D8D1
:10061000E1F29898F2EAEAE1A1EA90EAF2E9F2E17D
:1006200098EA98F2E9E9F2E190E1D9F2E1E1EAE150
:10063000989898F2E198E9E19090E1F2E1F2E1E135
:1006400098E1F2E198EADADADADADADADADADADA58
:10065000DA5D5DDADADADA5D6FB76F665DDA5D6F43
:100660005E003F5E6F5D665E3F003F3F5E66665EBA
:100670003F3F003F5E665D6F5E3F3F5E6F5DDA5DF0
:10068000666F6F665DDADADADADA33DADADADADAAC
:10069000DADA3233DADADADADADA337B2ADADADABF
:1006A000DADADA32732A2ADADA21DADA733233332F
:1006B0002A22212A7C33DA33332A212A3333DADA25
:1006C00032332A21332ADADADADADADADADADADA99
:1006D000DADADA2A2ADADADADA2A2A63DADADADAB1
:1006E00032325BDADADADA2A325BDADADADA2A3268
:1006F00029DADA737B332A2A2132337332DA292951
:100700002A33332ADADA121213131B1B1313911331
:10071000131312131C13910A0A0A1313131C9112B8
:10072000131C0A0A0B1C91911C13131313139191A0
:10073000130A131313139191910A13130A1391912E
:10074000910A0A0A09130A135C13131313120A13EA
:1007500013130A0A5C91130A0A0A09125C91131214
:10076000130A0A135C911B130A130A1391911313B2
:10077000130A0A139191121313130B9191910A12F8
:100780000A1252919191DADA5ABDFE5ADADADA5A3D
:10079000FEFEFFFE5ADA11B5FFFEFEFEB51111B5E1
:1007A000FEFEFEFEFE1111B5FEFFFEFFFE1111B5AD
:1007B000BDFEFEFEB511DA11B5BDBDB511DADADA4E
:1007C00011115A11DADA91915ABDFE5A9191915A4A
:1007D000FEFEFFFE5A9111B5FFFEFEFEB51111B5EA
:1007E000FEFEFEFEFE1111B5FEFFFEFFFE1111B56D
:1007F000BDFEFEFEB5119111B5BDBDB51191919132
:1008000011115A119191DADADADADADADADADADAB5
:10081000DADADADADADADADA030406FF0707DADA3A
:10082000DADA4080C0C0DADADA4080FFC0C0DADA53
:10083000DA4080C0C0C0DADADADA405D5E67DADA60
:10084000DADADA405D5EDADADADADADADADADADA9B
:10085000DADADADADADA0606040303DADADAC08098
:100860004040DADADADAC0C0804040DADADAC0C012
:10087000804040DADADA5E5D4040DADADADA5D40AA
:1008800040DADADADADADADADADADADA405DDADA79
:10089000DADADADA4080DADADADADA4080C0DADABA
:1008A000DADA4080C05DDADADA4080FF5D5EDADAFB
:1008B000DA40805D5E67DADADADA405D6767DADAF5
:1008C000030406FF07074040DADADADADADA4040F2
:1008D000DADADADADADA804040DADADADADAC0807A
:1008E0004040DADADADA5EC0804040DADADA5E5EB8
:1008F000804040DADADA5E5D4040DADADADA0606BB
:10090000040303DADADADADADADADA081018FFFFDF
:10091000FFFFFF081820DA5BADADADFF1828DADA6B
:10092000DADADA10AD18DADADADA08101820DADAF8
:10093000DADA10181828DADADADA10182028DADA0F
:10094000DADA095BA4A41008DADADADADADA1808F3
:10095000DADADADADADA18ADDADADADADADA181072
:10096000ADDADADADADA18181008080808DA28280E
:100970002820201818102828282828201818A4A46F
:10098000A4A4ADF6A45B9191919191081018FFFF7A
:10099000FFFFFF081820915BADADADFF18289191C6
:1009A00091919110AD189191919108101820919109
:1009B00091911018182891919191101820289191D7
:1009C0009191095BA4A410089191919191911808BB
:1009D00091919191919118AD91919191919118105E
:1009E000AD91919191911818100808080891282844
:1009F0002820201818102828282828201818A4A4EF
:100A0000A4A4ADF6A45BDADADADADADADADADADA78
:100A1000DADADADADADADADADADADADADADADADA36
:100A2000DADADA5DB767DADADADADA5D6667DADA9D
:100A3000DADADADA5D66DADADADADA525BF6DADAF2
:100A4000DADADA030406DADADADADADADADADADA87
:100A5000DADADADADADADADADADADADADADA665DE7
:100A6000DADADADADADA665DDADADADADADA5DDA54
:100A7000DADADADADADA5B52DADADADADADA04038A
:100A8000DADADADADADADADADADA03040606DADA1B
:100A9000DA0304F60607DADA03040606ADFFDA0322
:100AA0000406060752FFDA0404060607A4ADDA03BB
:100AB000040606F60707DADA030406060707DADA99
:100AC000DA0304040606060403DADADADADA06F6EA
:100AD0000403DADADADAAD06060403DADADA520700
:100AE00006060403DADAA40706060404DADA07F6CF
:100AF00006060403DADA0706060403DADADA06047D
:100B00000403DADADADA91919191919191919191CC
:100B100091919191919191919191919191919191C5
:100B20009191915DB76791919191915D6667919176
:100B3000919191915D669191919191525BF6919114
:100B4000919191030406919191919191919191913B
:100B50009191919191919191919191919191665DE4
:100B6000919191919191665D9191919191915D9108
:100B70009191919191915B529191919191910403F5
:100B80009191919191919191919103040606919186
:100B9000910304F60607919103040606ADFF910345
:100BA0000406060752FF910404060607A4AD91034C
:100BB000040606F6070791910304060607079191BC
:100BC000910304040606060403919191919106F69F
:100BD000040391919191AD060604039191915207FE
:100BE000060604039191A40706060404919107F6F2
:100BF00006060403919107060604039191910604E9
:100C0000040391919191DADADADADADADADADADA15
:100C1000DADADADADADADADADADADADADADADADA34
:100C2000DADADADADADADADADADADADADADADADA24
:100C3000DADADADADADADADADADADA525252DADAAC
:100C4000DA52525B5B5BDADADADADADADADADADA91
:100C5000DADADADADADADADADADADADADADADADAF4
:100C6000DADADADADADADADADADADADADADADA526C
:100C7000525D67DADADA525B5D5BDA5EDADA52AD80
:100C80005B52DADADADADADA525B5BA4ADA4DA5272
:100C90005B5BA4F6ADADDA525BA4F6ADADADDA5256
:100CA0005BA4ADADADADDA525B5BA4ADADA4DADA59
:100CB000525B5BA4A4A4DADADA525B5B5B5BDADA40
:100CC000DADA095252525B52525209DADADAA45B8A
:100CD0005B525209DADAA45B5B5B5252DADAA45B4C
:100CE0005B5B5252DADAA45B5B5B5252DADA5B5B33
:100CF0005B5252DADADA5B525252DADADADA52520A
:100D000009DADADADADADADADADADADA0818DADAA8
:100D1000DADADA081807DADADADADA080818DADA00
:100D2000DADADA083808DADADADADA081808DADACF
:100D3000DA0808180818DADA081838280808DA086B
:100D400018381808180808DADADADADADADA1808F5
:100D5000DADADADADADA0808DADADADADADA38080B
:100D6000DADADADADADA1808DADADADADADA08180B
:100D70000808DADADADA0828381808DADADA1808C5
:100D800018381808DADADA08381808080818DA08FB
:100D9000183838083808DADA081828081808DADAAB
:100DA000DA0808080808DADA081828380808DA081B
:100DB000182838380838DA08182838380828DADACD
:100DC000081828380818080808183808DADA38081F
:100DD00038381808DADA1808281808DADADA0808C9
:100DE0000808DADADADA0838281808DADADA083835
:100DF00038281808DADA083838281808DADA08182B
:100E0000281808DADADADADADADADADADADADADA88
:100E1000DADADADADADADADADADADADADADADADA32
:100E2000DADADA141E14DADADADA141E2726DADA53
:100E3000DADA1D262727DADADADA1D1E2627DADAC9
:100E4000DADA141D1E1DDADADADADADADADADADAFE
:100E5000DADADADADADADADADADADADADADA1D1E6B
:100E6000DADADADADADA131D1EDADADADADA26139D
:100E70001EDADADADADA27261DDADADADADA181D31
:100E800013DADADADADADADADADADA131418DADAD8
:100E9000DADADADA1028DADADADADA181020DADA74
:100EA000DA1828180818DADADADADADADA18DADA2E
:100EB00010DA08DA1820DA0818DA281020102010C2
:100EC0002018101820102813DADADADADADA101813
:100ED000281808DADADA080808DADADADADA10DAF8
:100EE000DADADADADADA18DADADADADADADA1810B0
:100EF00008DA1810DADA20081018201020DA10109A
:100F0000181810181018DADADADADADADADADADADD
:100F1000DADADADADADADADADA5D6640DADADADABC
:100F2000DA5D6740DADA0704665D665D0407DADADF
:100F3000DA5D6740DADADADADA5D6640DADADADA26
:100F4000DA5D6740DADADADADA525B40DADADADA2C
:100F5000DA5D6740DADADADADA5D6640DADADADA06
:100F6000DA5D6740DADADA5D665D675D5D40DADAE0
:100F70005D5D665D40DADADADA5D6740DADADADAE0
:100F8000DA525B40DADADADADADADADA5151DADA74
:100F9000DADADA51929BDADADADA519AF5FEDADA4B
:100FA000DADA92ECFFFFDADADADA92F5FFFFDADA70
:100FB000519292ECFFFF5192A3EDEDF6FFFF519B92
:100FC000F6FFFFFFFFFF5151DA51515151519B9AEA
:100FD0009292E4F5F6ECFFF6A3ECFFFFFFFFFFFFB4
:100FE000F5F5FFFFFFFFFFFFFEF6FFFFFFFFFFFF2F
:100FF000FFFFFFFFFFFFFFFFFFFFFFFFFFFFFFFF01
:10100000FFFFFFFFFFFF51DADADADADADADA5192BC
:10101000DADADADADADAED5192DADADADADAF6A408
:101020009B5192DADADAF6FFF6EC51DADADAFFFF00
:10103000FFF59B51DADAFFFFFEF59B51DADAFFFF8D
:10104000FEF6ED51DADA51A3F6FFFFFFFFFF51A3E1
:10105000F6FFFFFFFFFF519AEDFFFFFFF6FEDA926A
:10106000A3EDF6EDECF6DA51929B9B9BE4ECDADA19
:1010700051515192E4E4DADADADADA5192A3DADAA7
:10108000DADADADA5151FFFFFFFFFFFFFFFFFFFF60
:10109000FFFFFFFFFFFFFFFFFFFFFEFFFFFFFFFF61
:1010A000FFFFF6FFFFFFF6FEF6F5ECF6FEF6E4ECCA
:1010B000ECA3A3ECECECA3A39B92929A9B9B5151C3
:1010C00051DADA515151FFFFFFFFFFA351DAFFFF61
:1010D000FFFFFFEC51DAFFFEFFFFF6E451DAF6ED19
:1010E000F5F5ECA351DAEDA39B9B9A51DADAA39ABA
:1010F000515151DADADA5251DADADADADADA51DA85
:10110000DADADADADADAF2E1E1F2E190EAEAF2D80E
:10111000E1F29898F2EAEAE1A1EA90EAF2E9F2E172
:1011200098EA98F2E9E9DAE190E1D9F2E1E1DADA74
:10113000989898F2E198DAE19090E1F2E1F2DAE140
:1011400098E1F2E198EADADAE1F2E190EAEADADA51
:10115000E1F29898F2EADADADAEA90EAF2E9DADA2F
:10116000DAEA98F2E9E9DADADADAD9F2E1E1DADAB6
:10117000DADA98F2E198DADADADADAF2E1F2DADAFD
:10118000DADADAE198EAEAEA90E1F2E1E1F2EAF2A7
:101190009898F2E1D8F2E9F2EA90EAA1E1EAE9E905
:1011A000F298EA98E1F2E1E1F2D9E190E1DA98E12E
:1011B000F2989898DADAF2E1F2E19090E1DAEA98BE
:1011C000E1F2E198E1DAEAEA90E1F2E1DADAEAF270
:1011D0009898F2E1DADAE9F2EA90EADADADAE9E9B9
:1011E000F298EADADADAE1E1F2D9DADADADA98E18F
:1011F000F298DADADADAF2E1F2DADADADADAEA9874
:10120000E1DADADADADADADADADAEBF5F6F6DADAD3
:10121000DAECFFFFFFFFDADADAFEFFFFFFFFDADAD0
:10122000DAFEFEFEF6F6DADADAF4F5F4ECECDADA07
:10123000DADAE3E3E2EADADADADAE2E1F2FCDADA9B
:10124000DADAE2EAF2FBDADADADADAEAF2F2DADA6D
:10125000DADADAE1EAF2DADADADADAE2E9EADADA98
:10126000DADADADAE1F2DADADADADADAEAF2DADA97
:10127000DADADADADAEADADADADADADADADADADABE
:10128000DADADADADADAF6F6F5EBDADADADAFFFF10
:10129000FFFFECDADADAFFFFFFFFFEDADADAF6F662
:1012A000FEFEFEDADADAECECF4F5F4DADADAEAE2A7
:1012B000E3E3DADADADAFCF2E1E2DADADADAFBF2FA
:1012C000EAE2DADADADAF2F2EADADADADADAF2EAFE
:1012D000E1DADADADADAEAE9E2DADADADADAF2E121
:1012E000DADADADADADAF2EADADADADADADAEADA26
:1012F000DADADADADADADADADADADADADADADADA4E
:10130000DADADADADADAF5F6F5F5F5F5F5F5FFFF1A
:10131000FFFFFFFFFFFFFFFFFFFFFFFFFFFFFEFEDF
:10132000F5F5F6FEFFFFF5F4ECEBECECFEFFEAEB77
:10133000E1D89090ECFFF2FBE9E1D990F6F6F2F2F9
:10134000E1EAE190ECEAF5F5F5F5F5F5F5F5FFFFE5
:10135000FFFFFFFFFFFFFFFFFFFFFFFFFFFFFFFF9D
:10136000FEF6FEFFFFFEFFFFF5ECECF5FEF5FFFEDF
:10137000F4A298D9EBEBF5F5E3EAF2E999E2909A59
:10138000EAFBF2E99098F2E1E1F2E190EAEAF2D8C0
:10139000E1F29898F2EAEAE1A1EA90EAF2E9F2E1F0
:1013A00098EA98F2E9E9F2E190E1D9F2E1E1EAE1C3
:1013B000989898F2E198E9E19090E1F2E1DAE1E1C0
:1013C00098E1DAEADADAE150EAFBF2E99098E190A2
:1013D000E9FCF2E99898E190E1FBF2F29898989094
:1013E00098F2F3E9E998989890F2F3E1E9989890E7
:1013F00099F2F3E1E990DADADAEBF2E1A190DADAE4
:10140000DADAF2E2DA90DADADADADA3F3F3FDADA37
:10141000DADADADA3F3FDADADADADADADA3FDADAFD
:10142000DADADADADADADADADADADADADADADADA1C
:10143000DADADADADADADADADADADADADADADADA0C
:10144000DADADADADADADADADADADADADADA3F3F32
:10145000DADADADADADA3F3F3FDADADADADA3F3FF3
:101460003F3FDADADADA3F3F3F3F3FDADADADA3FB4
:101470003F3F3FDADADADA3F3F3F3FDADADADA3FA4
:101480003F3F3FDADADADADADADADADADADADADA8D
:10149000DADADADADADADADADADADADADADADADAAC
:1014A000DADADADADA3FDADADADADADA3F3FDADA6D
:1014B0003F3F3F3F3F3FDADADA3F3F3F3F3FDADA35
:1014C000DADADADADADADA3F3F3F3FDADADADA3F83
:1014D0003F3F3FDADADA3F3F3F3F3FDADADA3F3F7A
:1014E0003F3FDADADADA3F3F3FDADADADADA3F3F99
:1014F000DADADADADADA3FDADADADADADADADADAE7
:10150000DADADADADADADAF2F2F2F2F2DADAF2F293
:10151000F2F2F2F2F2DAF2F2DADADAF2F2DAF2F223
:10152000DADADAF2F2DAF2F2DADADAF2F2DAF2F25B
:10153000F2F2F2F2F2DADAF2F2F2F2F2DADADADA1B
:10154000DADADADADADADAF2F2F2F2F2DADADAF26B
:10155000F2F2F2F2DADADADADAF2F2F2DADADADA43
:10156000DAF2F2F2DADADADADAF2F2F2DADADADA4B
:10157000DAF2F2F2DADADADADAF2F2F2DADADADA3B
:10158000DADADADADADAF2F2F2F2F2F2DADAF2F2FB
:10159000F2F2F2F2F2DADADADAF2F2F2DADADADAEB
:1015A000F2F2F2DADADADAF2F2F2DADADADAF2F2DB
:1015B000F2F2F2F2DADAF2F2F2F2F2F2F2DADADA83
:1015C000DADADADADADAF2F2F2F2F2F2DADADAF2D3
:1015D000F2F2F2F2F2DADADADAF2F2F2DADADADAAB
:1015E000F2F2F2DADADADADADAF2F2F2DADAF2F29B
:1015F000F2F2F2F2F2DAF2F2F2F2F2F2DADADADA43
:10160000DADADADADADADADAF2F2F2F2DADADAF2C2
:10161000F2F2F2F2DADADAF2F2DAF2F2DADAF2F23A
:10162000DADAF2F2DADAF2F2F2F2F2F2F2DAF2F212
:10163000F2F2F2F2F2DADADADADAF2F2DADADADA62
:10164000DADADADADADAF2F2F2F2F2F2F2DAF2F222
:10165000F2F2F2F2DADAF2F2DADADADADADAF2F22A
:10166000F2F2F2F2DADADADADADAF2F2F2DADAF21A
:10167000F2F2F2F2DADAF2F2F2F2F2DADADADADAF2
:10168000DADADADADADADAF2F2F2F2F2DADAF2F212
:10169000F2F2F2DADADAF2F2DADADADADADAF2F202
:1016A000F2F2F2F2DADAF2F2DADADAF2F2DAF2F2AA
:1016B000F2F2F2F2F2DADAF2F2F2F2F2DADADADA9A
:1016C000DADADADADADAF2F2F2F2F2F2F2DADAF2BA
:1016D000F2F2F2F2F2DADADADAF2F2F2DADADADAAA
:1016E000F2F2F2DADADADADAF2F2F2DADADADAF2B2
:1016F000F2F2DADADADADAF2F2F2DADADADADADAD2
:10170000DADADADADADADAF2F2F2F2F2DADAF2F291
:10171000F2F2F2F2F2DAF2F2DADADAF2F2DADAF239
:10172000F2F2F2F2DADAF2F2DADADAF2F2DAF2F229
:10173000F2F2F2F2F2DADAF2F2F2F2F2DADADADA19
:10174000DADADADADADADAF2F2F2F2F2DADAF2F251
:10175000F2F2F2F2F2DAF2F2DADADAF2F2DADAF2F9
:10176000F2F2F2F2F2DADADADADADAF2F2DADAF219
:10177000F2F2F2F2F2DAF2F2F2F2F2F2DADADADAC1
:10178000DADADADADADADADADADADADADADADADAB9
:10179000DAF2F2F2DADADADADAF2F2F2DADADADA19
:1017A000DADADADADADADADADAF2F2F2DADADADA51
:1017B000DAF2F2F2DADADADADADADADADADADADA41
:1017C000DADADADADADADADADADADADADADADADA79
:1017D000DADADADADADAF2F2F2DAF2F2F2DADAF2C1
:1017E000F2F2F2F2DADADADAF2F2F2DADADADAF299
:1017F000F2F2F2F2DADAF2F2F2DAF2F2F2DADADA59
:10180000DADADADADADADADADADA090A145DDA1CDA
:101810006E261E151E66DA6E776F67675E5EDA6586
:10182000666715155F5FDA12130C14151515DA12B9
:101830000A0A0A0A0B0BDADADADADADADA09DADAB7
:10184000DADADADADADA141414141415155D6667C4
:101850006767675E16165F5E665D5D5D5D555F5F1F
:101860005F5E5E5E5E561515150D0D0D0D0D130BAD
:10187000140C0C0C0C0C0101020201020202DADA57
:1018800009090A0A0A0A5E665E6666150C151616CE
:10189000161E1516565F5555555E5F1E5E15565E33
:1018A0005E676F6F6F6F0D1515155E6727270C0C40
:1018B0000B0B0B1D1D1D020A0A0A0A0A0A020B1352
:1018C00013130A0A0A0A1414141414130B0A5E5F81
:1018D000565E561515150D0D0D0D0E1656566F67E5
:1018E0005F5E5E5F565627675E15151515151E5D02
:1018F000140B0B0B0B0B020A0A020A0A0A0A0A0A49
:101900000A0A0A53DADA0A0A0A0A0A0A020214144A
:101910001D666F6F6F675E16676F6F67675E565EF7
:1019200016161615151515151515140B0B0B0A0A99
:101930000101DADADADA09DADADADADADADADADA8A
:10194000DADADADADADA02020A0A0ADADADA675E06
:101950005E5E150BDADA161515151566DADA15144A
:101960000C141D1DDADA0A0A0A0A13DADADADADAEC
:10197000DADADADADADADADADADADADADADADADAC7
:10198000DADADADADADADADADADA09090A13DADAF0
:10199000DADADA090909DADADADADADADA09DADAEB
:1019A000DADADADADADADADADADADADADADADADA97
:1019B000DADADADADADADADADADADADADADADADA87
:1019C000DADADADADADA131313131313130A0A0A58
:1019D0000B131313130A090A131313130A0A090921
:1019E00009090A0A0A0BDA1209090A121314DADAC7
:1019F000DADADADADADADADADADADADADADADADA47
:101A0000DADADADADADA0A0A0A0A0ADADADA0A09E7
:101A1000090909DADADA0A135B1313DADADA5C5C39
:101A20001C14145CDADA5D1D5D14141B12DADADAA8
:101A3000DADADADADADADADADADADADADADADADA06
:101A4000DADADADADADA91919191919191919191D0
:101A500091919191919191919191910A91919191FD
:101A60009191121291519191919113120A0A9191AF
:101A700091910A0A1B0A919191910A1C0A1C919159
:101A800091131313131391919152120A120A919107
:101A9000910B131313129191130A0A1313139191BB
:101AA000130A130A131B915C130A0A131213915C95
:101AB00012090A0A0A13915C0A0A1313130A121371
:101AC0001313135C130A91919191919191919191BA
:101AD00091919191919191910A91919191915191BD
:101AE0001212919191910A0A1213919191910A1BEC
:101AF0000A0A919191911C0A1C0A919191911313D8
:101B00001313139191910A120A1252919191121387
:101B100013130B9191911313130A0A1391911B1331
:101B20000A130A1391911312130A0A135C91130AF0
:101B30000A0A09125C910A1313130A0A5C910A1328
:101B40005C131313131291919113131313139191A7
:101B500091910A1C0A1C919191910A0A1B0A919178
:101B6000919113120A0A91919191121291519191AE
:101B70009191910A919191919191919191919191DC
:101B800091919191919113131313139191911C0AB7
:101B90001C0A919191910A1B0A0A919191910A0A4A
:101BA0001213919191915191121291919191919160
:101BB0000A9191919191919191919191919191919C
:101BC0009191919191911C13135C1B1B0A130A0AAA
:101BD0000A1313130A130A0A0A13130A0A0A64914E
:101BE00091090A4B5B919191919191919191919170
:101BF00091919191919191919191919191919191D5
:101C000091919191919113130A5C13131313120A7A
:101C1000135C121C0A1C130A131B130A131312124F
:101C2000090A0B0A0A1391919191099191099191D5
:101C30009191919191919191919191919191919194
:101C4000919191919191DADADADADA09535CDADA80
:101C5000DA0909535C5CDADADA01090A5353DA0962
:101C60000909090A530A01090A530A09270A01093D
:101C70000A535C530A53DA090A0A0A090A0ADA0102
:101C8000090A090A0A090A0A6F6F0A530ABF53535D
:101C90000A09090937FF535C5C530A0A6F37533747
:101CA0005C5C530A536F37BF53530A0A530A6F37AA
:101CB0000A0A090A0A0A276F0A0A0A0A0A090A0A04
:101CC0006F0A0A090927530ADADADADADADA5C0A79
:101CD0005C5C0A5CDADA0A0A530A535C5CDA6FBFAE
:101CE0000A0A09535309530953FF0909090A370915
:101CF000096F530A0A533753270A5337370A0A0A18
:101D00000927535C530ADA0109090A0A0A09DA09A0
:101D100009090A090909DA090A0101090901DADAD6
:101D2000090101010909DADADA0101090101DADA46
:101D3000DADA01010A09DADADADADA010109DADAD9
:101D4000DADADADADADA0909090A535C0A0909097E
:101D5000010A090A0A09090A0A01090927010101F8
:101D60000909010101DA090101010901DADA0101B8
:101D7000010101DADADA01010101DADADADADADAB2
:101D8000DADADADADADADADADADADADADADADADAB3
:101D9000DADADA5D5D5DDADADA5D5D6FBFFFDADA75
:101DA0005D6FFFFFFFFFDA5DBFFFFF6F5D5DDA5D17
:101DB000FFFF5D5D66665DFFFF5D5D666F6F5DFFEA
:101DC000BF5D6F6F6F6FDADADADADADADADA5D5DB1
:101DD0005DDADADADADAFFBF6F5D5DDADADAFFFFF1
:101DE000FFBF6F5DDADA66FFBFFFBF775DDA665D62
:101DF000FFBF77BF5DDA6F665D77BF773F5D6F6668
:101E000066BF773F775D5DFF6F5D6F6F6F6F5DFFE3
:101E10006F5D6F6F6F6F5DFFFF5D6F6F6F6FDA5D8F
:101E2000FFBF666F6F6FDA5DBFFFBF776F6FDADA84
:101E30005D6F77BF77BFDADADA5D5D6FBF77DADAC9
:101E4000DADADA5D5D5D6F665D5D5D5D3F5D6F6F2A
:101E50006666665D775D6F6F6F6F66BF3F5D6F6FC4
:101E60006F6FBF3F5DDA6F6FBF773F775DDA773FA8
:101E7000773F6F5DDADA3F776F5D5DDADADA5D5D05
:101E80005DDADADADADADADADADADADADADADADA2F
:101E9000DADADA5D5D5DDADADADA5D5D7777DADAD9
:101EA000DADA5D7777BFDADADA5D775D5D5DDADA47
:101EB000DA6F5D5D5D5DDADADA775D5D5D66DADA2F
:101EC0005D775D5D5D6FDADADADADADADADA5D5D2E
:101ED0005DDADADADADA6F5D5D5DDADADADABF773F
:101EE0006666DADADADABFBF6F6666DADADA77BF41
:101EF000775D66DADADABF77BF6F6666DADA77BF00
:101F0000BF6F6F6FDADADADA5DBF5D5D666FDADAFE
:101F10005D775D5D666FDADADA776F5D6F6FDADAFB
:101F2000DA6FBF666F6FDADADA5D77BF666FDADABB
:101F3000DADA5D77BF77DADADADA5D5D773FDADA57
:101F4000DADADA5D5D5D6F6FBF776F6FDADA6F6F68
:101F5000BF6F6F6FDADA6F373F6F6666DADA6FBFBF
:101F6000775D66DADADABF776F6666DADADA773FF4
:101F70006666DADADADA6F5D5D5DDADADADA5D5D85
:101F80005DDADADADADADADADADADADADADADADA2E
:101F9000DADADADA5D5DDADADADADADA5D66DADA8C
:101FA000DADADADA666FDADADADADADA6F77DADA3E
:101FB000DADADADA77BFDADADADADADABFBFDADA35
:101FC000DADADADABFFFDADADADADADADADA5D5D61
:101FD000DADADADADADA665DDADADADADADA6F6631
:101FE000DADADADADADA776FDADADADADADABF779D
:101FF000DADADADADADABFBFDADADADADADAFFBF6D
:10200000DADADADADADADADADADADADAFFFFDADAE6
:10201000DADADADABFFFDADADADADADABFBFDADA4C
:10202000DADADADA77BFDADADADADADA6F77DADA5C
:10203000DADADADA666FDADADADADADA5D66DADAD0
:10204000DADADADA5D5DFFFFDADADADADADAFFBF96
:10205000DADADADADADABFBFDADADADADADABF7794
:10206000DADADADADADA776FDADADADADADA6F667D
:10207000DADADADADADA665DDADADADADADA5D5DAB
:10208000DADADADADADADADADADADADADADADADAB0
:10209000DADADA5D5D5DDADADADA5D5D5D6FDADAF9
:1020A000DADA666F77BFDADADA666F66BF6FDADAC6
:1020B000DA6F6F77BF5DDADADA6F6FBF6F66DADA21
:1020C0006FBFBF776F6FDADADADADADADADA5D5D44
:1020D0005DDADADADADA77BF6F5DDADADADABF77C1
:1020E000776FDADADADA5D6F77BF5DDADADA5D5DFB
:1020F000BF776FDADADA5D5D6F77BFDADADA5D5D06
:102100006FBF775DDADADADA6FBFBF776F6FDADA6F
:102110006FBFBF776F6FDADADA6F6F3F376FDADA78
:10212000DA6F6F77BF66DADADA666F6F77BFDADA9F
:10213000DADA66663F77DADADADA5D5D5D6FDADAC7
:10214000DADADA5D5D5D665D5D5DBF5DDADA6F5DD1
:102150005D5D775DDADA6F5D5D6F77DADADA6F5DD4
:1021600066BF6FDADADA5D66BFBF5DDADADA77BFEB
:10217000BF6FDADADADA3F776F5DDADADADA5D5D25
:102180005DDADADADADAE8E89A9A9A9A9A9AE8E874
:10219000E8E8E8E89A9A9A9AE8F5F5F5E8E89A9A6C
:1021A0009A9A9A9AF5F5E8E89A9A9A9A9A9AE8E8A1
:1021B000E8E8E8E89A9A9A9AE8F5F5F5E8E89A9A4C
:1021C0009A9A9A9AF5F59A9A9A9A9A9AE8E89A9A1D
:1021D000E8E8E8E8E8E8E8E8F5F5F5E89A9AF5F5DA
:1021E0009A9A9A9A9A9A9A9A9A9A9A9AE8E89A9AB3
:1021F000E8E8E8E8E8E8E8E8F5F5F5E89A9AF5F5BA
:102200009A9A9A9A9A9A9A9A9A9A9A9AF5F5E8E8DC
:102210009A9A9A9A9A9AE8E8E8E8E8E89A9A9A9A4A
:10222000E8F5F5F5E8E89A9A9A9A9A9AF5F5E8E8C1
:102230009A9A9A9A9A9AE8E8E8E8E8E89A9A9A9A2A
:10224000E8F5F5F5E8E8F5F59A9A9A9A9A9A9A9A3D
:102250009A9A9A9AE8E89A9AE8E8E8E8E8E8E8E8D2
:10226000F5F5F5E89A9AF5F59A9A9A9A9A9A9A9AB9
:102270009A9A9A9AE8E89A9AE8E8E8E8E8E8E8E8B2
:10228000F5F5F5E89A9A9A9AE8F5F5F5E8E89A9A54
:102290009A9A9A9AF5F5E8E89A9A9A9A9A9AE8E8B0
:1022A000E8E8E8E89A9A9A9AE8F5F5F5E8E89A9A5B
:1022B0009A9A9A9AF5F5E8E89A9A9A9A9A9AE8E890
:1022C000E8E8E8E89A9AE8E8F5F5F5E89A9AF5F585
:1022D0009A9A9A9A9A9A9A9A9A9A9A9AE8E89A9AC2
:1022E000E8E8E8E8E8E8E8E8F5F5F5E89A9AF5F5C9
:1022F0009A9A9A9A9A9A9A9A9A9A9A9AE8E89A9AA2
:10230000E8E8E8E8E8E8E8E8E8E8E8E89A9A9A9A85
:10231000E8F5F5F5E8E89A9A9A9A9A9AF5F5E8E8D0
:102320009A9A9A9A9A9AE8E8E8E8E8E89A9A9A9A39
:10233000E8F5F5F5E8E89A9A9A9A9A9AF5F5E8E8B0
:102340009A9A9A9A9A9A9A9AE8E8E8E8E8E8E8E87D
:10235000F5F5F5E89A9AF5F59A9A9A9A9A9A9A9AC8
:102360009A9A9A9AE8E89A9AE8E8E8E8E8E8E8E8C1
:10237000F5F5F5E89A9AF5F59A9A9A9A9A9A9A9AA8
:102380009A9A9A9AE8E8E8E89A9A9A9A9A9AE8E8D9
:10239000E8E8E8E89A9A9A9AE8F5F5F5E8E89A9A6A
:1023A0009A9A9A9AF5F5E8E89A9A9A9A9A9AE8E89F
:1023B000E8E8E8E89A9AF5F5E8F5F5F5E8E8F5F5DE
:1023C000F5F5F5F5F5F59A9A9A9A9A9AE8E89A9AAF
:1023D000E8E8E8E8E8E8E8E8F5F5F5E89A9AF5F5D8
:1023E0009A9A9A9A9A9A9A9A9A9A9A9AE8E89A9AB1
:1023F000E8E8E8E8E8E8E8E8F5F5F5E8F5F5F5F502
:10240000F5F5F5F5F5F5F5F5F5F5F5F5F5F5F5F57C
:10241000F5F5F5F5F5F5F5F5F5E8F5F5E8F5E8F593
:10242000F5F5F5E8F5E8F5E8F5F5F5F5E8F5F5F590
:10243000E8F5F5E8E8E8E8E8F5E8E8F5F5F5E8E8CE
:10244000E8F5F5F5E8E8F5F5F5F5F5F5F5F5F5F563
:10245000F5E8F5F5F5F5F5F5F5F5F5F5E8F5F5F546
:10246000E8E8E8F5F5F5E8E8F5F5F5E8E8F5F5F577
:10247000E8E8F5F5F5E8F5F5F5E8E8E8F5F5F5E867
:10248000E8E8E8DBE8E8E8DBE8E8E8E8E8E8E8E8E6
:10249000E89191E8DBE89191E891E891E8E8919181
:1024A000919191919191919191919191919191911C
:1024B000919191919191919191919191919191910C
:1024C000919191919191E8E8DBE8E8E8E8E8E8E8A3
:1024D000E8E8E8E8E89191E89191E891E8E89191DD
:1024E00091919191919191919191919191919191DC
:1024F00091919191919191919191919191919191CC
:102500009191919191919A9A9A9A9A9AF5F5E8E80F
:102510009A9A9A9A9A9AE8E8E8E8E8E89A9A9A9A47
:10252000E8F5F5F5E8E89A9A9A9A9A9AF5F5E8E8BE
:102530009A9A9A9A9A9AE8E8E8E8E8E89A9AF5F571
:10254000E8F5F5F5E8E8F5F59A9A9A9A9A9A9A9A3A
:102550009A9A9A9AE8E89A9AE8E8E8E8E8E8E8E8CF
:10256000F5F5F5E89A9AF5F59A9A9A9A9A9A9A9AB6
:102570009A9A9A9AE8E89A9AE8E8E8E8E8E8E8E8AF
:10258000F5F5F5E8F5F5F5F5F5F5F5F5F5F5F5F508
:10259000F5F5F5F5F5F5F5F5E8F5F5F5F5F5F5F5F8
:1025A000F5F5F5E8E8E8E8F5E8E8E8F5F5F5E8E850
:1025B000F5F5E8E8E8F5F5F5E8E8F5F5F5F5E8E826
:1025C000E8E8E8E8E8E8F5F5F5F5F5F5F5F5E8F516
:1025D000F5F5F5F5F5F5F5F5F5E8E8E8F5F5F5F5D2
:1025E000E8F5F5E8E8F5E8E8F5F5F5F5E8F5F5F5E9
:1025F000F5E8E8F5F5E8E8E8E8E8E8E8E8F5E8E827
:10260000E8E8E8DBE8E8E8DBE8E8E8E8E8E891E8BB
:10261000E89191E891919191E891E891919191914E
:10262000919191919191919191919191919191919A
:10263000919191919191919191919191919191918A
:10264000919191919191919191E8E8E8E8E89191C7
:102650009191E8E8E89191E89191E891E8E8919109
:10266000919191919191919191919191919191915A
:10267000919191919191919191919191919191914A
:102680009191919191919A9AE8F5F5F5E8E89A9AE5
:102690009A9A9A9AF5F5E8E89A9A9A9A9A9AE8E8AC
:1026A000E8E8E8E89A9A9A9AE8F5F5F5E8E89A9A57
:1026B0009A9A9A9AF5F5E8E8F59A9A9A9A9AF5F517
:1026C000E8E8E8E8F5F5E8E8F5F5F5E89A9AF5F5CB
:1026D0009A9A9A9A9A9A9A9A9A9A9A9AE8E89A9ABE
:1026E000E8E8E8E8E8E8E8E8F5F5F5E89A9AF5F5C5
:1026F0009A9A9A9A9A9A9A9A9A9A9AF5E8E8F5F58D
:10270000E8E8E8E8F5F5E8E8E8E8E8E89A9A9A9A67
:10271000E8F5F5F5E8E89A9A9A9A9A9AF5F5E8E8CC
:102720009A9A9A9A9A9AE8E8E8E8E8E89A9A9A9A35
:10273000E8F5F5F5E8E8F5F59A9A9A9AF5F5E8E8F6
:10274000F5F5F5F5F5F59A9AE8E8E8E8E8E8E8E857
:10275000F5F5F5E89A9AF5F59A9A9A9A9A9A9A9AC4
:102760009A9A9A9AE8E89A9AE8E8E8E8E8E8E8E8BD
:10277000F5F5F5E89A9AF5F59A9A9A9AF5F5F5F538
:10278000F5F5F5F5E8E8DADADADADADADADADADA21
:10279000DADADADADADADADADADADADADADADADA99
:1027A000DADADADADADADADADADADADADADADADA89
:1027B000DADADADADADADADADADA00DADADADADA53
:1027C00000DA00DADADADADADADADADADADA00DAF7
:1027D000DADADADADADA0057DADADADADADA005713
:1027E000DADADA00DADA0005DADADA00DADADA0086
:1027F000DADA0000DADADADADADA005700DADADA24
:10280000DADA005700DADADA000000DADA00DADAC7
:10281000000500DADA00DA0000570000DA00DA001A
:10282000005700000000DA00005705055705DA00E0
:1028300000575705057F00000557577F7FFF0005AC
:10284000577F7FFF7F7FDADA05DA000500DADA00EA
:102850000500005700DA00000505575700DA0500AB
:102860005705570500DA57055705050500DA57578C
:10287000577F575700DA7F57FF7F570505007F7F47
:102880007F7F7F7F0500DADADADADADADADADADAC3
:1028900000DADADADADADADA00DADADADADADA0026
:1028A00000DADADADADADA000500DADADADADA00C5
:1028B0005705DADA00DADADA0057DADA0000DADABB
:1028C000DA00DADA0005DADADADADADADADADADAF1
:1028D000DADADADA00DADADADADADADA0005DADAE1
:1028E000DADADADA0005DADADADADADA0057DADA54
:1028F000DADADADA0557DADADADADADA5700DADAED
:10290000DADADADA05DADADADADADADA0005DADAAB
:10291000DADADA005705DADADADA00005705DA002F
:10292000DA0000055705DA00000500057F05000004
:10293000055705577F57000005577F7FFF7F00052C
:10294000577F7F7F7F7FDADADA00DADADADADADA0B
:10295000DA000000DA00DADADA000000DA0000005B
:1029600000000500000005000005570500000505F2
:1029700005577F0500007F575757FF5705057F7F95
:10298000FF7F7F7F5705FFFFFFF5DADAF5FFFFFFD7
:10299000FFFFFFFFFFFFFFFFFFFFFFFFFFFF919123
:1029A000F5FFFFFFFF9191919191919191919191FB
:1029B0009191919191919191919191919191919107
:1029C000919191919191FFFFFFFFF5DADAF5FFFF09
:1029D000FFFFFFFFFFFFFFFFFFFFFFFFFFFF9191E3
:1029E00091F5FFFFFFFF91919191919191919191BB
:1029F00091919191919191919191919191919191C7
:102A0000919191919191F5FFFFFFFFF5DADAFFFFC8
:102A1000FFFFFFFFFFFFFFFFFFFFFFFFFFFFFF9134
:102A20009191F5FFFFFF91919191919191919191E8
:102A30009191919191919191919191919191919186
:102A4000919191919191DADAF2F2F2F2F2DADAF20C
:102A5000F2F2F2F2DADAF2F2F2DADADADADAF2F2FE
:102A6000DADADAF2F2DAF2F2F2F2F2F2F2DAF2F2BE
:102A7000DADADAF2F2DAF2F2F2DADAF2F2DADAF2F6
:102A8000F2DADADADADADAF2F2F2F2F2F2DADADAFE
:102A9000F2F2F2F2F2F2DADADADADADAF2DADAF2D6
:102AA000F2DADAF2F2DADAF2F2DADADAF2F2DAF2C6
:102AB000F2F2F2F2F2DADAF2F2F2F2F2DADADADA86
:102AC000DADADADADADADADAF2F2F2F2F2DADAF2D6
:102AD000F2F2F2F2F2DADAF2F2DADADADADADAF296
:102AE000F2DADADADADADAF2F2F2DADADADADADAE6
:102AF000F2F2F2F2F2F2DADADAF2F2F2F2F2DADA2E
:102B0000DADADADADADADAF2F2F2F2F2F2DADADA95
:102B1000F2F2F2F2F2F2DADADADADADAF2F2DAF23D
:102B2000F2DADADAF2F2DAF2F2DADAF2F2DADAF245
:102B3000F2F2F2F2DADADAF2F2F2F2DADADADADA35
:102B4000DADADADADADADAF2F2F2F2F2DADADAF255
:102B5000F2F2F2F2F2DADAF2F2DADADADADADAF215
:102B6000F2F2F2F2DADADAF2F2DADADADADADAF21D
:102B7000F2F2F2F2F2F2DAF2F2F2F2F2F2DADADA95
:102B8000DADADADADADADAF2F2F2F2F2F2DADAF2FD
:102B9000F2F2F2F2F2F2DAF2F2DADADADADADAF2BD
:102BA000F2F2F2DADADADAF2F2F2F2F2DADADAF2AD
:102BB000F2DADADADADADAF2F2DADADADADADAF215
:102BC000DADADADADADADADAF2F2F2F2F2DADAF2D5
:102BD000F2F2F2F2F2F2DAF2F2DADADADADADAF27D
:102BE000F2DADAF2F2F2DAF2F2F2DAF2F2F2DADA55
:102BF000F2F2F2F2F2F2DADADAF2F2F2F2F2DADA2D
:102C0000DADADADADADADAF2F2DADADAF2F2DAF2AC
:102C1000F2DADADAF2F2DAF2F2DADADAF2F2DAF254
:102C2000F2F2F2F2F2F2DAF2F2F2F2F2F2F2DAF2B4
:102C3000F2DADADAF2F2DAF2F2DADADAF2F2DAF234
:102C4000DADADADADADADADADAF2F2F2DADADADA9C
:102C5000DAF2F2F2DADADADADAF2F2F2DADADADA44
:102C6000DAF2F2F2DADADADADAF2F2F2DADADADA34
:102C7000DAF2F2F2DADADADADAF2F2F2DADADADA24
:102C8000DADADADADADADADADAF2F2F2F2DADADA44
:102C9000DADAF2F2F2DADADADADAF2F2F2DADADA04
:102CA000DADAF2F2F2DADADADADAF2F2F2DADADAF4
:102CB000DADAF2F2F2DADADAF2F2F2F2F2DADADAB4
:102CC000F2F2F2F2DADADAF2F2DADAF2F2F2DAF274
:102CD000F2DAF2F2F2DADAF2F2F2F2F2DADADAF264
:102CE000F2F2F2DADADADAF2F2F2F2F2DADADAF26C
:102CF000F2DAF2F2F2DADAF2F2DADAF2F2F2DADA5C
:102D0000DADADADADADADAF2F2F2DADADADADAF2C3
:102D1000F2F2DADADADADAF2F2F2DADADADADAF283
:102D2000F2F2DADADADADAF2F2F2DADADADADAF273
:102D3000F2F2F2F2F2DADAF2F2F2F2F2F2F2DADAD3
:102D4000DADADADADADADAF2F2DADADAF2F2DAF26B
:102D5000F2F2DAF2F2F2DAF2F2F2F2F2F2F2DAF29B
:102D6000F2F2F2F2F2F2DAF2F2DAF2DAF2F2DAF2A3
:102D7000F2DADADAF2F2DAF2F2DADADAF2F2DADA0B
:102D8000DADADADADADADAF2F2F2DADAF2F2DAF213
:102D9000F2F2F2DAF2F2DAF2F2F2F2F2F2F2DAF25B
:102DA000F2DAF2F2F2F2DAF2F2DADAF2F2F2DAF27B
:102DB000F2DADADAF2F2DAF2F2DADADAF2F2DADACB
:102DC000DADADADADADADADAF2F2F2F2F2DADAF2D3
:102DD000F2F2F2F2F2F2DAF2F2DADADAF2F2DAF24B
:102DE000F2DADADAF2F2DADAF2F2DAF2F2DADADA9B
:102DF000F2F2F2F2F2DADADADAF2F2F2DADADADA73
:102E0000DADADADADADAF2F2F2F2F2F2DADADAF27A
:102E1000F2F2F2F2F2DADADADADAF2F2F2DAF2F222
:102E2000DAF2F2F2DADAF2F2F2F2F2DADADAF2F212
:102E3000F2F2DADADADAF2F2DADADADADADAF2F262
:102E4000DADADADADADADAF2F2F2F2F2DADAF2F23A
:102E5000F2F2F2F2F2DAF2F2DADADAF2F2DAF2F2CA
:102E6000DADAF2F2F2DADAF2F2DAF2F2DADADAF202
:102E7000F2F2F2F2F2DADADAF2F2DAF2F2DADADADA
:102E8000DADADADADADAF2F2F2F2F2F2DADADAF2FA
:102E9000F2F2F2F2F2DADADADADAF2F2F2DAF2F2A2
:102EA000DAF2F2F2DADAF2F2F2F2F2DADADAF2F292
:102EB000DAF2F2F2DADAF2F2DADAF2F2F2DADADAB2
:102EC000DADADAF2F2F2DAF2F2F2F2F2F2DAF2F25A
:102ED000F2F2F2F2F2DADAF2F2F2DADADADADADA92
:102EE000F2F2F2DADADADADADAF2F2F2DADAF2F282
:102EF000F2F2F2F2F2DAF2F2F2F2F2F2DADADADA2A
:102F0000DADADADADADAF2F2F2F2F2F2F2DAF2F249
:102F1000F2F2F2F2F2DADADAF2F2F2DADADADADA51
:102F2000F2F2F2DADADADADAF2F2F2DADADADADA71
:102F3000F2F2F2DADADADADAF2F2F2DADADADADA61
:102F4000F2F2DADADADADADAF2F2DAF2F2DADAF239
:102F5000F2F2DAF2F2DAF2F2F2DADAF2F2DAF2F2C9
:102F6000DADADAF2F2DAF2F2DADADAF2F2DAF2F201
:102F7000F2F2F2F2F2DADAF2F2F2F2F2F2DADADAA9
:102F8000DADADADADADAF2F2DADADAF2F2DAF2F211
:102F9000F2DAF2F2F2DADAF2F2DAF2F2DADADAF2B9
:102FA000F2F2F2F2DADADADAF2F2F2DADADADADAD9
:102FB000F2F2F2DADADADADADAF2DADADADADADA11
:102FC000DADADADADADAF2F2DADADAF2F2DAF2F2D1
:102FD000DADADAF2F2DAF2F2DAF2DAF2F2DAF2F279
:102FE000F2F2F2F2F2DAF2F2F2F2F2F2F2DAF2F2F1
:102FF000F2DAF2F2F2DAF2F2DADADAF2F2DADADA71
:10300000DADADADADADAF2F2DADADAF2F2DAF2F290
:10301000F2DAF2F2F2DADAF2F2F2F2F2DADADADA38
:10302000F2F2F2DADADADAF2F2F2F2F2DADAF2F210
:10303000F2DAF2F2F2DAF2F2DADADAF2F2DADADA30
:10304000DADADADADADAF2F2DADADAF2F2DAF2F250
:10305000DADADAF2F2DAF2F2F2DAF2F2F2DADAF2F8
:10306000F2F2F2F2DADADADAF2F2F2DADADADADA18
:10307000F2F2F2DADADADADAF2F2F2DADADADADA20
:10308000DADADADADADADAF2F2F2F2F2F2DAF2F2E0
:10309000F2F2F2F2F2DADADADAF2F2F2DADADADAD0
:1030A000F2F2F2DADADADAF2F2F2DADADADAF2F2C0
:1030B000F2F2F2F2F2DAF2F2F2F2F2F2DADADADA68
:1030C000DADADADADADA911365AE6D5C5C9113B7AD
:1030D0006EB7B66EB7916EB7B6B7B7B76EB7B7B7CC
:1030E000B6B76E6EB7135C1CB76EB66EAE1413B780
:1030F0006EAEAE6E6E141313AEB6AE65135C910B6E
:103100000B0A530B6D91DA1365AE6D5C5CDA13B785
:103110006EB7B66EB7DA6EB7B6B7B7B76EB7B7B742
:10312000B6B76E6EB7135C1CB76EB66EAE1413B73F
:103130006EAEAE6E6E141313AEB6AE65135CDA0BE4
:103140000B0A530B6DDADADADADADADADADADA1308
:1031500065AE6D5C5CDA13B76EB7B66EB7DA6EB794
:10316000B6B7B7B76EB7B7B7B6B76E6EB7135C1C66
:10317000B76EB66EAE1413B76EAEAE6E6E1413139A
:10318000AEB6AE65135CDADADADADADADADADADAD5
:10319000DADADADADADADA1365AE6D5C5CDA13B74A
:1031A0006EB7B66EB7DA6EB7B6B7B7B76EB7B7B7B2
:1031B000B6B76E6EB7135C1CB76EB66EAE1413B7AF
:1031C0006EAEAE6E6E14DADADADADADADADADADAC1
:1031D000DADADADADADADADADADADADADADADA1316
:1031E00065AE6D5C5CDA13B76EB7B66EB7DA6EB704
:1031F000B6B7B7B76EB7B7B7B6B76E6EB7135C1CD6
:10320000B76EB66EAE14DADADADADADADADADADA2F
:10321000DADADADADADADADADADADADADADADADA0E
:10322000DADADADADADADA1365AE6D5C5CDA13B7B9
:103230006EB7B66EB7DA6EB7B6B7B7B76EB7B7B721
:10324000B6B76E6EB713DADADADADADADADADADAE7
:10325000DADADADADADADADADADADADADADADADACE
:10326000DADADADADADADADADADADADADADADA1385
:1032700065AE6D5C5CDA13B76EB7B66EB7DA6EB773
:10328000B6B7B7B76EB7DADADADADADADADADADABA
:10329000DADADADADADADADADADADADADADADADA8E
:1032A000DADADADADADADADADADADADADADADADA7E
:1032B000DADADADADADADA1365AE6D5C5CDA13B729
:1032C0006EB7B66EB7DADADADADADADADADADADAA0
:1032D000DADADADADADADADADADADADADADADADA4E
:1032E000DADADADADADADADADADADADADADADADA3E
:1032F000DADADADADADADADADADADADADADADA13F5
:1033000065AE6D5C5CDADA0B0B0A530B6DDADA131F
:1033100065AE6D5C5CDA13B76EB7B66EB7DA6EB7D2
:10332000B6B7B7B76EB7B7B7B6B76E6EB7135C1CA4
:10333000B76EB66EAE1413B76EAEAE6E6E141313D8
:10334000AEB6AE65135C1313AEB6AE65135CDA0BA6
:103350000B0A530B6DDADA1365AE6D5C5CDA13B7EA
:103360006EB7B66EB7DA6EB7B6B7B7B76EB7B7B7F0
:10337000B6B76E6EB7135C1CB76EB66EAE1413B7ED
:103380006EAEAE6E6E1413B76EAEAE6E6E141313D9
:10339000AEB6AE65135CDA0B0B0A530B6DDADA13BB
:1033A00065AE6D5C5CDA13B76EB7B66EB7DA6EB742
:1033B000B6B7B7B76EB7B7B7B6B76E6EB7135C1C14
:1033C000B76EB66EAE145C1CB76EB66EAE1413B7A5
:1033D0006EAEAE6E6E141313AEB6AE65135CDA0B42
:1033E0000B0A530B6DDADA1365AE6D5C5CDA13B75A
:1033F0006EB7B66EB7DA6EB7B6B7B7B76EB7B7B760
:10340000B6B76E6EB713B7B7B6B76E6EB7135C1CB0
:10341000B76EB66EAE1413B76EAEAE6E6E141313F7
:10342000AEB6AE65135CDA0B0B0A530B6DDADA132A
:1034300065AE6D5C5CDA13B76EB7B66EB7DA6EB7B1
:10344000B6B7B7B76EB76EB7B6B7B7B76EB7B7B7E9
:10345000B6B76E6EB7135C1CB76EB66EAE1413B70C
:103460006EAEAE6E6E141313AEB6AE65135CDA0BB1
:103470000B0A530B6DDADA1365AE6D5C5CDA13B7C9
:103480006EB7B66EB7DA13B76EB7B66EB7DA6EB799
:10349000B6B7B7B76EB7B7B7B6B76E6EB7135C1C33
:1034A000B76EB66EAE1413B76EAEAE6E6E14131367
:1034B000AEB6AE65135CDA0B0B0A530B6DDADA139A
:1034C00065AE6D5C5CDADA0B0B0A530B6DDADADA97
:1034D000DADADADADADADADADADADADADADADADA4C
:1034E000DADADADADADADADADADADADADADADADA3C
:1034F000DADADADADADADADADADADADADADADADA2C
:10350000DADADADADADA1313AEB6AE65135CDA0BAE
:103510000B0A530B6DDADADADADADADADADADADA6D
:10352000DADADADADADADADADADADADADADADADAFB
:10353000DADADADADADADADADADADADADADADADAEB
:10354000DADADADADADA13B76EAEAE6E6E141313B5
:10355000AEB6AE65135CDA0B0B0A530B6DDADADA32
:10356000DADADADADADADADADADADADADADADADABB
:10357000DADADADADADADADADADADADADADADADAAB
:10358000DADADADADADA5C1CB76EB66EAE1413B7D2
:103590006EAEAE6E6E141313AEB6AE65135CDA0B80
:1035A0000B0A530B6DDADADADADADADADADADADADD
:1035B000DADADADADADADADADADADADADADADADA6B
:1035C000DADADADADADAB7B7B6B76E6EB7135C1CE6
:1035D000B76EB66EAE1413B76EAEAE6E6E14131336
:1035E000AEB6AE65135CDA0B0B0A530B6DDADADAA2
:1035F000DADADADADADADADADADADADADADADADA2B
:10360000DADADADADADA6EB7B6B7B7B76EB7B7B70B
:10361000B6B76E6EB7135C1CB76EB66EAE1413B74A
:103620006EAEAE6E6E141313AEB6AE65135CDA0BEF
:103630000B0A530B6DDADADADADADADADADADADA4C
:10364000DADADADADADA13B76EB7B66EB7DA6EB795
:10365000B6B7B7B76EB7B7B7B6B76E6EB7135C1C71
:10366000B76EB66EAE1413B76EAEAE6E6E141313A5
:10367000AEB6AE65135CDA0B0B0A530B6DDADADA11
:10368000DADADADADADADA1365AE6D5C5CDA13B755
:103690006EB7B66EB7DA6EB7B6B7B7B76EB7B7B7BD
:1036A000B6B76E6EB7135C1CB76EB66EAE1413B7BA
:1036B0006EAEAE6E6E141313AEB6AE65135CDA0B5F
:1036C0000B0A530B6DDADADA1365AE6D5C5CDA1354
:1036D000B76EB7B66EB7DA6EB7B6B7B7B76EDAB75A
:1036E000B7B6B76E6EB7DA5C1CB76EB66EAEDA13ED
:1036F000B76EAEAE6E6EDA1313AEB6AE6513DADA2F
:103700000B0B0A530B6DDADADA1365AE6D5CDADA9D
:1037100013B76EB7B66EDADA6EB7B6B7B7B7DADA2E
:10372000B7B7B6B76E6EDADA5C1CB76EB66EDADAB9
:1037300013B76EAEAE6EDADA1313AEB6AE65DADA82
:10374000DA0B0B0A530BDADADADA1365AE6DDADA72
:10375000DA13B76EB7B6DADADA6EB7B6B7B7DADA5F
:10376000DAB7B7B6B76EDADADA5C1CB76EB6DADAA1
:10377000DA13B76EAEAEDADADA1313AEB6AEDADA61
:10378000DADA0B0B0A53DADADADADA1365AEDADAF6
:10379000DADA13B76EB7DADADADA6EB7B6B7DADAD8
:1037A000DADAB7B7B6B7DADADADA5C1CB76EDADAD1
:1037B000DADA13B76EAEDADADADA1313AEB6DADAC9
:1037C000DADADA0B0B0ADADADADADADA1365DADA03
:1037D000DADADA13B76EDADADADADA6EB7B6DADA52
:1037E000DADADAB7B7B6DADADADADA5C1CB7DADA02
:1037F000DADADA13B76EDADADADADA1313AEDADA39
:10380000DADADADA0B0BDADADADADADADA13DADA7D
:10381000DADADADA13B7DADADADADADA6EB7DADA81
:10382000DADADADAB7B7DADADADADADA5C1CDADA7A
:10383000DADADADA13B7DADADADADADA1313DADA60
:10384000DADADADADA0BDADADADADADADADADADAA7
:10385000DADADADADA13DADADADADADADA6EDADAFB
:10386000DADADADADAB7DADADADADADADA5CDADA59
:10387000DADADADADA13DADADADADADADA13DADA36
:10388000DADADADADADADADA1365AE6D5C5CDA1330
:10389000B76EB7B66EB7B76EB7B6B7B7B76E13B782
:1038A000B7B6B76E6EB7145C1CB76EB66EAE1413B7
:1038B000B76EAEAE6E6E5C1313AEB6AE6513DADAEB
:1038C0000B0B0A530B6D5CDADA1365AE6D5CB7DA7D
:1038D00013B76EB7B66E6EB76EB7B6B7B7B7B713E6
:1038E000B7B7B6B76E6EAE145C1CB76EB66E6E141C
:1038F00013B76EAEAE6E135C1313AEB6AE656DDA73
:10390000DA0B0B0A530B5C5CDADA1365AE6D6EB73B
:10391000DA13B76EB7B6B76EB76EB7B6B7B76EB7DE
:1039200013B7B7B6B76E6EAE145C1CB76EB66E6EDC
:103930001413B76EAEAE65135C1313AEB6AE0B6D5B
:10394000DADA0B0B0A536D5C5CDADA1365AEB66E2D
:10395000B7DA13B76EB7B7B76EB76EB7B6B76E6EE6
:10396000B713B7B7B6B7B66EAE145C1CB76EAE6E13
:103970006E1413B76EAEAE65135C1313AEB6530B75
:103980006DDADA0B0B0AAE6D5C5CDADA1365B7B68A
:103990006EB7DA13B76EB7B7B76EB76EB7B6B76EA6
:1039A0006EB713B7B7B66EB66EAE145C1CB7AEAEDC
:1039B0006E6E1413B76EB6AE65135C1313AE0A5376
:1039C0000B6DDADA0B0B65AE6D5C5CDADA136EB791
:1039D000B66EB7DA13B7B6B7B7B76EB76EB7B6B7D6
:1039E0006E6EB713B7B7B76EB66EAE145C1C6EAE24
:1039F000AE6E6E1413B7AEB6AE65135C13130B0A3E
:103A0000530B6DDADA0B1365AE6D5C5CDADAB76E08
:103A1000B7B66EB7DA13B7B6B7B7B76EB76EB7B695
:103A2000B76E6EB713B71CB76EB66EAE145CB76EDA
:103A3000AEAE6E6E141313AEB6AE65135C130B0B05
:103A40000A530B6DDADADADADADADADADADADADA69
:103A5000DADADADADADAB7DADADADADADADA13DAB0
:103A6000DADADADADADA14DADADADADADADA14DA42
:103A7000DADADADADADA5CDADADADADADADADADA24
:103A8000DADADADADADA5CDADADADADADADAB7DA37
:103A9000DADADADADADA6EB7DADADADADADAB713FF
:103AA000DADADADADADAAE14DADADADADADA6E149A
:103AB000DADADADADADA135CDADADADADADA6DDA18
:103AC000DADADADADADA5C5CDADADADADADA6EB7E1
:103AD000DADADADADADAB76EB7DADADADADA6EB787
:103AE00013DADADADADA6EAE14DADADADADA6E6E33
:103AF00014DADADADADA65135CDADADADADA0B6DE2
:103B0000DADADADADADA6D5C5CDADADADADAB66E0E
:103B1000B7DADADADADAB7B76EB7DADADADA6E6ED5
:103B2000B713DADADADAB66EAE14DADADADAAE6EF9
:103B30006E14DADADADAAE65135CDADADADA530B53
:103B40006DDADADADADAAE6D5C5CDADADADAB7B61E
:103B50006EB7DADADADAB7B7B76EB7DADADAB76EDB
:103B60006EB713DADADA6EB66EAE14DADADAAEAE51
:103B70006E6E14DADADAB6AE65135CDADADA0A53A4
:103B80000B6DDADADADA65AE6D5C5CDADADA6EB76A
:103B9000B66EB7DADADAB6B7B7B76EB7DADAB6B79B
:103BA0006E6EB713DADAB76EB66EAE14DADA6EAEE0
:103BB000AE6E6E14DADAAEB6AE65135CDADA0B0A04
:103BC000530B6DDADADA1365AE6D5C5CDADAB76E78
:103BD000B7B66EB7DADAB7B6B7B7B76EB7DAB7B6A1
:103BE000B76E6EB713DA1CB76EB66EAE14DAB76E78
:103BF000AEAE6E6E14DA13AEB6AE65135CDA0B0BB6
:103C00000A530B6DDADA01011C01011501010201F1
:103C100002050602020708090A0202090A07080249
:103C20000208070A0902020A09080701020B0C012F
:103C3000020D0E02010F10020111120102130C01FC
:103C400002140E0202070811120202090A111202DE
:103C5000020807111202020A0911120201181902C0
:103C6000011A1B04020B0F100D0C11120E02021E82
:103C70001F202102012223020124250202262728D7
:103C80002902022A2B2C2D02022E2F303102023261
:103C900033343502023637383901023A3B03023CED
:103CA0003D3E3F404101024243010244450102467C
:103CB000470102484902014A4B02014C4D020216DB
:103CC000164C4D0402464A4B48474C4D4902024EA1
:103CD0004F50510C0152535455565758595A5B5C2A
:103CE0005D06025E5F6061626300646566000001FC
:103CF0000267680102696A01021A6B01021B6C0209
:103D0000016D6E02026769686A02021A1B6B6C021F
:103D10000207086D6E0202090A6D6E020208076D45
:103D20006E02020A096D6E03036F7071707070721B
:103D3000707303030708071A0A1B6B086C030367F9
:103D40000869680A6A07080704064A4B4A00160011
:103D5000004B16000016162E2F161630314D4D4C06
:103D60004D000406004A4B004B00004A1622231661
:103D700016161616160000164D00004C0406004AD2
:103D80004B3B4D00004A004D000000004D004D032C
:103D9000004D004D4C0004064A00004B1626271625
:103DA00016282916164A4B16160000164C00004D10
:103DB000020B0D00070D090A0714140000000D0086
:103DC000070D090A0914120E0601AABBA9A7BAB960
:103DD0000B01B9BAAFBAA9AE00AFB400030601B97E
:103DE000B6ABABAABF0901AAB8A7ADB5B4ACB2BF18
:103DF0000501ACB2B5A7BA0401B2ABA7B60601B1D2
:103E0000A7A8B5B5B30601B6B5AFB9B5B4070103F8
:103E100000ACB2AFABB90101C10101C202027475BD
:103E2000767778797A7B7C7D7E7F808182830201C0
:103E30008485868788898A8B02048C8D8E8F9091E9
:103E40000101929394959697010198998E8E909086
:103E500001019A9B94949696010102029C9D9E9F5B
:103E6000A0A1A2A30101A4A5A6A50E01A8BF00B60A
:103E7000A7BBB200B3A9B6AEABABB3BBB9AFA90099
:103E8000A8BF00ADB8A7A70000000000BBC0ABA84A
:103E9000B5BE0000000000B6B8ABB9B90000B9BAB1
:103EA000A7B8BA00FEFEFEFEFEFEFEFEFEFEFEFE11
:103EB000FEFEFEFEFEFEFEFEFEFEFEFEFEFEFEFE22
:103EC000FEFEFEFEFEFEFEFEFEFEFEFEFEFEFEFE12
:103ED000FEFEFEFEFEFEFEFEFEFEFE00FEFEFEFE00
:103EE000FEFE0000FEFEFEFEFEFEFEFEFEFEFEFEEE
:103EF000FEFEFEFEFEFEFEFEFEFEFEFEFEFEFEFEE2
:103F0000FEFEFEFEFEFEFEFEFEFEFEFEFEFEFEFED1
:103F1000FEFEFEFE00000052525252520052525B10
:103F20005B5B5B52FEFEFEFEFEFEFEFEFEFEFEFE46
:103F3000FEFEFEFEFEFE00FEFEFEFEFEFEFE520049
:103F40000000FEFEFE005200003F00FE0052000096
:103F50005252000000005252000000525252000023
:103F6000000CFFFEFEFEFEFEFE000000FEFEFEFE5A
:103F700000000000FEFEFE0052FE0000FEFEFE00FD
:103F8000FEFE0000FEFEFE00FEFE0000FEFEFEFE47
:103F9000FEFE5200FEFEFEFEFEFE0000FEFEFEFEE7
:103FA000FEFEFE00520000525252520052520000D9
:103FB000000000000052000000000000000000FEB1
:103FC000FEFE0000000000FEFEFEFE00FE0000FE01
:103FD000FEFEFEFEFE0000FEFEFEFEFE00FE0052A5
:103FE000FEFEFEFE52520000FEFE52FE0052000097
:103FF000FEFEFEFE000000FEFEFEFEFE000000FED5
:10400000FEFEFEFE00000000FEFEFEFE005252001C
:1040100052FEFEFE0052FEFE0000FEFE520052FE68
:104020005200FEFEFEFEFEFEFEFEFEFEFEFEFEFE5A
:10403000FEFEFEFEFEFE00FEFEFEFEFEFEFE520048
:104040000000FEFEFE005200003F00FE0052000095
:104050005252000000005252000000525B52000019
:10406000000CFFFEFEFEFEFEFE000000FEFEFEFE59
:1040700000000000FEFEFE0052FE0000FEFEFE00FC
:10408000FEFE0000FEFEFE00FEFE0000FEFEFEFE46
:10409000FEFE5200FEFEFEFEFEFEFE52FEFEFEFE96
:1040A000FEFEFEFE520000525252520052520000DA
:1040B000000000000052000000000000000000FEB0
:1040C000FEFE0000000000FEFEFEFEFE00FE0052AE
:1040D000FEFEFE000000000000FEFEFEFE0000529C
:1040E0000000FEFE5B520000FEFE52FE0052000089
:1040F000FEFEFEFE000000FEFEFEFEFE00000000D2
:104100000000FEFE00005B5B0000FEFE0052FEFEB3
:104110000000FEFEFEFEFEFEFEFEFEFEFEFEFEFEBB
:10412000FEFEFEFEFEFEFEFE00000000FEFE520051
:1041300052520000FEFE00FEFEFE0000FE00FEFEEB
:10414000FEFE0000FEFEFEFEFE000000FEFEFEFE85
:10415000FE0000FEFEFEFEFEFE000000FEFEFEFE75
:10416000FEFE000052000052525252005252000015
:1041700000000000005200000000000000000000ED
:104180005200000052000052FEFEFEFE520052FE9F
:10419000FEFEFE52520052FEFEFEFEFEFE520000E9
:1041A000FEFEFEFE5B520000FEFE52FE00520000CC
:1041B0000052FEFE000000000000FEFE00000000B5
:1041C0000000FEFE0000FEFE00FEFEFE0000FEFE01
:1041D000FEFEFEFEFEFEFEFEFEFEFEFEFEFEFEFEFF
:1041E000FEFEFEFEFEFEFEFEFEFEFEFEFEFEFEFEEF
:1041F000FEFEFEFEFEFEFEFEFEFEFEFEFEFEFEFEDF
:10420000FEFEFEFEFEFEFEFEFEFEFEFEFEFEFEFECE
:10421000FEFEFEFEFEFEFEFEFEFEFE52FEFEFE5216
:1042200000000000FEFEFEFEFEFEFEFEFEFEFEFEA6
:10423000FEFEFEFEFEFEFEFEFEFEFEFEFEFE00FE9C
:10424000FEFEFEFEFEFE52000000FEFEFE005200DC
:10425000003F00FE00520000525200000000525287
:10426000000000520000000000000000FEFEFEFE04
:1042700052000052FEFEFEFE00000052FEFEFE5204
:1042800000000000FE5B00000000005252005200DF
:1042900000FEFEFEFEFEFE0052FEFEFEFEFE5B0087
:1042A000FEFEFEFE520052525B5B52525200005222
:1042B00052520000000000000000000000525B525B
:1042C00000000000FEFEFEFEFE000000FEFEFEFE00
:1042D000FEFEFEFEFEFEFEFEFEFEFEFEFEFEFEFEFE
:1042E000FEFEFEFE52520000000CFFFE52000000D7
:1042F000FEFE52FE00000000FEFEFEFE000000007A
:104300000052FEFE0000000052000052FEFE0000BF
:1043100000FEFEFEFEFEFEFE000000FEFEFEFEFEB5
:10432000FEFEFEFEFEFEFEFEFEFEFEFEFEFEFEFEAD
:10433000FEFEFEFE00FEFEFEFEFEFEFEFE00FEFE99
:10434000FEFEFEFEFE5252FEFEFEFEFEFEFE0000E1
:1043500000000052FEFEFEFE5B000000FEFEFEFEC0
:10436000FE000000FEFEFEFEFEFEFEFEFEFEFEFE67
:10437000FEFEFEFEFEFEFEFEFEFEFEFEFEFEFEFE5D
:10438000FEFEFEFEFEFEFEFEFEFEFEFE000000FE47
:10439000FEFEFEFE00525252525252005200525B3A
:1043A0005B5B5B52FEFEFEFEFE000052FEFEFEFE6A
:1043B00000000000FEFEFE0000FE0000FEFE000009
:1043C00000525200FEFE0052FEFEFEFEFEFEFEFE0B
:1043D000FEFEFEFEFEFEFEFEFEFEFEFEFEFEFEFEFD
:1043E000FEFEFEFE520000525252525200000000E9
:1043F00000520000005252000000000052FEFEFE7B
:1044000000000000FEFEFEFEFEFE0000FEFEFEFEC0
:10441000FEFEFE00FEFEFEFEFEFEFE00FEFEFEFEB8
:10442000FEFEFE5252520000FEFE52FE52000052AC
:10443000FEFEFEFE00000052FEFEFEFE000000FE3C
:10444000FEFEFEFE000000FEFEFEFEFE5252005288
:10445000FEFEFEFE52FEFE000000FEFE0052FEFECC
:104460005200FEFEFEFEFEFEFEFEFEFEFEFEFEFE16
:10447000FEFEFEFEFEFEFEFEFEFEFEFEFEFEFEFE5C
:10448000FEFEFEFEFEFEFEFEFEFEFEFEFEFE000048
:1044900052FE0000FE0052FE00000000FEFEFEFE86
:1044A00052000052FEFEFEFEFEFEFEFEFEFEFEFE80
:1044B000FEFEFEFEFEFEFEFEFEFEFEFEFEFEFEFE1C
:1044C000FEFEFEFEFEFEFEFEFEFEFEFE00525BFE59
:1044D000FEFEFEFE52525252525252000000525BF9
:1044E0005B5B5B52FEFEFEFE00005252FEFE9DFE36
:1044F00000000052FE52000000000000FE0000001C
:1045000000000000520052FEFEFEFEFE0052FEFEC3
:10451000FEFEFEFEFEFEFEFEFEFEFEFEFEFEFEFEBB
:10452000FEFEFEFE000000525B5B5B5B00000000D5
:10453000005252520000000000000052FEFEFE0039
:1045400000000000FEFEFEFEFE000000FEFEFEFE7D
:10455000FEFE0000FEFEFEFEFE520052FEFEFEFECD
:10456000FE0052FE5B520000FEFE52FE520000FEB4
:10457000FEFEFEFE000000FEFEFEFEFE000000FE4F
:10458000FEFEFEFE0000FEFEFEFEFEFE0000FEFE43
:10459000FEFEFEFEFE000000FEFEFEFEFEFE000031
:1045A000FEFEFEFEFEFEFEFEFEFEFEFEFEFEFEFE2B
:1045B000FEFEFEFEFEFEFEFEFEFEFEFEFEFEFEFE1B
:1045C000FEFEFEFEFEFEFEFEFEFEFEFEFEFEFEFE0B
:1045D000FEFEFEFEFEFEFEFEFEFE0000FEFE0000F3
:1045E0005B5200000000FEFEFE520000FEFEFEFEDA
:1045F000FE520000FEFEFEFEFEFE5200FEFEFEFE2D
:10460000FEFEFE5BFEFEFEFEFEFEFEFEFEFEFEFE6D
:10461000FEFEFEFEFEFEFEFEFEFEFEFEFEFEFEFEBA
:10462000FEFEFEFE52000052525B5B5252520000F0
:104630000000525200525200000000000000000032
:10464000000000525200000000FE0000520000FE78
:1046500000000000FE52000000000000FEFE9D0071
:1046600000525B5B52000000FEFE52FE00000000A4
:10467000FEFEFEFE00000052FEFEFEFE000000FEFA
:10468000FEFEFEFEFE0052FEFEFEFEFE0052FEFE9E
:10469000FEFEFEFE52FEFEFEFEFEFEFEFEFEFEFEE6
:1046A000FEFEFEFEFEFEFEFEFEFEFEFEFEFEFEFE2A
:1046B000FEFEFEFEFEFEFEFEFEFEFEFEFEFEFEFE1A
:1046C000FEFEFEFEFEFEFEFEFEFEFEFEFEFEFEFE0A
:1046D000FEFEFEFEFEFE090909090909525BA4A4BB
:1046E000A4A45B09FEFEFEFEFEFEFEFEFEFEFEFE36
:1046F000FEFEFEFEFEFEFEFEFEFEFEFEFEFEFEFEDA
:10470000FEFEFEFEFEFEFEFEFEFEFEFEFEFEFEFEC9
:10471000FEFEFEFEFEFEFEFEFEFEFEFE09FEFEFEAE
:10472000FEFEFEFEFE525B5B5B5BA4A4FEFEFEFE95
:10473000FEFE525BFEFEFEFEFE5D5E5DFEFE10288E
:1047400030185D67FE1038281808FE031038201056
:10475000FEFE04FE302010FEFEFEFE042010FEFED3
:10476000FEFEFEFE09FEFE5E40FEFEFEA45D5DFF57
:10477000C040FEFE5D5E675EFF5DFEFE045EFE5EA7
:104780005D67FEFE0703FEFEFEFE67FE04FE04FEFE
:10479000FEFEFE67FE04FEFEFEFEFEFEFEFEFEFECA
:1047A000FEFEFEFEFEFEFEFEFEFEFEFEFEFEFEFE29
:1047B000FEFEFEFEFEFEFEFEFEFEFE52FE525BA46E
:1047C000FEFE5252FE525B5BA4FE5252FEFE525B54
:1047D0005BA45252FEFEFE525B5BA452FEFEFEFE46
:1047E000FE525BA4FEFEFEFEFEFEFEFEFEFEFEFE92
:1047F000FEFEFEFEFEFEFEFEFEFEFEFE52FEFEFE85
:10480000FEFEFEFE52FEFEFEFEFEFEFE52FEFEFE20
:10481000FEFEFEFE52FEFEFEFEFEFEFE52FEFE5EB0
:1048200040FEFEFEFEFEFEFE30185252FEFE102836
:1048300018105E5DFE103028FEFE5D6710382010F7
:10484000FEFEFE03302010FEFEFE04FE2010FEFEE3
:10485000FEFEFE04FEFEFEFEFEFEFEFEFEFEFEFE72
:10486000FEFEFEFEA45D5DFFC040FEFE5D5E675E77
:10487000FF5DFEFE045EFE5E5D67FEFE0703FEFE5C
:10488000FEFE67FE04FE04FEFEFEFE67FE04FEFE64
:10489000FEFEFEFEFEFEFEFEFEFEFEFEFEFEFEFE38
:1048A000FEFEFEFEFEFEFEFEFEFEFEFEFEFEFEFE28
:1048B000FEFEFEFEFEFEFEFEFEFEFEFEFEFEFEFE18
:1048C000FEFEFEFEFEFEFEFEFEFEFEFEFEFEFEFE08
:1048D000FEFEFEFEFEFEFEFEFEFEFEFEFEFEFEFEF8
:1048E000FEFEFEFEFEFEFEFEFEFEFEFEFEFEFEFEE8
:1048F000FEFE5BA4FEFEFEFE525BA4A4FEFE08527A
:104900005BA4A467FE08525BA4A4FE0318285BA462
:10491000A4FE04FE281808FEFEFEFE041808FEFE93
:10492000FEFEFEFEFEFEFE5D5D5E5E1DFEFE1D5E8B
:1049300066666666FE1D5E66666666665D5D5D5EF3
:10494000666666665D5D655D5E66665EFE28181875
:104950001D5D1D5DFE283828FEFEFEFEFE2828286F
:10496000FEFEFEFE5DFEFEFEFEFEFEFE5E5D5DFEEA
:104970002828FEFE665E1528FF8028185E5D5D28EB
:10498000383828285D655D28282818FE281818FE64
:10499000FEFEFEFE283828FEFEFEFEFE282828FE2B
:1049A000FEFEFEFEFEFEFE5D5D5E5E1DFEFE1D5E0B
:1049B00066666666FE1D5E66666666665D5D5D5E73
:1049C000666666665D5D655D5E66665EFE281818F5
:1049D0001D5D1D5DFE283828FEFEFEFEFEFE282819
:1049E00028FEFEFE5DFEFEFEFEFEFEFE5E5D5DFE40
:1049F0002828FEFE665E1528FF8028185E5D5D286B
:104A0000383828285D655D28282818FE281818FEE3
:104A1000FEFEFEFE283828FEFEFEFEFEFE282828AA
:104A2000FEFEFEFEFEFEFE5D5D5E5E1DFEFE1D5E8A
:104A300066666666FE1D5E66666666665D5D5D5EF2
:104A4000666666665D5D655D5E66665EFE28181874
:104A50001D5D1D5DFE283828FEFEFEFE282828FE6E
:104A6000FEFEFE285DFEFEFEFEFEFEFE5E5D5DFEBF
:104A70002828FEFE665E1528FF8028185E5D5D28EA
:104A8000383828285D655D28282818FE281818FE63
:104A9000FEFEFEFE283828FEFEFEFEFE2828FEFE54
:104AA000FEFEFEFEFE665EFEFE38FEFE6F5D665E8C
:104AB000FE1818FE66665E6628FF40186F6F665E19
:104AC0006618382866665E6F5E3818FE6F6F6F6610
:104AD0005D38FEFEFE5E5E5D3828FEFE2838383802
:104AE000383818FE00010203040500010607080912
:104AF0000001060A0B0C0D010E0F10111213021407
:104B00001516171802191A1B1C01021D1E1F202141
:104B1000222324252627282829232A2B2C2D2E2F13
:104B2000300603020100000000E44A06030206000A
:104B3000000400EA4A04020203000004000E4B02D3
:104B4000020103000008001A4B010101010000806E
:104B500000204B02020104000008012E3E0802045E
:104B60000400000801383E01010104000010016446
:104B70003E04020202000008005A3E040202040041
:104B8000000A001C3E0101010400001000643E0EFA
:104B90000E0104000080006A3E00020B0008550070
:104BA000030C0104020104020104020104020104D5
:104BB00002010402010402010402010402010402D0
:104BC00001040201040201040201040201040201C1
:104BD000050000FF0007FF0002030000FC0008289A
:104BE000010405010404010403010402010401009D
:104BF0000990000A60020401020401020401020497
:104C00000102040102040102040102040102040180
:104C10000204010204010204010204010205000071
:104C2000FF0000FB00083C02030602030602030625
:104C300004050000FF0002020008530007FF0009FE
:104C400090000A3C0204060203060000F600FF0082
:104C500000FB0008320204060204060204060405F2
:104C60000000FF0002020000F702030C02040C0126
:104C7000030C03040C01030C02040C01030C0304D9
:104C80000C01030C02040C02030C02040C01030CC3
:104C900003040C00FF0000E7000106030105010109
:104CA0000100FF0007FE0000E70001080101070204
:104CB00001050101010B078A0000DD00010001016F
:104CC000010607EE0000F20001000101010D078A54
:104CD0000000DD0001000101010607FE0000E70001
:104CE00001320101070201050101010B078A0000E1
:104CF000DD0001000101010607EE0000F2000100E5
:104D00000101010D078A0000DD000100010101051C
:104D1000050000FF0000DD000100010101070500A2
:104D200000FF0000F100010001010100FF0002028C
:104D30000000F10400F800FF000202000960000A10
:104D40001E0000F800FF0002020000F6010303024B
:104D50000304010407020303010304010407010320
:104D60000301030402040701030301030401040710
:104D70000103030203040104070103030103040107
:104D800004070203030103040104070103030103F1
:104D90000402040701050000FF0002020000F60102
:104DA00003040103030104070203040103030104D4
:104DB00007010304010303020407010304020303C0
:104DC00001040701030401030301040702030401B2
:104DD00003030104070103040103030204070103A1
:104DE0000401030301040701050000FF00020101A3
:104DF00006000100E200FF000201150402070302A1
:104E0000160404070304160402070302240700071C
:104E100003030007FF0F07000704030007FF0E0747
:104E20000000FF000000634C00000000010000953E
:104E30004C00000000000000A34C00000000010036
:104E400000144D00000000010000224D0000000091
:104E50000000002D4D00000000000000384D000053
:104E60000000000000464D00000000000000994DC9
:104E700000000000000000F74D00000000000000EE
:104E8000EC4D00000000000000994B000000000005
:104E90000000D44B00000000000000214C00000086
:104EA00000000000354C000000000000004F4C00E6
:104EB00000000000FF06015300C00600B0075400C8
:104EC0005C0100C10500B1075000C20900B20766CD
:104ED00000C30000B3072601C0060090247F00C273
:104EE000090092307F0093025E08C1050D90307F6B
:104EF00016247F0E2E7F162E7F07247F0193025EDD
:104F00000D90307F08247F0E2E7F16247F07267F8A
:104F10000E277F07247F0092307F0093025E169059
:104F2000307F16247F0E2E7F16227F0693025E01AD
:104F300090247F0E307F07247F0F2E7F15247F085B
:104F4000267F0E277F0693027F0190247F009148E1
:104F50007F0092307F07914A7F084B7F0790307F18
:104F600000914D7F1590247F0F2E7F182E7F049384
:104F7000027F0190247F0E307F07247F0F2E7F1544
:104F8000247F07267F0091417F08437F0790277F7A
:104F90000091447F0790247F0091487F0092307FEA
:104FA0000093027F07914A7F074B7F0890307F0074
:104FB00091507F074B7F074A7F0790247F00914BDA
:104FC0007F074A7F08902E7F0091487F074A7F071E
:104FD000487F0790227F0091467F0790247F0091B1
:104FE000487F0093027F0F90307F07247F0E2E7F33
:104FF00016247F07267F0F277F0693027F019024C8
:105000007F0091487F0092307F07914A7F074B7F56
:105010000790307F0091507F1690247F0E2E7F1ACC
:105020002E7F0293027F0190247F0F307F07247F21
:105030000E2E7F16247F0091487F0790267F0091D7
:105040004A7F074B7F0790277F00914D7F07930290
:105050007F0190247F0091547F0092307F0791520E
:105060007F07547F0790307F0091507F07547F085F
:105070004F7F0790247F0091527F074D7F07902E2E
:105080007F0091527F074B7F08527F0790227F005D
:10509000914A7F0693027F0190247F0091487F0E02
:1050A00090307F08247F0E2E7F16247F07267F07EF
:1050B000C1000790277F07247F0091487F0092302E
:1050C0007F0093027F1690307F16247F0091487FE7
:1050D0000E902E7F16913C7F03902E7F02C105011A
:1050E00093027F0190247F0091487F0E90307F00D3
:1050F00091447F0790247F0091467F0F902E7F0080
:10510000914B7F1590247F08267F00914F7F0CC123
:10511000000290277F0693027F0190247F00915424
:10512000640092307F1690307F15247F0091546484
:105130000F902E7F07913C7F0C487F01C1050190A5
:10514000227F0091487F0693027F0290247F009186
:105150004A7F074B7F0790307F00914A7F0790245A
:105160007F0091487F0F902E7F0791487F0E9024FB
:105170007F00913C7F0790267F00913C7F0F902716
:105180007F00913C7F04C1000293027F0190247F45
:105190000091487F0092307F1690307F15247F0069
:1051A00091487F0F902E7F15913C7F04902E7F01B8
:1051B000C1050193027F0190247F0091487F0F90E9
:1051C000307F0091447F0790247F0091467F0E90AE
:1051D0002E7F00914B7F11902E7F05247F07267F25
:1051E00000914F7F0F90277F02C1000590247F0020
:1051F0009154640092307F0093027F1590307F16A7
:10520000247F009154640E902E7F08913C7F0C48BF
:105210007F01C1050190227F0091487F0790247F84
:1052200000914A7F0093027F07914B7F0890307F67
:1052300000914A7F0790247F0091487F0E902E7F37
:105240000791487F0F90247F00913C7F0790267F35
:1052500000913C7F0E90277F00913C7F0793027F57
:1052600001C0070090487F00913C7F0092307F078B
:10527000913E7F073F7F0790487F0091417F073F26
:105280007F083E7F073C7F07417F07437F07447FBE
:1052900008437F07417F0693027F0190467F00917C
:1052A000487F07437F07447F0890467F0091467FF1
:1052B00007437F07447F073C7F07377F08307F071E
:1052C000377F07387F073A7F0790437F00913C7F05
:1052D0000092307F0093027F08913E7F073F7F0757
:1052E00090437F0091417F073F7F073E7F08487FC3
:1052F000074A7F074B7F0790437F00914D7F074B05
:105300007F084A7F0693027F01C0080090447F0017
:1053100091487F07437F07447F0790447F0091486F
:105320007F08437F07447F07487F074B7F074A7FFB
:1053300008487F15C0070090487F00913C7F00928D
:10534000307F0093027F07913E7F083F7F079048A0
:105350007F0091417F073F7F073E7F073C7F0841E9
:105360007F07437F07447F07437F07417F079302FF
:105370007F0190467F0091487F07437F07447F0766
:1053800090467F0091467F07437F08447F073C7F1C
:1053900007377F07307F07377F08387F073A7F0757
:1053A00090437F00913C7F0092307F0093027F0703
:1053B000913E7F073F7F0890437F0091417F073FE9
:1053C0007F073E7F07487F074A7F084B7F07904350
:1053D0007F00914D7F074B7F074A7F07C0080090F1
:1053E000447F0091487F0093027F0891437F0744E8
:1053F0007F0790447F0091487F07437F07447F08E1
:10540000487F074B7F074A7F07487F0EC00704C1CC
:10541000000490487F0091487F0093027F159048D8
:105420007F1691487F243C7F05487F00C10502908C
:10543000467F0091487F0093027F0F91447F079041
:10544000467F0091467F0E4B7F1D4F7F14C10002A7
:1054500090437F009154550093027F1590437F162F
:105460009154551590437F00913C7F0C487F01C1BA
:10547000050291487F01C0080690447F00914A7F51
:105480000093027F07914B7F074A7F0890447F007B
:1054900091487F15487F0F3C7F073C7F0E3C7F0281
:1054A000C00703C1000290487F0091487F0093022B
:1054B0007F1690487F1691487F243C7F06C10500E7
:1054C00093027F0190467F0091487F0E447F0790B2
:1054D000467F0091467F0F4B7F1D4F7F11C1000417
:1054E00090437F009154550093027F1690437F159F
:1054F0009154551690437F00913C7F0C487F01C129
:10550000050191487F04C0080393027F0190447F06
:1055100000914A7F074B7F074A7F0790447F0091A5
:10552000487F16487F00922B7F0E913C7F073C7F7F
:1055300000922E7F0F913C7F02C0070590487F00AC
:1055400091307F0092307F0093027F1690487F0059
:10555000912E7F15247F16307F1590467F00912E67
:105560007F0093027F1690467F0091307F16337F35
:1055700015307F1690437F0091307F0092307F007E
:1055800093027F1590437F00912E7F16247F169003
:10559000437F00912B7F12C0080390447F00912E1F
:1055A0007F0093027F1690447F0091377F15337FF1
:1055B00016307F0E2E7F02C0070690487F00913084
:1055C0007F0093027F1590487F00912E7F16247FE5
:1055D00015307F1690467F00912E7F0093027F1634
:1055E00090467F0091307F15337F16307F159043B2
:1055F0007F0091307F0093027F1690437F00912EB1
:105600007F16247F1590437F00912B7F12C00803E3
:1056100093027F0190447F00912E7F1590447F007C
:1056200091377F16337F16307F0E2E7F06FF0601DF
:105630004501FF2F0001040C3C04060C3C0D010C3D
:105640003C1B039D3C03040C3C0A06CD3C0C0D0C9A
:105650003C0E029D3C11060C3C16010C3C19039DAE
:105660003C1B0D0C3C0A050C3C0D029D3C16020C2B
:105670003C02019D3C11020C3C0704933C0904933D
:105680003C0B04933C0D04933C1104933C13049392
:105690003C1504933C1704933C0C020C3C13030C84
:1056A0003C03020C3C17020C3C0406933C0D020C1C
:1056B0003C19115B3C06050C3C0D155B3C1C030CB6
:1056C0003C0A020C3C10125B3C0F020C3C16030C13
:1056D0003C1C065B3C16105B3C04010C3C1504931F
:1056E0003C1A010C3C0F055B3C19020C3C15010CEB
:1056F0003C1D04933C08010C3C0B165B3C14010C54
:105700003C1A0A0C3C05165B3C110A0C3C12165B59
:105710003C1C0C0C3C02020C3C040C933C05049D0C
:105720003C0E030C3C17060C3C180C933C19019DD5
:105730003C03040C3C06049D3C0D060C3C140D5B24
:105740003C19050C3C1A029D3C04080C3C08010C59
:105750003C0B029D3C100C933C140C933C1D010C23
:105760003C1C059D3C04020C3C07039D3C0F040CB3
:105770003C14029D3C1A020C3C09050C3C0B039D99
:105780003C1A050C3C04019D3C0B0A0C3C18040C13
:105790003C1B039D3C03020C3C0A060C3C0D019D86
:1057A0003C15030C3C03030C3C07019D3C14030C0B
:1057B0003C01075B3C04020C3C1A080C3C07090C3A
:1057C0003C0C010C3C1E030C3C0A010C3C1A020C64
:1057D0003C07039D3C14049D3C0A030C3C17070C3A
:1057E0003C05029D3C0C040C3C130C5B3C16060C67
:1057F0003C17019D3C03040C3C11060C3C130C0CA3
:105800003C1A020C3C03020C3C0C010C3C0C0A5BE5
:105810003C0F040C3C17020C3C1A09933C050E0C7F
:105820003C08030C3C15020C3C160A5B3C1D0D0C9D
:105830003C03030C3C0B095B3C14020C3C1A089320
:105840003C1D050C3C02010C3C0508933C0D030C6F
:105850003C1508933C1B020C3C03095B3C0A020C00
:105860003C0B020C3C0C020C3C0A040C3C0B040CE0
:105870003C0E020C3C10020C3C0E060C3C10060CBC
:105880003C13030C3C14040C3C16060C3C17095B3F
:105890003C0308933C0C020C3C0D020C3C0E020C29
:1058A0003C0C060C3C0D060C3C0E060C3C0E050C8C
:1058B0003C0E040C3C0D040C3C11020C3C12020C7E
:1058C0003C11060C3C12060C3C1708933C02030CDE
:1058D0003C03080C3C0706933C0E060C3C0F110CD5
:1058E0003C1B000C3C1B04CD3C1B110C3C1C080C4D
:1058F0003C040C483D0A0C623D100C7C3D160C9695
:105900003D03056D3C030A733C030E063C03118DF9
:105910003C1401993C1405873C14097B3C140E0986
:105920003C150E093C0502C83D0506D03D050ADDC3
:105930003D050EE53D0512F03D1602F73D1606FD4C
:105940003D160A053E160E0D3E16120D3E03010CC5
:105950003C0409933C0E070C3C15000C3C180993C1
:105960003C1B040C3C2B3C333C2F3C133CF73CFBD6
:105970003C1B3DE13C873C0F3D813C5F3C773CFF5D
:105980003C0F3C153D253C193C993C373C493C3F7C
:105990003C3B3C6D3C8D3C1F3C733C433CEF3CF33B
:1059A0003C323D3D3D7B3C213D033D093DC33CAD8B
:1059B0003CB13CB53CB93CA53CA93CBD3C633C4832
:1059C0003D623D7C3D963D4F3CB03D553C0500055C
:1059D00001060003000400010001000200020001B2
:1059E000000500010002000300040005000600029B
:1059F0000004000C00020006000200110013000861
:105A00000002000100010001000300040002000385
:105A10000005000100030001000200010002000275
:105A2000000700070108000300040004010300044C
:105A3000000401050001000100010008000100014F
:105A4000000200000006000B000D000F0001000323
:105A5000000400010001010001010203010402062B
:105A60000107030A010B010C020E0210031302408E
:105A700020380204B8E8304040184001022050307D
:105A8000384090D001FEA8C030384020880102384C
:105A90004840484040800202405078804070C00139
:105AA0000480A0283040206C020240603038811809
:105AB0004802023050208081285802FE789850B069
:105AC0008118480202C0E0389840389C02FE18381D
:105AD00038404018C001FC28483848403878020255
:105AE000586848504088D801FCC0D02838401898E1
:105AF00001F890A820384050D001F8C8E020384084
:105B0000189001FC889028384040B801FCB0B828B3
:105B1000384068E001FCD8E0283840184802027894
:105B200088203040407002027888485801010009FE
:105B30000A0B000D090A0A0B0103000A0B190100E8
:105B4000090A000201010A1A000101021A1B0002DF
:105B500002000A1A011002010A1A101400010A1A9E
:105B6000141900011A201719000B1A1B0A0B010146
:105B70001B200A0B01031A200B1501041A1B151711
:105B800001061B2015170101000C0A0B0103000C74
:105B90000B150109000C151701020C0D0A0C01016F
:105BA0000C140C0D01030C140D1501060C13151724
:105BB000010513141517010214150C0E0001001431
:105BC0001719820214201112000A14201112000168
:105BD000142012190107191F0E10810804060D0F59
:105BE0000102040A0F118107040A0F110208040AB6
:105BF0000F11820200201112030A0020111200016D
:105C000000201219820416180A0C040016180A0C37
:105C10000107141A0C0E820200201112050A00203E
:105C200011120001002012190107040A0B0D0107CF
:105C3000161C0A0C810A14161517060114161517DE
:105C4000010B141617188202001C1112070A001CFF
:105C500011120001001C12198204080A0709080029
:105C6000080A07090107060C090B010710160709A6
:105C700001001B1C060800011C20131901011C2037
:105C8000060701031C20071381031C201319090CAC
:105C90001C20131901010020060701030020071230
:105CA000010D0020121300010020131982040F11AE
:105CB00004060A000F110406810C050716170B03D2
:105CC00005071617010B05071718820500200C0D94
:105CD0000C0A00200C0D000100200D19010E00041B
:105CE00006088108070904060D02040C0608810E47
:105CF000040C06080E08040C0608010E0C12060817
:105D00008108151704060F02121A0608810E121ACE
:105D100006081008121A0608010E1A2006080101CA
:105D20000008060701030008070F010400010F1116
:105D3000010F01070F11010507080F11006800018D
:105D40001516011001071516006A0708151601033C
:105D500000081619010E080F0608000100081115A9
:105D6000820208200C0D110A08200C0D00010820E9
:105D70000D19820200200C0D120A00200C0D0001EA
:105D800000200D19820413150406130013150406D0
:105D900001001F20080A0101000908090103000988
:105DA0000912010900081214010508091214000162
:105DB000000F14198202090F1112140A090F11128F
:105DC0000001090F1214820411130E101500111393
:105DD0000E1001010F17101101030F171119010205
:105DE00017181012010117181213010317181319AD
:105DF0000101181B12130111181B131901021B1C9E
:105E0000121401011B1C141501111B1C1519010191
:105E10001C20141501111C201519010E0920080A57
:105E200001010003141501110003151901020304F7
:105E300014160101030416170103030417190101C5
:105E40000411161701030411171981120A0B1416F5
:105E500016050A0B1416010010110E10010111187D
:105E60000E0F010311180F1982040E1003051700FD
:105E70000E100305820415170C0E180015170C0ED2
:105E800001001718080A0101181A08090111181A47
:105E90000919801C1B1C121319061B1C121301016B
:105EA0001A20080901111A20090C01131A200C0DDF
:105EB00001111A20131901110004090B0114000328
:105EC0000B0D011503040B0D0111000413198203BE
:105ED000000407091A0D000407098205040E1415B1
:105EE0001B0A040E14150001040E1519810A04067C
:105EF00015171C0104061517010B040617180103DA
:105F00000E1C13158117161811131D0716181113DF
:105F10008118191B11131E04191B111300010E20E7
:105F2000151901160E0F080A011B0F20080A82031B
:105F30000E2006081F0D0E20060801031C200E155A
:105F4000010300020E15010100200708011B0020BB
:105F5000080A820302080F11200D02080F11010325
:105F6000020C111501030C0D111301050C0D131575
:105F700000010012151982050D121112210A0D12CD
:105F8000111200010D12121501031220111300014C
:105F900012201319810312201319220C1220131935
:105FA000010100020708000D02030708011B00029F
:105FB000080A01150203080A010300101113000169
:105FC00000201319011E0A0D131681180E100F114F
:105FD00023040E100F1101000F100608011F1417E3
:105FE0001619011E1D2013160101102006070103BA
:105FF0001020071301010005060701030005071320
:106000008205050E0809240A050E080981080709FA
:1060100004062502050E06098110050E0609260E46
:10602000040400000001050E0911810A0C0E0F1175
:1060300027010C0E0F11801D0A0B101128060A0BE8
:106040001011000100201319810A050716182901F3
:1060500005071618010B05071819011E0D10131658
:10606000011F171A161901010E10060701110E1053
:1060700007110102101106088120151704062A01D4
:106080001517040601001516060801021617060862
:106090008204191B06082B00191B06088205101C18
:1060A00008092C0A101C08090001101C0911000124
:1060B0001C200C1101001B1C0002011105201113F2
:1060C00001011C20000101031C20010A01041C1D08
:1060D0000A0C010F1D200A0C01010020000101091A
:1060E00000200103010300201719000100200317FD
:1060F00001030406020901230406090B01030A0C2B
:10610000020901230A0C090B01030D0F11170122CB
:106110000D0F0F11010313151117012213150F1184
:1061200001031618020901231618090B01031C1E8E
:10613000020901231C1E090B0001001000120101BD
:1061400000040001010900040103011C00011214F4
:106150000103000114190119010E121901010409AA
:106160000001010304090103010404050305010FF3
:10617000050903050101090E00010119090E0105B8
:106180000104090A050701090A0E050701010E109D
:10619000000101030E10010901230E10090B010279
:1061A000101100028205101608092D0A10160809A0
:1061B00000011016090E010015160608011C0E0F2D
:1061C0000E1001030E0F101901110F160E19010107
:1061D0001620060701031620071901010002060711
:1061E000010300020719000D020306070103020361
:1061F00007190107111707090111032017190103D6
:10620000001B17190107090F0E108204151702044D
:106210002E001517020401001A1B0E1001011B208D
:106220000E0F01111B200F19010100200E0F010399
:1062300000200F1982040E1007092F000E10070905
:1062400081120E0F0C0E30050E0F0C0E01010020F6
:106250000E0F010300200F1982040F1103053100F6
:106260000F110305010100200E0F010300200F197B
:1062700082041517030532001517030501010006F6
:106280000E0F010300060F19010206070E10010789
:106290000F150D0F8204191B090B3300191B090B75
:1062A000820206201011340A062010110001062077
:1062B0001119010700060D0F820200201011350A86
:1062C0000020101100010020111982040B0D090B90
:1062D00036000B0D090B010712180D0F82041D1F4C
:1062E000090B37001D1F090B820200201011380A0C
:1062F000002011190001002011190107040A0D0FD7
:1063000082041012090B39001012090B0107161C28
:106310000D0F8202002010113A0A00201011000116
:1063200000201119820404060A0C3B0004060A0C22
:10633000012403070C0E01240F130B0D01241B1F56
:106340000A0C8202001710113C0A001710110001FC
:10635000001711198204080A07093D00080A0709F5
:106360000124070B090B81080C0E07093E020B0FD5
:10637000090B81240B0F090B3F080B0F090B810A36
:106380000F11141640010F111416010B0F111617DF
:1063900001251617080A811A1B1D070841031B1D3A
:1063A00007080127172008090016172009190127D7
:1063B0000007080900160007091901260708080A3E
:1063C0008204080A0B0D4200080A0B0D80150D12FD
:1063D0000C0D430D0D120C0D012707170D0E0016A5
:1063E00007170E19012617180D0F8117141603052C
:1063F00044071416030501241317050781201C1EEA
:106400000F1145011C1E0F11012717201112001634
:106410001720121901251E1F000201271F2000014D
:1064200000161F20010501291F2005070127001163
:1064300000010016001101060128001106070127BE
:1064400000031112001600031219012502030F1197
:10645000012703100F10012610110F110016031051
:106460001011001603101119012710201119001620
:106470001020121901271120000100161120010817
:106480000129111207090128121F0809012A1F20DA
:10649000070901260001000201270006111200165B
:1064A00000061219012606071113811805070305B6
:1064B00046040507030501240408050701251112F8
:1064C000070902001220081302011220131700010D
:1064D00012201719820506121314470A0612131404
:1064E000000106121419012712200708800010204D
:1064F0001314480A102013140127002007088000F5
:1065000000201314490A0020131482040305020416
:106510004A000305020402000020081302010020C3
:106520001317000100201719012700200708800019
:10653000002013144B0A00201314820403050204E4
:106540004C00030502040200001E08130201001E95
:1065500013170001001E171902021E201314000158
:106560001E20141901261E1F070982020020131481
:106570004D0A0020131400010020141901240509FC
:106580000E10012415190E108202002013144E0A59
:1065900000201314000100201419012404080E1017
:1065A00001240F130E1001241A1E0E108202000780
:1065B00013144F0A000713140001000714190124D3
:1065C00003071012012506070D0F0127071B0D0EEB
:1065D0000016071B0E1980150C110C0D500D0C1117
:1065E0000C0D01261B1C0D0F82021B201314510AD7
:1065F0001B20131400011B20141982020020131405
:10660000520A002013140001002014190107080E7B
:106610000B0D0107171D0B0D820200051314530A01
:1066200000051314000100051419010004050B0DE9
:10663000010105200B0C010305200C1901020001CA
:106640000B0D820200201314540A002013140001C1
:1066500000201419012C070B0B0D012C15190B0D23
:1066600001001F200A0C010100200A0B0103002079
:106670000B19010100200A0B010300200B19010175
:1066800000200A0B010300200B190002090A02076F
:1066900000020F1002070002121302070002151673
:1066A000020700021C1E000A010100200A0B010360
:1066B00000200B1900020B0C020700021011020748
:1066C00000021314020700021C1E000A020500202B
:1066D0001516000100201619010004050002010131
:1066E000050A00010103050B010201190507020853
:1066F0000103050708090101070A08090131050A14
:10670000090B01320A0C000B0103070A05060204FB
:106710000D0F090B000B11120001010112180001ED
:10672000000D1819000101031119010201101113C4
:10673000020901161112090B01331218090B011578
:106740001819090B000B17190708000D171907086E
:10675000010317190809020313170709011617186F
:10676000020401151819020402041A1C090B011273
:1067700013140B0C0206081614158205000A1314D4
:10678000550A000A13140001000A1419000B0A0B21
:10679000131401010B20131401030A20141902041D
:1067A00003050103020314161113010100200B0C51
:1067B000010D00200C0D020000200D15020100202B
:1067C000151901070C12020401030000000A0A193E
:1067D00006000A000003000A01010300090A000282
:1067E000010104000A1A0001010105001A1B000240
:1067F000000306000A1A0119060009000A1A1114FA
:10680000000109001A20171901050A001A200A17A9
:1068100006010A000104001901030F00000C0A1709
:10682000010112000C0D0A0C010413000C140C17CA
:106830000101170014150C0E00011800001417199F
:10684000800319001420111911011C00191F0E10CA
:10685000060009001420111480021D0004060D0F0B
:1068600091021F00040A0F110600090000201114F4
:1068700080032100002011198002240016180A0C40
:1068800011012600141A0C0E060009000020111434
:10689000800327000020111911012A00040A0B0DA2
:1068A00011012B00161C0A0C80022C00141615175F
:1068B00001012E001416171806000900001C1114FF
:1068C00080032F00001C111980023200080A0709FA
:1068D00011013400060C090B1101350010160709CF
:1068E000010136001B1C0608000137001C2013198B
:1068F000010238001C20061380023A001C201319E4
:1069000001033C000020061300013F000020131982
:10691000800240000F11040680024200050716178E
:1069200001014400050717180600090000200C0F9C
:106930008003450000200C190101480000040608EE
:10694000800249000709040680024B00040C060877
:1069500001014D000C12060880024E0015170406B6
:1069600080025000121A0608010152001A2006087F
:10697000010553000008061101045800000815190C
:1069800001015C00080F060800015D0000081115F8
:106990000600090008200C0F80035E0008200C1977
:1069A0000600090000200C0F8003610000200C1974
:1069B0008002640013150406010166001F20080A06
:1069C000010467000009081400016B00000F14198E
:1069D00006000900090F111480036C00090F11143F
:1069E00080026F0011130E10010571000F181019AD
:1069F00001057600181C121901027B001C201419D5
:106A000001017D000920080A01057E000004141917
:106A10000102830004111619800285000A0B141666
:106A20000101870010110E100102880011180E19C3
:106A300080028A000E10030580028C0015170C0ED0
:106A400001018E001718080A01028F00181A081990
:106A5000800291001B1C1213010393001A20080DE1
:106A6000010196001A201319010397000004090D73
:106A700001019A000004131980029B000004070919
:106A800006000900040E131680039D00040E14195D
:106A90008002A000040615170101A20004061718C1
:106AA0000101A3000E1C13158002A4001618111377
:106AB0008002A600191B11130001A8000E20151951
:106AC0000102A9000E20080A8002AB000E20060871
:106AD0000101AD001C200E150101AE0000020E15D3
:106AE0000102AF000020070A8002B10002080F1166
:106AF0000103B300020D11150001B60000121519B3
:106B0000060009000D1210138003B7000D121115B5
:106B10000001BA00122013190101BB001220111349
:106B20008002BC00122013190104BE000003070AF2
:106B30000101C200001011130001C300002013194D
:106B40000101C4000A0D13168002C5000E100F11BA
:106B50000101C7000F1006080101C800141716191B
:106B60000101C9001D2013160102CA0010200613DE
:106B70000102CC000005061306000900050E070AF5
:106B80008002CE00050E08098002D0000709040625
:106B90008002D200050E06090001D400050E09117D
:106BA0008002D5000C0E0F118002D7000A0B1011C5
:106BB0000001D900002013198002DA000507161819
:106BC0000101DC00050718190101DD000D10131685
:106BD0000101DE00171A16190102DF000E1006115E
:106BE0000101E100101106088002E20015170406F9
:106BF0000102E400151706088002E600191B0406CE
:106C000006000900101C070A8003E800101C081188
:106C10000001EB001C200C110101EC001B1C000208
:106C20000101ED00052011130104EE001C20000CF1
:106C30000102F200002000030101F40000201719F6
:106C40000001F500002003170102F6000406020B04
:106C50000102F8000A0C020B0102FA000D0F0F17D7
:106C60000102FC0013150F170102FE001618020B9B
:106C7000010200011C1E020B0001020100100012A3
:106C8000010203010004000301030501000E1219B3
:106C9000010408010409000501040C01090E0007A4
:106CA000010310010E10000B01011301101100026D
:106CB000060009001016070A800314011016080EBA
:106CC0000101170115160608010318010E160E1909
:106CD00006000200171A000601021B011620061901
:106CE00001041D0100030619010121011117070903
:106CF000010122010320171901012301001B1719AB
:106D000001012401090F0E1080022501151702044C
:106D1000010127011A1B0E10010228011B200E1968
:106D200001022A0100200E1980022C010E10070911
:106D300080022E010E0F0C0E0102300100200E19F0
:106D4000800232010F1103050102340100200E19E7
:106D500080023601151703050102380100060E19DD
:106D600001013A0106070E1011013B010F150D0F2D
:106D700080023C01191B090B80033E0106201019FB
:106D80000600090006200F121101410100060D0F37
:106D90000600090000200F12800342010020101994
:106DA000800245010B0D090B1101470112180D0F4F
:106DB000800248011D1F090B0600090000200F1268
:106DC00080034A010020101911014D01040A0D0F22
:106DD00080024E011012090B11015001161C0D0FFB
:106DE0000600090000200F12800351010020101935
:106DF0008002540104060A0C1101560103070C0E0F
:106E0000110157010F130B0D110158011B1F0A0C23
:106E10000600090000170F1280035901001710190E
:106E200080025C01080A070911015E01070B090BCA
:106E300080025F010C0E0709900261010B0F090B24
:106E4000800263010F111416010165010F1116175D
:106E5000010166011617080A800267011B1D070859
:106E6000010269011720081901026B0100070819C6
:106E700001016D010708080A80026E01080A0B0D66
:106E8000800270010D120C0D0102720107170D191D
:106E90000101740117180D0F800275011416030506
:106EA0000101770113170507800278011C1E0F11DD
:106EB00001027A011720111901017C011E1F000235
:106EC00001037D011F20000701038001001100075D
:106ED00001028301000311190104850102110F1140
:106EE000010189010310111901028A0110201119F1
:106EF00001058C011120000906000A0000030011A1
:106F00000101910100010002010292010006111924
:106F1000010194010607111380029501050703057D
:106F200011019701040805070101980111120709D1
:106F3000000399011220081980039C0106121319FD
:106F400001019F0112200708060009000620121502
:106F50008402A001102013140101A20100200708DF
:106F600006000900002012158402A301002013145A
:106F70008002A501030502040003A70100200819EF
:106F80000101AA01001E07080600090000201215D1
:106F90008402AB01002013148002AD01030502043A
:106FA0000003AF01001E08190002B2011E201319D0
:106FB0000101B4011E1F0709060009000020121577
:106FC0008003B501002013191101B80105090E1045
:106FD000060004000A0D001906010A000E1100192E
:106FE0001101B90115190E10060009000020121533
:106FF0008003BA01002013191101BD0104080E100D
:107000001101BE010F130E101101BF011A1E0E1047
:1070100006000900000712158003C00100071319BC
:107020000101C301030710120101C40106070D0F7E
:107030000102C501071B0D198002C7010C110C0DBF
:107040000101C9011B1C0D0F060009001B201215B0
:107050008003CA011B201319060009000020121525
:107060008003CD01002013191101D001080E0B0D72
:107070001101D101171D0B0D0600090000051215A5
:107080008003D201000513190101D50104050B0D80
:107090000102D60105200B190101D80100010B0DD9
:1070A00006000900002012158003D90100201319E1
:1070B0001101DC01070B0B0D1101DD0115190B0D81
:1070C0000101DE011F200A0C0102DF0100200A1964
:1070D0000102E10100200A190102E30100200A195E
:1070E0000001E501090A02070001E6010F1002078D
:1070F0000001E701121302070001E801151602075B
:107100000001E9011C1E000A060008001C1F000AFD
:107110000102EA0100200A190001EC010B0C020730
:107120000001ED01101102070001EE011314020726
:107130000001EF011C1E000A060001001C1F000ACE
:107140000002F001002015190103F201040A0002F7
:107150000101F501050702080103F601050A080B04
:107160000101F9010A0C000B0101FA01070A0506E9
:107170000001FB010D0F090B0104FC0111190002B4
:107180000101000211130209010301021119090B87
:107190000103040217190709000107021317070961
:1071A000010208021719020400010A021A1C090B45
:1071B00001010B0213140B0C00010C02081614152C
:1071C00005010D020002111380030D02000A1319BC
:1071D000010310020A201319000113020305010321
:1071E00000011402141611130501150211131113D5
:1071F0000102150200200B0D0002170200200D19DC
:10720000000119020C120204000000000009020033
:10721000080200FF0000040900090200060102FF45
:107220000400081200060402000203FF0C00031809
:1072300000060202000105FF0F00021E0009020005
:10724000070206FF1100082700050101000108FFE1
:107250001900012C00090301000109FF1A00013582
:107260000006020004010A001B00023B00040202A7
:1072700003020B011D00033F0009010007020DFF7F
:1072800020000348000C01000A020F0223000254F0
:10729000000E03000B03110325000462000A020123
:1072A000080214FF2900036C0009020007001604FD
:1072B0002C00027500180100160316FF2E00008D29
:1072C00000090202080019052E00008D00090202C3
:1072D000080019052E000296000D03000B0119FF8E
:1072E000300004A30003010002001A06340004A6C3
:1072F0000005010004011A07380007AB0003010173
:1073000000011BFF3F0006AE0002010100011CFF4F
:10731000450007B00002010100011DFF4C0005B24D
:107320000006010004021EFF510003B8000603021C
:10733000050320FF540004BE00050202000223FFE3
:10734000580004C300060202050225FF5C0003C9C1
:10735000000B02000A0227FF5F0003D4000C0100AB
:10736000080129FF620000E00006030004002AFF74
:10737000620000E00006030004002AFF620000E053
:107380000006030004002AFF620003E6000C03006D
:1073900009032A08650000F20005030300032D0914
:1073A000650002F7000703020604300A670002FEC8
:1073B00000060202000134FF690002040105020216
:1073C000040135FF6900020401050202040135FFD2
:1073D0006900020401050202040135FF6B00050982
:1073E00001090300070236FF6B00050901090300CC
:1073F000070236FF6B00050901090300070236FF8B
:107400007000041201040202000138FF700004122F
:1074100001040202000138FF70000412010402029C
:10742000000138FF7400061601040200030139FF51
:107430007A00051A0106030205013A0B7F000520B8
:107440000101010100003BFF840005210101010150
:1074500000003BFF840005210101010100003BFF0A
:10746000840005210101010100003BFF89000E227B
:107470000107010106003BFF97000F2901060101EA
:1074800005003BFFA6000D2F0110000000053BFF8B
:10749000B300133F01060000000340FFC60006458D
:1074A00001030000000243FF000000000000000094
:1074B000000000FF11241FBECFEFD0E1DEBFCDBF23
:1074C00014BE88E10FB6F8948093600010926000BB
:1074D0000FBE11E0A0E0B1E0E6EAFBEE02C00590CD
:1074E0000D92A035B107D9F71EE0A0E6B1E001C0CA
:1074F0001D92AF3BB107E1F7F894EDEEF9E080E0C3
:1075000090E020E802C02193019632E08C3093078E
:10751000D4F38DEE99E09093FA0B8093F90B1092CF
:10752000FB0BEEEFFBE080E090E003C010820196E1
:107530003A9684309105D4F39093300C80932F0CBD
:1075400091E090931E0C90931F0C90931D0C109241
:10755000810015BC8FEF87B984B988E98AB95C9A34
:107560008CE081B98BEF82B91092BC0986E08093E0
:10757000BD09109285001092840083E080938900F9
:107580008DE88093880089E08093810082E0809379
:107590006F0082E484BD17BC95BD83E88093B00082
:1075A0001092B3009093B10081E185B91092D10996
:1075B0001092C0091092C1091092CC091092CB0907
:1075C0001092D0091092CF091092E0090E948145D3
:1075D00080E00E94C34380FF03C084E00E94C04358
:1075E0000E94334B78940E94324B0E94786D0C9429
:1075F000D1750C940000E0E0E0936F00AAECB0E0DD
:107600001197F1F70000E8E6F9E0C0E6D1E020913B
:10761000A00C0027A081B181AC0FBD1F1C9112836B
:10762000021708F4102F1C9333960395003190F342
:1076300000E2005116E01A95F1F70A95D9F7C0E675
:10764000D1E02091B909922F2695269526951127EC
:10765000C20FD11F6E010091BA09602F06950695E1
:10766000069510E2019FC00DD11D67701CE1101B33
:10767000F12E4091C6095091C7094ABD5BBD5E011C
:10768000762F8F2D992E3091B80930300FB601FE2C
:10769000662701FEC0EE01FED4E001FE83E001FE9C
:1076A000992400EE802E0E94A13B2FE02A95F1F74D
:1076B0000000000000C0000000C063958A94B9F08B
:1076C000683031F004E00A95F1F700C000C0EBCF5C
:1076D0006627A0968A9509F4E6013A9509F4672F82
:1076E00009F4E50109F48F2D09F4992EDCCFC89532
:1076F000C895C895C895C895C895C895000000005C
:1077000061D311240E94DB4A11E00091BF090127D7
:107710000093BF092091C009002309F0212720937D
:10772000C009E1E0E093BE09F8944091BD09405ED4
:107730004093BD09E2E0E0936F00E2E0E0933600A1
:107740000895CF93DF937F936F933F93DF92CF9210
:107750009F923C2F307EAAE9B9E02898D7D428819F
:107760002D93C395CF71C32B28812D93C395CF71D2
:10777000C32B28812D93C395CF71C32B28812D93C3
:10778000C395CF71C32B28812D93C395CF71C32B84
:1077900028812D93C395CF71C32B28812D93C39539
:1077A000CF71C32B28812D93C395CF71C32B288113
:1077B0002D93C395CF71C32B28812D93C395CF7182
:1077C000C32B28812D93C395CF71C32B28812D9373
:1077D000C395CF71C32B28812D93C395CF71C32B34
:1077E00028812D93C395CF71C32B28812D93C395E9
:1077F000CF71C32B2881289A2D93C395CF71C32BAA
:1078000028812D93C395CF71C32B28812D93C395C8
:10781000CF71C32B28812D93C395CF71C32B2881A2
:107820002D93C395CF71C32B28812D93C395CF7111
:10783000C32B28812D93C395CF71C32B28812D9302
:10784000C395CF71C32B28812D93C395CF71C32BC3
:1078500028812D93C395CF71C32B28812D93C39578
:10786000CF71C32B28812D93C395CF71C32B288152
:107870002D93C395CF71C32B28812D932CE02A958E
:10788000F1F7CAE9D9E078E0679F0AB51BB5005067
:107890001440000D111D180108E615E0000D111D22
:1078A000280130E41BE1692D6770E62EF89409F099
:1078B00078942C8D239F020C131CF00195906F017E
:1078C000299120310FB7239FA10100FDA201040ED1
:1078D000151ED001299120317FB670FA239FA10196
:1078E0000EF4A201040E151EF0013F010024A60FA4
:1078F000B01D73E0679F00FF22C000C065E87CE315
:10790000600D711D6F937F9308950D91C89508B90F
:107910000D91C89508B90D91C89508B90D91C895F4
:1079200008B90D91C89508B90D91C89508B90D9180
:10793000C89508B90D91C89508B91EF540C0FD015C
:1079400067EA7CE3600D711D6F937F930895059145
:1079500000C008B9059100C008B9059100C008B978
:10796000059100C008B9059100C008B9059100C093
:1079700008B9059100C008B9059100C008B9F30124
:10798000F6F0059108B92991059108B9239F059151
:1079900008B920316FB6059108B908F4A201059124
:1079A00008B960FA040E059108B9151E1A950591DB
:1079B00008B9059139F1F00108B91EF700C001912D
:1079C00008B929910191000008B9239F0191000095
:1079D00008B920316FB660FA019108B90EF0A10123
:1079E0000191040E08B9151E00C0019108B97190EB
:1079F0000191F00178B800C01A9521F0000008B993
:107A000006F6DDCF08B927F536F4F001019108B983
:107A1000EA94E1F71FC0F601000098B8EA94C9F0B3
:107A2000059108B9EA94A9F0059108B9EA9489F09A
:107A3000059108B9EA9469F0059108B9EA9449F00A
:107A4000059108B9EA9429F0059108B9EA9409F07A
:107A500000000000002708B99F90CF90DF903F9171
:107A60006F917F91DF91CF91089520E4E091C60955
:107A7000F091C7098051829FE00DF11DA8E6B5E0A5
:107A8000629FA00DB11D002405900D9205900D92EE
:107A900005900D9205900D9205900D9205900D9216
:107AA00005900D9205900D9205900D9205900D9206
:107AB00005900D9205900D9205900D9205900D92F6
:107AC00005900D9205900D9205900D9205900D92E6
:107AD00005900D9205900D9205900D9205900D92D6
:107AE00005900D9205900D9205900D9205900D92C6
:107AF00005900D9205900D9205900D9205900D92B6
:107B000005900D9205900D9205900D9205900D92A5
:107B100005900D9205900D9205900D9205900D9295
:107B200005900D9205900D9205900D9205900D9285
:107B300005900D9205900D9205900D9205900D9275
:107B400005900D9205900D9205900D9205900D9265
:107B500005900D9205900D9205900D9205900D9255
:107B600005900D9205900D9205900D9205900D9245
:107B700005900D9205900D9205900D9205900D9235
:107B800005900D9205900D92112408950F931F9367
:107B900095E0899FE0E4F5E0E00DF11D048182812C
:107BA0009381E0E48E9FD0019E9FB00DE0919809F3
:107BB000F0919909EA0FFB1FA8E6B5E090E4699FF0
:107BC000A00DB11D1124403051F4A20FB11D822F20
:107BD000122F00FF11C0379610E1121B0DC088E074
:107BE000821B00FD04C0182FE80FF11D05C018E02E
:107BF000120FE20FF11D3197503031F498E0939F4E
:107C0000A00DB11D932F06C098E0931B58E0599F1B
:107C1000E00DF11D11243EEFE89400FD689458E05A
:107C2000591B48E0481B3EF0259123132C931196D5
:107C30004A95D1F707C02491319723132C931196BD
:107C40004A95C9F7E10FF11DA80FB11D5A9549F7E3
:107C500011241F910F910895F03EFA3E083F303EE7
:107C600028980E949A40E7E1EA95F1F7289A0FD107
:107C7000E0E0F6E0F2D0E0FF32D0E0FF2FC02F933B
:107C80003F934F935F936F937F938F939F93AF93A4
:107C9000BF9378941124E091C209F091C309E115D2
:107CA000F10509F009950E94894C0E94CA450E947D
:107CB000D2440E94C73F1124E091C409F091C50944
:107CC000E115F10509F00995BF91AF919F918F9151
:107CD0007F916F915F914F913F912F910895EF9315
:107CE000E091BD09E63EE0F5E630D0F12F923F92FB
:107CF0004F925F926F927F928F929F92AF92BF92BC
:107D0000CF92DF92EF92FF920F931F932F933F93A7
:107D10004F935F936F937F938F939F93AF93BF9393
:107D2000CF93DF930E94FB3ADF91CF91BF91AF9148
:107D30009F918F917F916F915F914F913F912F9183
:107D40001F910F91FF90EF90DF90CF90BF90AF9079
:107D50009F908F907F906F905F904F903F902F906B
:107D6000EF910895FF93EF93EFB7EF93E0918400C5
:107D7000EE50E13000F0E23000F0E33000F0E430AB
:107D800000F0E53000F0E63000F0E73000F0E830D9
:107D900000F0E93000F005D0EF91EFBFEF91FF91D7
:107DA00018950F921F92E8E5FCE70090BC09000CC3
:107DB0001124E00DF11D05901490F00109951F901C
:107DC0000F90089528980E949A40E5E1EA95F1F70E
:107DD000E091BD09EA95E093BD09289A00C0089595
:107DE00028980E94C140289A0000E1E0F6E035D0D2
:107DF00047D0089528980E94C140E0EB0000EA9522
:107E0000E9F700000000289AF6E0E2E026D00895A5
:107E100028980E94C140289A0000E3E0FDEF1DD0A1
:107E2000E091BD09E53091F4E091BF09E130000037
:107E3000F091D10919F4F091D109F195E3E0E093C3
:107E40008900EDE8EF0FE09388000895E3E0E09308
:107E50008900EDE8E093880008950090BD090A9438
:107E600010905F0011FC0F2E0092BD090090BC091C
:107E700011FC0E2E0092BC09E0E011FCE1E0089537
:107E8000E3E0E0938900EDE8E09388000895E7E0FF
:107E9000E0938900EBE1E093880008950000000082
:107EA00000000000000000000000000000000000D2
:107EB00000000000000000000000000000000000C2
:107EC00000000000000000000000000000000000B2
:107ED00000000000000000000000000000000000A2
:107EE0000000000000000000000000000000000092
:107EF0000000000000000000000000000000000082
:107F000099277727833008F00895E0E0F6E8660FB8
:107F1000771FE60FF71FA591B491EEEFFBE02AE083
:107F2000289FE00DF11DA183B28311240895909143
:107F30001D0C9170880F892B80931D0C0895992733
:107F40007727EEEFFBE02AE0289FE00DF11D6E3F62
:107F500031F460911D0C6E7F60931D0C0BC06F3F60
:107F600031F460911D0C6E6F60931D0C03C072E8BC
:107F7000760F75831124089599277727EEEFFBE09C
:107F80002AE0289FE00DF11D6083112408950E94CE
:107F9000BF470090FB0B002019F4ADEEB9E002C022
:107FA000A3EFBAE021E002260092FB0B22E020932F
:107FB000FC0B2F923F924F925F926F927F928F9223
:107FC0009F92AF92BF92CF92DF92EF92FF920F9368
:107FD0001F93CF93DF9350911C0C60911E0C7091F6
:107FE0001F0C8091200C2090FF0B3090000C4090D3
:107FF000020C5090030C6090010C1091FE0B7090DD
:10800000090C80900A0C90900B0CA0900C0CB09076
:108010000D0C2091080CC090130CD090140CE09023
:10802000160CF090170C0091150C3091120C9FEF6C
:10803000620C431CF2014491410300240008C12D4D
:10804000D02D970CA81CF501449142030024000890
:10805000C10DD01D0C0DED1CF7014491430300240C
:108060000008C10DD01D8A956AF440911D0C842F23
:108070008695062E0694062600FA7695679576F97B
:1080800040FF66F940E860FD4FE745030024000823
:10809000C10DD01D0024C038D0050CF0CFE70A94E4
:1080A000C038D0050CF4C0E8C058CD939A9509F0BB
:1080B000BFCF4091FC0B4A954093FC0B97E009F031
:1080C000B7CF6092010C4092020C90920B0CA092E0
:1080D0000C0C0093150CE092160C60931E0C709320
:1080E0001F0C8093200CDF91CF911F910F91FF9077
:1080F000EF90DF90CF90BF90AF909F908F907F9048
:108100006F905F904F903F902F900895E091F90B02
:10811000F091FA0B019100000093B3000BE0E93FEE
:10812000F0070DEE19E008F0F801E093F90BF09379
:10813000FA0B08950C949C400C949E400F931F934F
:108140002F93E091F90BF091FA0B01910093B3009A
:108150000BE0E93FF00710F40000000010F0EDEE36
:10816000F9E0E093F90BF093FA0BC895C895C89520
:10817000C895C895C895000000002F911F910F91D8
:1081800008950000E091BD09E0FFD8CFE1E1EA9554
:10819000F1F700000000089500000000000000005A
:1081A00000000000000000000000000000000000CF
:1081B00000000000000000000000000000000000BF
:1081C00000000000000000000000000000000000AF
:1081D000000000000000000000000000000000009F
:1081E000000000000000000000000000000000008F
:1081F000000000000000000000000000000000007F
:10820000808182838485868788898A8B8C8D8E8FF6
:10821000909192939495969798999A9B9C9D9E9FE6
:10822000A0A1A2A3A4A5A6A7A8A9AAABACADAEAFD6
:10823000B0B1B2B3B4B5B6B7B8B9BABBBCBDBEBFC6
:10824000C0C1C2C3C4C5C6C7C8C9CACBCCCDCECFB6
:10825000D0D1D2D3D4D5D6D7D8D9DADBDCDDDEDFA6
:10826000E0E1E2E3E4E5E6E7E8E9EAEBECEDEEEF96
:10827000F0F1F2F3F4F5F6F7F8F9FAFBFCFDFEFF86
:10828000000102030405060708090A0B0C0D0E0F76
:10829000101112131415161718191A1B1C1D1E1F66
:1082A000202122232425262728292A2B2C2D2E2F56
:1082B000303132333435363738393A3B3C3D3E3F46
:1082C000404142434445464748494A4B4C4D4E4F36
:1082D000505152535455565758595A5B5C5D5E5F26
:1082E000606162636465666768696A6B6C6D6E6F16
:1082F000707172737475767778797A7B7C7D7E7F06
:1083000000020406080A0C0E10121416181A1C1E7D
:1083100020222426282A2C2E30323436383A3C3E6D
:1083200040424446484A4C4E50525456585A5C5E5D
:1083300060626466686A6C6E70727476787A7C7E4D
:108340007F7D7B79777573716F6D6B69676563612D
:108350005F5D5B59575553514F4D4B49474543411D
:108360003F3D3B39373533312F2D2B29272523210D
:108370001F1D1B19171513110F0D0B0907050301FD
:10838000FFFDFBF9F7F5F3F1EFEDEBE9E7E5E3E1ED
:10839000DFDDDBD9D7D5D3D1CFCDCBC9C7C5C3C1DD
:1083A000BFBDBBB9B7B5B3B1AFADABA9A7A5A3A1CD
:1083B0009F9D9B99979593918F8D8B8987858381BD
:1083C00080828486888A8C8E90929496989A9C9EBD
:1083D000A0A2A4A6A8AAACAEB0B2B4B6B8BABCBEAD
:1083E000C0C2C4C6C8CACCCED0D2D4D6D8DADCDE9D
:1083F000E0E2E4E6E8EAECEEF0F2F4F6F8FAFCFE8D
:108400007F7F7F7F7F7F7F7F7F7F7F7F7F7F7F7F7C
:108410007F7F7F7F7F7F7F7F7F7F7F7F7F7F7F7F6C
:108420007F7F7F7F7F7F7F7F7F7F7F7F7F7F7F7F5C
:108430007F7F7F7F7F7F7F7F7F7F7F7F7F7F7F7F4C
:108440007F7F7F7F7F7F7F7F7F7F7F7F7F7F7F7F3C
:108450007F7F7F7F7F7F7F7F7F7F7F7F7F7F7F7F2C
:108460007F7F7F7F7F7F7F7F7F7F7F7F7F7F7F7F1C
:108470007F7F7F7F7F7F7F7F7F7F7F7F7F7F7F7F0C
:1084800080808080808080808080808080808080EC
:1084900080808080808080808080808080808080DC
:1084A00080808080808080808080808080808080CC
:1084B00080808080808080808080808080808080BC
:1084C00080808080808080808080808080808080AC
:1084D000808080808080808080808080808080809C
:1084E000808080808080808080808080808080808C
:1084F000808080808080808080808080808080807C
:108500007F7F7F7F7F7F7F7F7F7F7F7F7F7F7F7F7B
:108510007F7F7F7F7F7F7F7F7F7F7F7F7F7F7F7F6B
:108520007F7F7F7F7F7F7F7F7F7F7F7F7F7F7F7F5B
:108530007F7F7F7F7F7F7F7F7F7F7F7F7F7F7F7F4B
:10854000808080808080808080808080808080802B
:10855000808080808080808080808080808080801B
:10856000808080808080808080808080808080800B
:1085700080808080808080808080808080808080FB
:1085800080808080808080808080808080808080EB
:1085900080808080808080808080808080808080DB
:1085A00080808080808080808080808080808080CB
:1085B00080808080808080808080808080808080BB
:1085C00080808080808080808080808080808080AB
:1085D000808080808080808080808080808080809B
:1085E000808080808080808080808080808080808B
:1085F000808080808080808080808080808080807B
:1086000022002400260028002B002D00300033001B
:10861000360039003D004000440048004C00510045
:1086200056005B00600066006C00730079008100FA
:10863000880090009900A200AC00B600C100CC00F8
:10864000D800E500F30001011001210132014401CD
:1086500057016C0181019801B001CA01E5010202D4
:108660002102410264028802AE02D70203033003F2
:1086700061039403CB03050442048304C70410057B
:108680005D05AF0505066106C206290796070908BC
:10869000830805098E09200ABA0A5D0B0A0CC10C71
:1086A000840D510E2B0F121007110A121D134014C6
:1086B0007415BA1614188319071BA31C571E2420FF
:1086C0000E22142439267F28E82A752D29300633F6
:1086D0000F364539AD3C49401B442848734CFE5089
:1086E000CF55EA5A51600C661D6C8B725A79928094
:1086F00037885090E598FDA19FABD3B5A3C000008B
:10870000FB01DC0102C005900D9241505040D8F7AA
:108710000895DC0101C06D9341505040E0F7089589
:10872000FB01DC0101900D920020E1F70895809398
:108730009809909399090895E0E8F3E0A0E6B1E084
:1087400060E16D933197E9F7112408959927772710
:1087500020E2629F080E191EA0E6B1E0A00DB11D37
:10876000405F4C93112408958093C6099093C709E4
:1087700008958091BE09089511241092BE090895AC
:108780008093D1090895882329F48091C909909193
:10879000CA0908958091CD099091CE090895882342
:1087A00029F48091CB099091CC0908958091CF094B
:1087B0009091D009089578E07A95F1F7000001973B
:1087C000D1F70895F999FECF92BD81BD60BDF894AF
:1087D000FA9AF99A78940895F999FECF92BD81BDDD
:1087E000F894F89A80B5789408951F9380E090E00B
:1087F0000E94EC43182F81E090E00E94EC4390E04F
:10880000382F20E0210F311D2A55354509F491E01C
:10881000892F1F910895BF92CF92DF92EF92FF921E
:108820000F931F93CF93DF936C01062FB72E0E94F7
:10883000F5438823F1F18FEFC8168FEFD80611F4B6
:1088400081E03AC0EE24FF24C7010E94EC43182FB8
:10885000C70101960E94EC43D82FC0E0CE01810FE2
:10886000911D8C159D0521F4E114F10459F423C0E8
:1088700080E290E0E80EF91E90E0E91694E0F90637
:1088800019F719C0802F9B2D9C01E90180E2C82EA9
:10889000D12CC20ED31E87010F5F1F4FC7010E944C
:1088A000EC438993CC15DD0511F480E005C0780117
:1088B000F2CF84E001C083E0DF91CF911F910F914F
:1088C000FF90EF90DF90CF90BF900895BF92CF922E
:1088D000DF92EF92FF920F931F93CF93DF936C0180
:1088E0000E94F543882311F484E04EC0F601808194
:1088F0009181FFEF8F3F9F0709F445C08A55954549
:1089000009F441C002E010E020E4E22EF12CC7019E
:108910000E94EC43B82EC70101960E94EC43D82F69
:10892000C0E09E012B0D311DF60180819181281739
:10893000390719F41123B1F00EC02F5F3F4F19F41E
:10894000112309F4102F0F5F80E290E0E80EF91E6A
:108950000034E9F623C0E12EFF2495E0EE0CFF1C65
:108960009A95E1F7C0E0D0E0F601EC0FFD1FCE01D3
:108970008E0D9F1D60810E94E2432196C032D10579
:1089800099F780E001C081E0DF91CF911F910F91B5
:10899000FF90EF90DF90CF90BF9008951123D9F60C
:1089A00082E0F2CF0F938091E009882309F4A7C0F9
:1089B0008091E109882309F043C08091E2090E9477
:1089C000C343282F86FF0FC08091E3099091E409EB
:1089D00002979093E4098093E30997FF04C01092F3
:1089E000E4091092E30927FF12C08091E3099091F6
:1089F000E40902969093E4098093E309883E910587
:108A000034F087EE90E09093E4098093E30924FF2B
:108A10000FC08091E5099091E60902979093E609CD
:108A20008093E50997FF04C01092E6091092E509CA
:108A300025FF59C08091E5099091E609029646C04C
:108A40008091E2090E94CF439C014091E30950913B
:108A5000E4098F77907027FF0EC0BA01681B790B6D
:108A60007093E4096093E30977FF14C01092E4095E
:108A70001092E3090FC0840F951F9093E40980932F
:108A8000E309883E910534F087EE90E09093E40985
:108A90008093E3094091E5095091E609832F9927D6
:108AA00037FF10C08F7790709A01281B390B3093D5
:108AB000E6092093E50937FF16C01092E6091092E7
:108AC000E50911C08F779070840F951F9093E60988
:108AD0008093E509883D910534F087ED90E090930F
:108AE000E6098093E50980912D0C6091E30940919E
:108AF000E50920912E0C0091330C0E94F54A0F914C
:108B00000895FF920F931F93CF93DF93129A809152
:108B1000E009882329F081E090E00E94DB4302C055
:108B2000C895C895129800E010E0C0E0D0E0FF249E
:108B300016950795D695C79513988091E0098823D7
:108B400029F085E090E00E94DB4302C0C895C895FB
:108B5000009B1068019BD068139A8091E0098823DC
:108B600029F085E090E00E94DB4302C0C895C895DB
:108B7000F39480E1F816E1F61093CA090093C9094D
:108B8000D093CE09C093CD09DF91CF911F910F9162
:108B9000FF900895FF920F931F93CF93DF930E944E
:108BA00081458091C9099091CA0997FD06C08091BD
:108BB000CD099091CE0997FF27C081E090E00E94F7
:108BC000DB4300E010E0C0E0D0E0FF24000F111F05
:108BD000CC0FDD1F1398C895C895C895C895009B04
:108BE0000160019BC160139A88E090E00E94DB4322
:108BF000F39480E1F81651F71093CC090093CB0958
:108C0000D093D009C093CF09DF91CF911F910F91DD
:108C1000FF90089590E026E130E0829FF001839F6D
:108C2000F00D929FF00D1124EA5CF34F62870895D6
:108C300060931D0C089590E026E130E0829FF001E2
:108C4000839FF00D929FF00D1124EA5CF34F138681
:108C50001182089590E026E130E0829FF001839F29
:108C6000F00D929FF00D1124EA5CF34F81E0838BAD
:108C7000089590E026E130E0829FF001839FF00D9F
:108C8000929FF00D1124EA5CF34F6187089590E004
:108C900026E130E0829FF001839FF00D929FF00D5E
:108CA0001124EA5CF34F6483089590E026E130E0FC
:108CB000829FF001839FF00D929FF00D1124EA5CDA
:108CC000F34F658308959093910C8093900C8FE6F9
:108CD0008093960C1092EC09E6E3FCE021E08FEF24
:108CE00098E120831086868387831486118295837A
:108CF00076963CE0EE38F307A1F708951092370C12
:108D000010924D0C1092630C1092790C0196909376
:108D10009A0C8093990C9093350C8093340C90931B
:108D20009D0C80939C0C1092980C1092970C1092B2
:108D30008F0C10928E0C1092920C81E08093EC09B3
:108D40001092950C1092940C08958091400C87FD20
:108D500003C08AEF8093400C8091560C87FD03C0BE
:108D60008AEF8093560C80916C0C87FD03C08AEFCC
:108D700080936C0C8091820C87FD03C08AEF8093F6
:108D8000820C1092EC090895DC01ED91FC91119791
:108D9000AF014F5F5F4F11965C934E93E4912E2F7E
:108DA00030E0E7FF13C02F7730703695322F22273F
:108DB00037952795FA014F5F5F4FE4918E2F8F779C
:108DC000280F311DE7FDF1CF4D935C93C901089544
:108DD0008093960C08950E949F3F0895EF92FF9212
:108DE0000F931F93CF93DF93182F062FF42EE22EAD
:108DF000C82FD0E086E190E0C89FF001C99FF00D38
:108E0000D89FF00D1124EA5CF34F8385882321F06D
:108E10008181882309F0ACC0EE2091F486E190E0D6
:108E2000C89FF001C99FF00DD89FF00D1124EA5C96
:108E3000F34F138A8285882309F09AC0108698C060
:108E4000133059F481E091E090931F0C80931E0C35
:108E500081E080931D0C0F2D08C0812F60E00E94DF
:108E60009F3F812F6F2D0E94803F0F3799F486E13D
:108E700090E0C89FF001C99FF00DD89FF00D11241C
:108E8000EA5CF34F8091930C878784E99CE0958B93
:108E9000848B30C089E0089FC0011124E091900CC0
:108EA000F091910CE80FF91F3396459154914115BB
:108EB000510571F486E190E0C89FF001C99FF00D63
:108EC000D89FF00D1124EA5CF34F158A148A12C062
:108ED000FA01249186E190E0C89FF001C99FF00D4E
:108EE000D89FF00D1124EA5CF34F27874F5F5F4F47
:108EF000558B448B86E190E0C89FD001C99FB00D8F
:108F0000D89FB00D1124AA5CB34F50961C92509775
:108F10001A961C921A971C960C931C9711961C92E9
:108F200011972FEF19962C9319971896EC92189782
:108F30008BE090E0C89FF001C99FF00DD89FF00D25
:108F40001124EE0FFF1FE85CF34FF08251961C9244
:108F5000519781E01B968C931B9753961C925397C5
:108F600052961C92529714961C92149716962C9314
:108F7000DF91CF911F910F91FF90EF900895CF92C5
:108F8000DF92FF920F931F93CF93DF93EFE3FCE009
:108F90008181282F332727FD30958081280F311DAF
:108FA0002F3F310519F014F02FEF30E0C90137FFE2
:108FB00002C080E090E0808376964CE0E739F407C9
:108FC00039F78091EC09882309F028C144C1E09168
:108FD000990CF0919A0C9F012F5F3F4F30939A0CA0
:108FE0002093990C44914F3F69F5A9014F5F5F4F62
:108FF00050939A0C4093990CF90184918F3219F493
:109000001092EC0919C1863009F0FBC0FA013196C3
:10901000CF01019690939A0C8093990CE491E335DB
:1090200029F490939D0C80939C0CEBC0E53409F0DF
:10903000E8C080919C0C90919D0C90939A0C809329
:10904000990CDFC047FF02C04093920C542F5F7011
:10905000842F90E0807F9070803B910531F1803CBF
:10906000910581F18039910509F043C0C90101964C
:10907000F9014491019690939A0C8093990C019771
:10908000FC012491852F90E08C9FF0018D9FF00DC5
:109090009C9FF00D1124EA5CF34F8081882309F432
:1090A000B0C0220F852F648553C0C9010196F90114
:1090B0004491019690939A0C8093990C0197FC012E
:1090C000249153C02F5F3F4F30939A0C2093990CFB
:1090D00021503040F9012491852F90E08C9FF001C0
:1090E0008D9FF00D9C9FF00D1124EA5CF34F2487B7
:1090F00088C08091920C582F5F7090E0807F9070B4
:10910000803B910541F1803C910509F46EC08039A6
:10911000910509F076C02F5F3F4F30939A0C209352
:10912000990C21503040F9012491852F90E08C9FBB
:10913000D0018D9FB00D9C9FB00D1124AA5CB34F40
:109140008C91882309F45DC0220F852F1C966C91A9
:109150000E94EE4656C02F5F3F4F30939A0C2093EB
:10916000990C21503040F9012491473071F4852F3A
:1091700090E08C9FF0018D9FF00D9C9FF00D1124CD
:10918000EA5CF34F220F27833CC04B3071F4852FEC
:1091900090E08C9FF0018D9FF00D9C9FF00D1124AD
:1091A000EA5CF34F220F26832CC04C3571F4852FD7
:1091B00090E08C9FF0018D9FF00D9C9FF00D11248D
:1091C000EA5CF34F220F24831CC04436D1F4852F70
:1091D00090E08C9FF0018D9FF00D9C9FF00D11246D
:1091E000EA5CF34F220F25830CC0852F90E08C9F03
:1091F000F0018D9FF00D9C9FF00D1124EA5CF34F60
:10920000448789E99CE00E94C4469093980C80931F
:10921000970C10928F0C10928E0C02C0C6E1D0E019
:1092200060918E0C70918F0C8091970C9091980C9E
:109230006817790709F4CBCE6F5F7F4F70938F0C5F
:1092400060938E0C8091940C9091950C0196909364
:10925000950C8093940C0EEF1BE0C7E3DCE0FF2439
:10926000BFEFCB2ED12C8A89882309F05EC08B8971
:109270009C89892B09F456C09F858E85981708F024
:109280004CC050C08B852B893C898F37E9F4D901BC
:109290008D91BC8BAB8B8F3F01F1F90161811196F0
:1092A000BC8BAB8BE82FF0E0EE0FFF1FE059FF4FB8
:1092B0000190F081E02D8F2D0995EB89FC8981913A
:1092C0008E87FC8BEB8B28C0A9014F5F5F4F5C8BB7
:1092D0004B8BF90184918F3F21F418821C8A1B8AE1
:1092E00021C04F5F5F4F5C8B4B8B41505040FA0168
:1092F000649190E0880F991F80599F4FFC01259140
:1093000034918F2DF9010995EB89FC893196FC8BFD
:10931000EB8B3197E491EE871F869F858E8598179A
:1093200009F4B0CF8F858F5F8F878A85882319F4E2
:1093300020E030E06BC088898F3F11F08F5F888B11
:109340009F81992309F45CC02885222309F458C021
:109350008E81882309F454C04091960C442309F46B
:109360004FC0899FC001112480509F4F892F99279A
:1093700030E0B901869F9001879F300D969F300D98
:10938000112420503F4F232F33278D8190E0FC0183
:109390002E9FC0012F9F900D3E9F900D1124805055
:1093A0009F4F892F9927242F30E0AC01429FC001A5
:1093B000439F900D529F900D112480509F4F292F55
:1093C00033278B818823F1F0EA81F0E0E050FE47FB
:1093D000E491E058E89FC001112480509F4F892FED
:1093E0009927B601681B790B629FC001639F900D9E
:1093F000729F900D112480509F4F292F332702C058
:1094000020E030E08A819C81890F8A83F8012083E3
:10941000F394065F1F4F6696F4E0FF1609F023CF22
:10942000DF91CF911F910F91FF90DF90CF90089522
:109430001F93CF93DF93582F89E0589FC0011124C9
:109440002091900C3091910C280F391FC90103967F
:10945000FC01A591B491F90184918150823010F4FE
:1094600013E01DC08091630C8823B1F080916F0CD4
:10947000851711F4442381F480914D0C882371F0F9
:109480008091590C851711F4442341F490915D0C9F
:109490008091730C891710F012E001C011E0212FA8
:1094A00030E0FD01449186E190E0289FE001299F92
:1094B000D00D389FD00D1124CA5CD34F4F87119621
:1094C000BD8BAC8B188A8BE090E0289FF001299F20
:1094D000F00D389FF00D1124EE0FFF1FE85CF34FE5
:1094E00080E5808368878FEF89871A861B8A198AAF
:1094F00021E02B871A8A5D8729831C828E83133093
:1095000049F481E091E090931F0C80931E0C20930E
:109510001D0C08C0812F60E50E94803F812F6A8961
:109520000E949F3FDF91CF911F910895FF920F936B
:109530001F93082FF62E0E94803F10E08BE090E0F2
:10954000089FF001099FF00D189FF00D1124EE0FF8
:10955000FF1FE85CF34FF0821F910F91FF90089579
:10956000962F482F50E02BE030E0429FF001439FC0
:10957000F00D529FF00D1124EE0FFF1FE85CF34F2A
:109580006081691B60830E94803F0895482F50E0EE
:109590002BE030E0429FF001439FF00D529FF00D11
:1095A0001124EE0FFF1FE85CF34F9081690F608379
:1095B0000E94803F08953091A00C20E010C0822FBF
:1095C00090E0FC01EE0FFF1FE80FF91FE859F64F7E
:1095D000A081B181A05ABE4F82818C932F5F231747
:1095E00070F30895809300010895DF92EF92FF9247
:1095F0000F931F93CF93DF93182FD62E622F70E017
:10960000A0E0B0E0E42EFF241BC090E0FC01EE0FD0
:10961000FF1FEE0FFF1FE80FF91FE05CFA4F5083AA
:10962000C13ED10514F0218301C041833F5F585FE3
:10963000832F810F361748F3160F7F5F485F189608
:10964000701740F4242F205E5D2D30E0ED01CE0D2B
:10965000DF1DEECFDF91CF911F910F91FF90EF9023
:10966000DF9008950895E0E4F5E080EE808335967C
:1096700095E0E836F907D1F7E0EEF4E080E1819378
:1096800095E0E034F907D9F708951F93CF93DF935E
:10969000FA01549131961491C52FD0E09F012F5FAC
:1096A0003F4F70E095E0660F771F9A95E1F7680FDE
:1096B000711D40E00CC08491805F8D939F5F319657
:1096C0009517C8F34F5F2C0F3D1F605E7F4F41170A
:1096D00030F4DB01A05ABE4FF90190E0F1CFDF91E9
:1096E000CF911F9108958091A10C8823F9F080916A
:1096F000A20C8823C1F480919E0C8093A20C9091BF
:10970000A30CE92FF0E0E050FF4F808187B98091F2
:109710009F0C890F8093A30C882311F08D3031F4B6
:109720001092A10C089581508093A20C08952F925D
:109730003F924F925F926F927F928F929F92AF92E1
:10974000BF92CF92DF92EF92FF920F931F93DF931E
:10975000CF9300D000D0CDB7DEB71092A00C80918F
:109760000001882309F4BEC070E4872E75E0972EAF
:109770007724F4012081203E09F495C08091B90935
:1097800030E0280F311D9091BA098181482F50E0B7
:10979000490F511DC90163E0969587956A95E1F7D8
:1097A0008983277019F0F2E0FA8302C081E08A838E
:1097B000CA0153E0969587955A95E1F7982F842F23
:1097C000877019F032E0632E02C066246394B82ECD
:1097D000AA242501420E511C192FCC24DD2456C089
:1097E000183310F0832D05C01C3110F4812F01C0F7
:1097F000822D003210F4902F02C0902F9052282F0B
:1098000030E085E0220F331F8A95E1F7290F311DE3
:10981000B0E6EB2EB1E0FB2EE20EF31EF701608105
:109820006031F0F04091A00C403100F5842F90E0C1
:10983000FC01EE0FFF1FE80FF91FE859F64F3183C7
:1098400020836283862F642F0E94353D6091A00C97
:10985000F70160836F5F6093A00C6150603130F45A
:10986000872D4B815C8192010E94C63D8B819C813A
:1098700001969C838B830F5F9A81891708F4B0CF80
:109880000894C11CD11C1F5FC61468F480E09C2D95
:109890009C013C832B830981F4EE2F2E210EE8ECF2
:1098A0003E2E310E9DCF7394E5E0F0E08E0E9F1EAC
:1098B000F8E07F1609F05DCF3091A00C20E010C0D9
:1098C000822F90E0FC01EE0FFF1FE80FF91FE8590F
:1098D000F64FA081B181A05ABE4F82818C932F5F39
:1098E000231770F30F900F900F900F90CF91DF918F
:1098F0001F910F91FF90EF90DF90CF90BF90AF90AE
:109900009F908F907F906F905F904F903F902F909F
:1099100008950E94734B0E94974B08956093260C04
:109920008093A40C0895FC013996F093B40DE09354
:10993000B30D3696F093B60DE093B50D3F97A7EBB8
:10994000BDE040E050E0CA0133E0880F991F3A952E
:10995000E1F7840F951F880F991F8253924F11963C
:109960009C938E939A01220F331FC90173E0880FD5
:10997000991F7A95E1F7820F931F9C012C52324F69
:1099800013963C932E9312978652924F15969C9362
:109990008E9314974F5F5F4F16964230510599F69C
:1099A00082818093A40C61506093B00D08958093E0
:1099B000A60C6093A50C4093A80C2093A70C0895C7
:1099C000EF92FF920F931F93CF93DF93B82FE42E64
:1099D000E901F02E00FD04C0162F00E041E004C0B4
:1099E000062F01501FEF4FEF70E019C08B2F90E052
:1099F000F901E50FF11DEC0FFD1FA491FC01EE0F25
:109A0000FF1FEE0FFF1FE80FF91FE05CFA4FA28364
:109A10001382F482540FBF5F511740F37F5F7E15AE
:109A200028F4769F90011124502FF6CFDF91CF912B
:109A30001F910F91FF90EF900895FC0132815381A7
:109A4000A0E6B1E014C0208141810EC0862F90E2D3
:109A5000A0E6B1E0399F9927020E191EA00DB11D95
:109A6000805F8C9311242F5F241780F33F5F35179D
:109A700050F308952F923F924F925F926F927F9290
:109A80008F929F92AF92BF92CF92DF92EF92FF920E
:109A90000F931F93DF93CF93CDB7DEB729970FB600
:109AA000F894DEBF0FBECDBFFC01862FE42EA901C6
:109AB00028012081A180A21A9281B380B91AFA01EB
:109AC00064914F5F5F4FFA01149141505040681705
:109AD00010F01E1530F4615086236F5F1150E122A3
:109AE0001F5F082FFF24622E7724892E992480E699
:109AF000282E81E0382E40C0061709F400E07E2DA4
:109B00001B821A829201200F311D39872887C301D9
:109B10008F0D911D9D838C832AC0711709F470E00D
:109B2000769FF0011124A885B985EA0FFB1FE40F89
:109B3000F51FB491B983EA81FB81E80DF91D2C81F1
:109B40003D81DB2ED1018D2D90E2A0E6B1E0E99FB1
:109B50009927020E191EA00DB11D805F8C93112450
:109B60007F5F2A813B812F5F3F4F3B832A833A816E
:109B70003B1598F2F3940F5FFA1408F4BDCF2996C1
:109B80000FB6F894DEBF0FBECDBFCF91DF911F910E
:109B90000F91FF90EF90DF90CF90BF90AF909F908C
:109BA0008F907F906F905F904F903F902F9008958F
:109BB0002F923F924F925F926F927F928F929F92DD
:109BC000AF92BF92CF92DF92EF92FF920F931F93CB
:109BD000DF93CF9300D000D00F92CDB7DEB7FC015A
:109BE000DB01BA01408151818D919C911197841BB9
:109BF000950B1C01442437FC4094542C2281338162
:109C000012968D919C911397821B930B5C01CC242F
:109C1000B7FCC094DC2CFB0180819181841B950BE7
:109C20007C010027F7FC0095102FE982FA820B8354
:109C30001C8382819381821B930B3C01882477FCD7
:109C40008094982CC401B301A20191010E94A675D1
:109C50007B018C0169817A818B819C81A6019501B0
:109C60000E94A6756E157F05800791071CF401E020
:109C70000D8347C0E616F706080719070CF43FC026
:109C800069817A818B819C81A20191010E94A675D4
:109C900097FD35C0C401B301A60195010E94A675C8
:109CA00097FD2DC01D82C601B5010E94A6755B01FE
:109CB0006C01C201B101A20191010E94A675A60E1C
:109CC000B71EC81ED91EC401B301A40193010E948E
:109CD000A6757B018C0169817A818B819C819B01B6
:109CE000AC010E94A675E60EF71E081F191FAE14E0
:109CF000BF04C006D1062CF411E01D8302C08FEF13
:109D00008D838D810F900F900F900F900F90CF91BA
:109D1000DF911F910F91FF90EF90DF90CF90BF9058
:109D2000AF909F908F907F906F905F904F903F90FB
:109D30002F900895AF92BF92CF92DF92EF92FF9251
:109D40001F93CF93DF93EC017B0124E0A22EB12C73
:109D5000A80EB91EB501A7010E94D84D182F94E096
:109D6000C92ED12CCE0CDF1CCE01B501A6010E945C
:109D7000D84D8102C0011124181619061CF480E088
:109D800090E016C0C701B601AE010E94D84D182F51
:109D9000C701B601A5010E94D84D20E08102C00193
:109DA0001124181619060CF421E081E02827822FCF
:109DB000DF91CF911F91FF90EF90DF90CF90BF90F8
:109DC000AF900895FC01DB01938112968C9112975C
:109DD000981790F091818C91981770F0908111965E
:109DE0008C911197891740F020E0928113968C9105
:109DF000891718F021E001C020E0822F0895FC01AE
:109E0000DA0121818081882309F412826083772717
:109E100067FD709577FF03C0709561957F4F962F12
:109E200096959695637060FD02C081E001C083E065
:109E30008383862F8150823018F4892F8F5F01C071
:109E4000892F8483633009F49F5F9583808187FF26
:109E500008C08FEF81838481819584839195958358
:109E600004C0882311F081E08183109731F0818153
:109E7000821719F08C9181958C9308952F923F92BF
:109E80004F925F926F927F928F929F92AF92BF920A
:109E9000CF92DF92EF92FF920F931F93DF93CF93B6
:109EA000CDB7DEB761970FB6F894DEBF0FBECDBF5A
:109EB0007C01788B6F871982DC011A968C911A9736
:109EC00019969C911997892321F01C96BC91BC830B
:109ED00003C0F701F385FC83D70150968C9150970E
:109EE0001F969C911F97892321F05296BC91BB83AA
:109EF00003C0F701F189FB83D701CC901596DC9064
:109F0000BC2DBD19EC81BE0FBE87D70111960C91F7
:109F1000119716961C91802E811ABB818B0EE091B1
:109F2000A70DF091A80D309769F081E0898380E05A
:109F300090E0BE016F5F7F4F09958981882309F406
:109F400065C119829D2C9C0CEC819E0E100FF12F87
:109F50002B81F20FFA83C70107969D878C87D70163
:109F60001396BB87AA87F7013D96F987E887C70153
:109F700004969F838E8357EC252E5DE0352E662454
:109F800077249A81492E55249F5F998BD1019C910A
:109F90008091A30D981709F02DC11D82C301880F70
:109FA000991F5C0133E0AA0CBB1C3A95E1F7A80E9F
:109FB000B91EEBE1F0E06E9E60016F9ED00C7E9EBC
:109FC000D00C112410C1FD810F2F10E0F801EE0F0D
:109FD000FF1FE00FF11FEE0FFF1FEA0DFB1DE953FE
:109FE000F24F80859781892311F0328501C0318538
:109FF000F80183E0EE0FFF1F8A95E1F7E00FF11FF4
:10A00000EC0DFD1DE953F24F84A5813009F06CC0C1
:10A01000332309F4E5C090A92A81291758F086A5B1
:10A02000981640F087A5AE858A1720F081A988157B
:10A0300008F005C1BC81BB23C9F1D2C06581F7011D
:10A040008781992787FD909597FF03C0909581950B
:10A050009F4F262F332727FD309537FF03C03095BC
:10A0600021953F4F8217930754F48C859D8503C03B
:10A070008C859D8565814A855B850E94FF4EFC81AC
:10A080009F1AF801B3E0EE0FFF1FBA95E1F7E00F5A
:10A09000F11FEC0DFD1DE953F24F86A5998198162D
:10A0A00010F4916001C0926099839AC029892917A0
:10A0B00008F496C0F801A3E0EE0FFF1FAA95E1F7A0
:10A0C000E00FF11FEC0DFD1DE953F24F86A5981628
:10A0D00008F486C087A59E85891708F481C081A9E8
:10A0E000881508F0BFC07CC086A5981608F478C013
:10A0F00087A5AE85A81708F073C020A9821658F16D
:10A1000081A9881540F1F7012681280F2F5F832F41
:10A11000992787FD909597FF03C0909581959F4F54
:10A12000280FD70111962C93BB81B31794F4F80133
:10A13000EE0FFF1FE00FF11FEE0FFF1FEA0DFB1DDB
:10A14000E953F24F8885998565814E815F810E9430
:10A15000FF4EE8E044C0F80153E0EE0FFF1F5A95B0
:10A16000E1F71316C4F4432F552747FD5095E00F30
:10A17000F11FEC0DFD1DE953F24F81A990E001970D
:10A18000841B950B481659065CF5822F90E00297C8
:10A19000841B950B0EC0E00FF11FEC0DFD1DE95364
:10A1A000F24F81A990E048165906D4F4822F90E02E
:10A1B000019748165906A4F02150D70116968C91A4
:10A1C0001697281B11962C93BB811B163CF488858F
:10A1D000998560E04E815F810E94FF4EE4E0E98353
:10A1E000FD81FF5FFD83D10112968C91BD81B8176F
:10A1F00008F4E9CE0894611C711C0894211C311CE0
:10A20000E2E06E16710409F0C1CE898161960FB645
:10A21000F894DEBF0FBECDBFCF91DF911F910F919C
:10A22000FF90EF90DF90CF90BF90AF909F908F9076
:10A230007F906F905F904F903F902F900895F8011E
:10A24000EE0FFF1FE00FF11FEE0FFF1FEA0DFB1DCA
:10A25000E953F24FD70118969C918681981709F41B
:10A26000EDCE06CFEF85F8898081830F8083B8CF4C
:10A270002F923F924F925F926F927F928F929F9216
:10A28000AF92BF92CF92DF92EF92FF920F931F9304
:10A29000CF93DF9339EC632E3DE0732ECC24DD2485
:10A2A0008824992426E0422E8AC0452D50E0FA01E8
:10A2B000EE0FFF1FE40FF51FEE0FFF1FEA0DFB1D52
:10A2C000E953F24F80859781892311F0628501C09F
:10A2D0006185662309F45FC09A0103E0220F331FF2
:10A2E0000A95E1F7240F351F220D331DF901E953BB
:10A2F000F24F84A5813059F415EFE12E1DE0F12EC7
:10A30000E20EF31E96A589010A50124F0AC0B7EF5C
:10A31000EB2EBDE0FB2EE20EF31E90A98901085042
:10A32000124FFA01A3E0EE0FFF1FAA95E1F7E40F29
:10A33000F51FE20DF31DE953F24F83A5981718F4AA
:10A3400082A5891700F1EA01CC0FDD1FC40FD51FCC
:10A35000CC0FDD1FCA0DDB1DC953D24F6D81619536
:10A360006D83549CC0011124880D991D8453924F14
:10A3700040E050E00E94FF4E88859F81892311F0C4
:10A380006A8501C06985F7018081860F8083F801A5
:10A390008081860F80835394F3018081581608F4DE
:10A3A00084CF0894C11CD11C0894611C711C82E1EB
:10A3B00090E0880E991E92E0C916D104B1F05524A0
:10A3C000C601880F991F5C0163E0AA0CBB1C6A954B
:10A3D000E1F7A80EB91EEBE1F0E0CE9E1001CF9E92
:10A3E000300CDE9E300C1124D7CFDF91CF911F911E
:10A3F0000F91FF90EF90DF90CF90BF90AF909F9024
:10A400008F907F906F905F904F903F902F90089526
:10A410002F923F924F925F926F927F928F929F9274
:10A42000AF92BF92CF92DF92EF92FF920F931F9362
:10A43000DF93CF93CDB7DEB767970FB6F894DEBF43
:10A440000FBECDBF8B8B0091B90906950695069579
:10A450002091A50C2B873091A60C3C878091A80CED
:10A460008A879091A70C9987A9ECBDE0BE87AD873C
:10A47000CC24DD24E02FF0E0FD8BEC8BBEC1DB01B2
:10A480001396BC91BA8BEB89BE1709F09CC1DB0116
:10A4900017963C911797832E8694869486948B8288
:10A4A00018968C9118978695869586958C83159627
:10A4B0002C911597922E969496949694998216962E
:10A4C0004C914695469546954A83E13011F4122FFA
:10A4D00001C0132F1770412E31F044244394FB0127
:10A4E000808187FD70C1FA89F13009F06DC0CC2000
:10A4F00089F5842F90E0840D911DAC89BD898A1760
:10A500009B070CF460C1F5018081813091F409153D
:10A5100028F00983842D840F8A83C3C0112309F096
:10A520004FC0DB0111968C91281709F4BAC051E095
:10A530007AC0112331F4FB018281281729F052E0FF
:10A5400004C04F5F4A83415050E0091508F468C0C9
:10A55000098366C0091508F436C1D5018C91813094
:10A56000D9F4112311F050E005C050E0FB018181C6
:10A57000281351E0842F90E0840D911D2C893D8992
:10A580002817390714F40A834BC0112309F448C073
:10A590004F5F4A83415044C0842F90E0840D911D49
:10A5A000AC89BD898A179B0714F00A837AC01123EE
:10A5B00039F4FB018281281709F473C052E033C0DB
:10A5C0004F5F4A8341506DC0CC2049F4401708F4D6
:10A5D000FAC0892D901608F4802F898308C00915C8
:10A5E00008F4F1C0842F041708F4802F8A83112304
:10A5F00099F4D5019C91191634F4FB018181381727
:10A6000011F051E01BC197FF49C0DB0112968C91FC
:10A61000381709F012C142C08C818F5F8C833EC015
:10A62000552309F43EC09E012B5F3F4FFE01369635
:10A6300089819A81AB81BC818D839E83AF83B887EA
:10A6400050FF07C0D9018C9180838C9181508C93ED
:10A6500006C08081D9018C9380818F5F8083FB014C
:10A6600050815F733F81F884FD81EE8113C0A0E6C5
:10A67000B1E0852F90E2A0E6B1E0399F9927020E64
:10A68000191EA00DB11D805F8C9311242F5F2E1712
:10A6900070F33F5F3F1510F42F2FF9CFBA89B13017
:10A6A00059F49A818980AC853E010894611C711C23
:10A6B000B2E0EB2EF12C0AC09C81AB85F3E06F2E4B
:10A6C000712C6C0E7D1EE4E0EE2EF12CEC0EFD1EC6
:10A6D000FB01808187FF06C0FA89F13011F0A9855E
:10A6E00001C0AA85592E58188394F7018082491910
:10A6F000F42FF40DFF8750E0252D30E0215030403D
:10A700003F8B2E8B195F212E2A0E195F312E3A0EA8
:10A710001E504A2E410E54C03A893130D1F48F85F3
:10A720005816B8F4112331F191E0591619F4CC20E0
:10A73000A1F41CC0552319F4CC2079F419C0852F3D
:10A7400090E0EE89FF898E179F0791F4CC2081F469
:10A750000DC0112379F0552311F4342D0CC0852F31
:10A7600090E02E893F898217930711F4332D03C09F
:10A77000322D01C03A2F4B818C809980BA8113C051
:10A78000E0E6F1E0832F90E2E0E6F1E0499F9927CF
:10A79000020E191EE00DF11D805F808311242F5FD2
:10A7A0002B1770F34F5F481510F4292DF9CFF301E3
:10A7B00080818F5F8083F70180818F5F80835F5FFF
:10A7C000551508F4A9CFF889FF5FF88B675F7F4FB5
:10A7D00026E030E0A20EB31E38898989381708F4C4
:10A7E0004ECE0894C11CD11CAD85BE851196BE8786
:10A7F000AD87B2E0CB16D10439F1ED85FE85F0814D
:10A80000F98B2BE130E0C29EB001C39E700DD29E49
:10A81000700D11246051724FC601880F991F5C01A1
:10A8200043E0AA0CBB1C4A95E1F7A80EB91E8DECBB
:10A830009DE0A80EB91E188ACFCF52E09E01295F75
:10A840003F4FFE013896F4CE67960FB6F894DEBF00
:10A850000FBECDBFCF91DF911F910F91FF90EF9071
:10A86000DF90CF90BF90AF909F908F907F906F9030
:10A870005F904F903F902F9008952F923F924F926C
:10A880005F926F927F928F929F92AF92BF92CF9280
:10A89000DF92EF92FF920F931F93DF93CF9300D03D
:10A8A00000D0CDB7DEB7D090B909D694D694D6945F
:10A8B000EE24FF246624772488249924B5C00C2D27
:10A8C00010E0D801AA0FBB1FBD01600F711F660FFA
:10A8D000771FFB01EA0DFB1DE755F34F868987FFC4
:10A8E0001EC0E091B10DF091B20D3097C1F0660D30
:10A8F000771DAB014550534F980183E0220F331F62
:10A900008A95E1F72A0F3B1F280D391D295C324F2C
:10A9100082E06154734F0995882309F470C0F801EF
:10A92000EE0FFF1F980153E0220F331F5A95E1F7F6
:10A930002E0F3F1F240D351D2755334F2D563F4FEA
:10A94000D9018C9123593040882309F058C0E00F79
:10A95000F11FEE0FFF1FEA0DFB1DE755F34F808D32
:10A96000918DA28DB38D89839A83AB83BC83EE20B6
:10A9700061F089818D1508F042C09A818D2D9D1559
:10A9800008F4892F8A8360E015C08A81D816B8F54B
:10A9900099819D1510F060E008C06D2D691BF901CB
:10A9A000E157FF4F8081815068238D2DD91608F41F
:10A9B000892F8983F80123E0EE0FFF1F2A95E1F725
:10A9C000000F111FE00FF11FE40DF51DE755F34FC8
:10A9D000EA56FF4F20813181E659F040DF01AE5643
:10A9E000BF4FE257FF4F00818C91089F80011124D7
:10A9F0000E5F1F4FCE01019640E00E943A4DC39476
:10AA0000F1018081C81608F45ACF0894E11CF11CAA
:10AA10008EE190E0680E791EA2E3B0E08A0E9B1EE4
:10AA2000B2E0EB16F104E1F0CC2489EA282E8CE0A8
:10AA3000382E2E0C3F1CC701880F991F570115E0B7
:10AA4000AA0CBB1C1A95E1F7A81AB90AE2E3F0E0D8
:10AA5000EE9E2001EF9E500CFE9E500C1124D0CF94
:10AA60000F900F900F900F90CF91DF911F910F914A
:10AA7000FF90EF90DF90CF90BF90AF909F908F901E
:10AA80007F906F905F904F903F902F90089520E0BF
:10AA900030E062E370E025C012968C9112978F5FD0
:10AAA00012968C93129713969C911397891781F4A1
:10AAB00012961C92129711968C9111978F5F119696
:10AAC0008C9311979C91891719F411961C921197E8
:10AAD0004F5F1A964E1700F32F5F3F4F223031051C
:10AAE00079F0F901E755F34FE081269FD001279FC8
:10AAF000B00D369FB00D1124A65CB24F40E0EACFF6
:10AB00000895FC01E0818E2F86958695869591F4B7
:10AB10008091A20D8695869586958F31E9F4909166
:10AB2000A30D8091B00D981710F080E013C0892F0D
:10AB30008F5F10C08F3181F48091A20D869586952C
:10AB4000869551F48091A30D882311F0815002C0A5
:10AB50008091B00D8093A30DE093A20D0895A3EB17
:10AB6000BDE0ED91FD9180818F5F80838DE0A33CFE
:10AB7000B807B9F708952F923F924F925F926F9264
:10AB80007F928F929F92AF92BF92CF92DF92EF927D
:10AB9000FF920F931F93DF93CF93CDB7DEB7289724
:10ABA0000FB6F894DEBF0FBECDBFD82E0091A90D11
:10ABB0001091AA0D613019F0E0E081E002C0E1E0FF
:10ABC00080E0E82EFF246E2F70E0D701A755B34F29
:10ABD000FB01E755F34F80818C93D701AA0FBB1F70
:10ABE000C701E3E0880F991FEA95E1F7A80FB91FA5
:10ABF000FB01EE0FFF1FCB0143E0880F991F4A9521
:10AC0000E1F7E80FF91FA555B34FE555F34F8AE07B
:10AC100001900D928150E1F7C701880F991FA7019C
:10AC200025E0440F551F2A95E1F7481B590BCB012E
:10AC3000880F991F9B01A5E0220F331FAA95E1F70A
:10AC4000281B390BFFEB8F2EFCE09F2E820E931EEC
:10AC5000DA01A154B34FF4018EE101900D928150BD
:10AC6000E1F7DA01A550B34FF901E550F34F8EE15A
:10AC700001900D928150E1F782E390E0689F90018E
:10AC8000699F300D789F300D1124295C324FE89E6A
:10AC9000F001E99EF00DF89EF00D1124E95CF24FF1
:10ACA000D90182E30D9001928150E1F78CE0D89EAA
:10ACB000C0011124FC013996E00FF11F4491FB0102
:10ACC000E755F34F442309F4F7C04083FC013A965B
:10ACD000E00FF11F54910396800F911FFC01A59185
:10ACE000B491BE83AD83CB01880F991F5B0105E052
:10ACF000AA0CBB1C0A95E1F7A81AB90AEFEBFCE015
:10AD0000AE0EBF1E3C832B8322E330E0629F6001C6
:10AD1000639FD00C729FD00C11248BE39DE0C80E72
:10AD2000D91E852F90E03C01660C771C8B01000F2B
:10AD3000111F000F111F060F171F000F111F0555C0
:10AD4000134F1C01240E311C220C331CD701A755B4
:10AD5000B34FB887AF83E29E2001E39E500CF29E72
:10AD6000500C1124EBE3FDE04E0E5F1EA0C060917D
:10AD7000C50D7091C60D660D771DCE01019642E09E
:10AD800050E00E94804389819A81D8018D939C93E1
:10AD90008981ED81FE81E80FF11DCF01E3E0880F8D
:10ADA000991FEA95E1F7E0919B0DF0919C0DE80F5A
:10ADB000F91F3296E590F4908A819701280F311D92
:10ADC000C901880F991F820F931F880F991F6091E7
:10ADD000280E7091290E680F791FC40146E050E0DB
:10ADE0000E948043D5018C9187FF18C08A8190E032
:10ADF00001968E0D9F1D9C01220F331F280F391FB6
:10AE0000220F331F6091280E7091290E620F731F5D
:10AE1000C401CC9646E050E00E948043F501818158
:10AE2000FAE08F9FC00111246091A50D7091A60DCD
:10AE3000680F791F8B819C814AE050E00E9480431B
:10AE4000D60113968C918823E1F0EF81F88550812B
:10AE5000F20140E014C08381882379F0D601149672
:10AE60002D913C911597848195812817390729F4F4
:10AE700080818C93818111968C934F5F3A96451710
:10AE800050F3E6E0F0E0AE0EBF1E2B813C81265F62
:10AE90003F4F3C832B838AE090E0C80ED91EA2E08E
:10AEA000B0E06A0E7B1E0E5F1F4F8E0E9F1E621457
:10AEB000730409F05CCF01C0108228960FB6F89495
:10AEC000DEBF0FBECDBFCF91DF911F910F91FF90DD
:10AED000EF90DF90CF90BF90AF909F908F907F903A
:10AEE0006F905F904F903F902F9008959F92AF92F8
:10AEF000BF92CF92DF92EF92FF920F931F93DF9357
:10AF0000CF9300D0CDB7DEB7982E4091A90D5091C8
:10AF1000AA0D613019F0E0E081E002C0E1E080E0DC
:10AF2000282F30E0EE2EFF24D901A953B24FF701AC
:10AF3000E953F24F80818C93828112968C93C701E2
:10AF4000880F991F6C0163E0CC0CDD1C6A95E1F75A
:10AF5000C80ED91EC901880F991FFC0113E0EE0F1E
:10AF6000FF1F1A95E1F7E80FF91FE453F24FD601DE
:10AF7000A453B24F82E10D9001928150E1F78BE131
:10AF800090E0E89E5001E99EB00CF89EB00C1124B0
:10AF9000289FF001299FF00D389FF00D1124E051FA
:10AFA000F24FD501A051B24F8BE10D90019281502B
:10AFB000E1F78CE0989EC00111240B96480F591FB1
:10AFC000FA01849187010953124F8F3F09F451C050
:10AFD00090E0880F991F6091AB0D7091AC0D680FD8
:10AFE000791FCE01019642E050E00E9480434A81E1
:10AFF000F80142839082898129E0829FC001112457
:10B000006091A00D7091A10D680F791F429FA00162
:10B010001124C5018051924F0E94804310E006E048
:10B020008BE190E0E89E5001E99EB00CF89EB00CD8
:10B0300011241BC0109FC00111248C0D9D1D212FB8
:10B0400030E0F901A3E0EE0FFF1FAA95E1F7E20F50
:10B05000F31FEA0DFB1DE953F24F8453924F65A590
:10B0600040E050E00E94FF4E1F5F8A81181710F3E6
:10B0700003C0F801128290820F900F90CF91DF9160
:10B080001F910F91FF90EF90DF90CF90BF90AF9006
:10B090009F9008952F923F924F925F926F927F926E
:10B0A0008F929F92AF92BF92CF92DF92EF92FF92D8
:10B0B0000F931F93DF93CF93CDB7DEB7CD55D0401D
:10B0C0000FB6F894DEBF0FBECDBF4C012F966FAF09
:10B0D0002F97DC011A968C911A9719969C911997C3
:10B0E000892321F01C96BC91BDAF03C0F401F38508
:10B0F000FDAFD40150968C9150971F969C911F974D
:10B10000892321F05296BC91BCAF03C0F401F189B0
:10B11000FCAFD4011C911396BC91B10FF401718165
:10B12000A481A70FE72EFF24FCAD2F2F332727FD87
:10B1300030952E0D3F1DF4016681462F50E0C90168
:10B14000840F951F883C91054CF06195671B6953EE
:10B150006CAFF4E02996FFAF29970EC0241B350B86
:10B1600037FD04C029961FAE299706C0671B6CAF38
:10B1700008E029960FAF2997812F90E0F4012581EF
:10B1800030E08C01021B130B2E961FAF0EAF2E97D3
:10B19000B901680F791F2C967FAF6EAF2C97C7014E
:10B1A000841B950B9FAB8EABFA01EE0DFF1DFDAB23
:10B1B000ECABFDAD8F2F992787FD90955801A80E18
:10B1C000B91E2B01480E591E0CAD802F992787FD03
:10B1D00090952E962EAD3FAD2E9737FD14C0B7FC3F
:10B1E00012C06F3F710509F074F43FEF431651042C
:10B1F00009F04CF44091A30D28964FAF289726965E
:10B200001FAE269707C028961FAE289752E02696B5
:10B210005FAF269719826EA97FA9680F791F79AF52
:10B2200068AFECA9FDA9E80FF91FFBAFEAAF2796BD
:10B230001FAE279721961FAE21971FAE1EAE0B2F74
:10B2400010E06A961FAF0EAF6A972A2F30E06C9617
:10B250003FAF2EAF6C976CC426963FAD2697323029
:10B2600009F044C0B7FC0AC04FEF4416510409F07E
:10B270002CF453E026965FAF26975AC4D4018C91E4
:10B280009091A30D8138B8F0E0E0FFEFAE0EBF1E45
:10B290004E0E5F1E8091B00D981730F028961FAEAD
:10B2A0002897F1E0FFAF1DC09F5F28969FAF2897BA
:10B2B00001E00FAF16C021E031E0A20EB31E420E36
:10B2C000531E992339F0915028969FAF28973FEF4E
:10B2D0003FAF07C04091B00D28964FAF28975FEF62
:10B2E0005FAF61E8A616B104E4F134C02696BFADA5
:10B2F0002697B33009F048C0E091A30D2896EFAF30
:10B300002897FFADF195FFAF0DAD202F332727FD17
:10B3100030952E96AEACBFAC2E97A20EB31E1CADD0
:10B32000812F992787FD90954EA95FA9480F591F36
:10B3300059AF48AF2C964EAC5FAC2C97420E531EC3
:10B340006CA97DA9680F791F7BAF6AAF71E8A7165A
:10B35000B1043CF02E968EAD9FAD2E9780389105AE
:10B3600064F090E8A916B10474F42E96AEADBFADAA
:10B370002E97A138B1053CF003C0B1E0BEAF04C0C8
:10B38000EFEFEEAF01C01EAE8CE02896FFAD289720
:10B39000F89FC00111246091A90D7091AA0D680F4A
:10B3A000791FCE0186964CE050E00E94804326969D
:10B3B0000FAD26970023D1F58091C70D28961FADBC
:10B3C0002897811781F48091C90D282E332421E01C
:10B3D00030E023963FAF2EAF239720E030E0219658
:10B3E0001FAE21976EC08091C80D28963FAD28975B
:10B3F000831759F041E050E023965FAF4EAF23979B
:10B4000020E030E0222433245CC08091CA0D282E35
:10B41000332461E070E023967FAF6EAF239720E086
:10B4200030E071E021967FAF21974BC08FAD1816A9
:10B430006CF429A53AA58CA51901280E311CA1E0B0
:10B44000B0E02396BFAFAEAF23973BC0BFADBB23E9
:10B45000C9F069A57AA58CA5482F50E09A01260F5E
:10B46000371F8DA5281B31098EA5882321F41901CA
:10B47000240E351E12C08BA51B01280E311C01E0C5
:10B4800010E01BC0D40118968C9129A53AA59BA564
:10B49000813051F41901290E311CE1E0F0E02396CE
:10B4A000FFAFEEAF23970DC01901089421083108B2
:10B4B0009101290F311D0FEF1FEF23961FAF0EAF24
:10B4C00023971EAD812F992787FD9095982F882768
:10B4D0002C964EAD5FAD2C97480F591F2E966EAD32
:10B4E0007FAD2E97680F791F7BAB6AAB25963FAF78
:10B4F0002EAF25972A961FAE2A9721967FAD2197CA
:10B50000272F30E08BE190E0289FD001299FB00DDC
:10B51000389FB00D11246196BFAFAEAF6197BCA943
:10B520006296BFAF6297EDA96396EFAF6397FEA9EE
:10B530006496FFAF64970FA965960FAF65976696FF
:10B540004FAF669767965FAF679768966FAF6897DC
:10B55000E0C219821FAD17FF10C08CA590E02596A0
:10B560002EAD3FAD25972817390739F48EA5482F02
:10B5700050E025965FAF4EAF259726965FAD269794
:10B58000552331F52A966FAD2A97862F90E0FC015E
:10B5900003E0EE0FFF1F0A95E1F7E80FF91F619630
:10B5A0008EAD9FAD6197E80FF91FE953F24F86A565
:10B5B000682E772487A5E82EFF2480A9C82EDD24D5
:10B5C00081A9082F10E06F5F2A966FAF2A9735C0C8
:10B5D00025968EAD9FAD259713E0880F991F1A957C
:10B5E000E1F760919B0D70919C0D680F791FCE0162
:10B5F0004E9648E050E00E9480438AA1682E77244E
:10B60000B3E0660C771CBA95E1F78BA1E82EFF2416
:10B61000A3E0EE0CFF1CAA95E1F78CA1C82EDD2457
:10B62000F3E0CC0CDD1CFA95E1F78DA1082F10E0BA
:10B63000E3E0000F111FEA95E1F7AAADBBADAC1531
:10B64000BD050CF458C2461457040CF454C2EA1455
:10B65000FB040CF450C2E8ADF9AD0E171F070CF453
:10B660004AC2BDC26E8D862F61FF4FC02F96FFADBF
:10B670002F97FF2309F43FC26A962EAD3FAD6A971C
:10B68000261537050CF437C22E153F050CF033C2D2
:10B690006C964EAD5FAD6C974C155D050CF42BC2EE
:10B6A000401751070CF027C298012C193D09C7011A
:10B6B000861997094F8D2817390764F43595279512
:10B6C000021B130B6C968EAD9FAD6C978017910784
:10B6D0007CF40BC095958795E81AF90A6A96AEAD89
:10B6E000BFAD6A97AE15BF051CF4442329F402C010
:10B6F000442311F041E001C04FEFE0919E0DF09125
:10B700009F0D88A199A10995F6C1817809F4F3C12B
:10B7100067FF43C08091B10D9091B20D892BE9F183
:10B7200028A139A1C901880F991F820F931F880F83
:10B73000991F6091280E7091290E680F791FCE0114
:10B74000029646E050E00E94804388A199A10196AC
:10B750009C01220F331F280F391F220F331F6091C6
:10B76000280E7091290E620F731FCE01089646E0D5
:10B7700050E00E948043E091B10DF091B20D84E061
:10B78000BE016E5F7F4FAE01485F5F4F9E01225E3C
:10B790003F4F0995882309F4AEC1BDADBB2309F421
:10B7A00096C0FCADFF2319F423E0298395C03DAD7D
:10B7B00013162CF068969FAD68978BA906C0669605
:10B7C0009FAD669767968FAD67979E878F874CADC5
:10B7D00014163CF064969FAD649765968FAD65979F
:10B7E00006C062969FAD629763968FAD6397988B04
:10B7F000898B5DAD852F992787FD90956E857F8517
:10B80000860F971F9B8B8A8B8CAD282F332727FDA4
:10B81000309588899989280F391F3D8B2C8B6615A7
:10B82000770534F06E157F051CF49CE0998354C0B5
:10B83000488959894C155D0534F0401751071CF4AF
:10B84000A3E0A98349C08A899B89861597054CF096
:10B850008E159F0534F42C153D051CF0201731077B
:10B86000DCF0661577051CF06E157F05ACF040170F
:10B8700051071CF44C155D057CF4BDAD1B1624F47A
:10B880004E145F0434F003C06A147B0414F08CE09F
:10B8900001C083E0898320C07F8A6E8AFB8EEA8E96
:10B8A000888999898C159D052CF4D98EC88EDD8EDA
:10B8B000CC8E04C0198F088F1D8F0C8FCE010E9671
:10B8C000BE016A5E7F4F0E949A4E882319F0ECE019
:10B8D000E98302C0F3E0F983E091A70DF091A80D90
:10B8E000309749F08E8D84FF06C0CE014E96BE0182
:10B8F0006F5F7F4F0995E091A70DF091A80D3097EC
:10B9000059F026962FAD2697222331F480E090E05F
:10B91000BE016F5F7F4F09958981E82FF0E0AF018D
:10B92000437050706E965FAF4EAF6E97452B31F1FE
:10B930005DAD151624F461E041E050E007C06DAD47
:10B94000662309F453C14FEF5FEF6FEF93016A1461
:10B950007B040CF49501C7014E145F040CF4C20182
:10B96000281B390B429FC001439F900D529F900DA1
:10B9700011247DAD780F761B7DAF2EC0CF018C706A
:10B980009070892B49F18CAD181624F461E041E0E8
:10B9900050E007C09CAD992309F42CC14FEF5FEF35
:10B9A0006FEF9601A8ADB9ADCA16DB060CF49D0188
:10B9B000C8010AAD1BAD081719070CF4C801281BF4
:10B9C000390B429FC001439F900D529F900D11244F
:10B9D0001CAD180F161B1CAF4DAD242F332727FDB0
:10B9E00030952E96AEACBFAC2E97A20EB31E5CADBA
:10B9F000852F992787FD90956EA97FA9680F791FDC
:10BA000079AF68AF2C964EAC5FAC2C97420E531EAC
:10BA1000ACA9BDA9A80FB91FBBAFAAAF2696BFADF1
:10BA20002697B23099F5D4018C919091A30D81386D
:10BA3000B8F000E01FEFA00EB11E400E511E809125
:10BA4000B00D981730F028961FAE289711E01FAF61
:10BA50001DC09F5F28969FAF289721E02FAF16C08B
:10BA600040E051E0A40EB51E440E551E992339F056
:10BA7000915028969FAF28975FEF5FAF07C0609106
:10BA8000B00D28966FAF28977FEF7FAF6E968EAD83
:10BA90009FAD6E97892BB9F02C96AEADBFAD2C97AC
:10BAA000A615B70544F42996BFAD2997B16029962C
:10BAB000BFAF299720C02996EFAD2997E26029965C
:10BAC000EFAF299718C0EC70F070EF2BA1F00CA924
:10BAD0001DA90C151D0544F429961FAD2997146066
:10BAE00029961FAF299707C029962FAD299728605F
:10BAF00029962FAF299725964EAD5FAD25972396B2
:10BB00006EAD7FAD2397460F571F25965FAF4EAFA3
:10BB1000259725968EAD9FAD25978215930509F043
:10BB200018CD26969FAD26979F5F26969FAF2697A6
:10BB30002796AFAD2797AF5F2796AFAF2797A33074
:10BB400009F08ACB2996BFAD29970B2F10E0C801C9
:10BB500083709070892B81F0EDAD6E2F772767FD94
:10BB60007095660F771F660F771FA4014D5F5F4FBB
:10BB7000C40107960E94FF4E0C701070012B91F0CB
:10BB8000FCAD6F2F772767FD7095660F771F660FE7
:10BB9000771FC4010D9604E010E0800E911EA401F1
:10BBA0000E94FF4E29968FAD2997C35ADF4F0FB6DB
:10BBB000F894DEBF0FBECDBFCF91DF911F910F91E3
:10BBC000FF90EF90DF90CF90BF90AF909F908F90BD
:10BBD0007F906F905F904F903F902F9008952696A2
:10BBE0002FAD2697222309F4D8CD3CCD40E050E07C
:10BBF00060E0ACCE40E050E060E0D3CEEF92FF9248
:10BC00000F931F93DF93CF93CDB7DEB763970FB634
:10BC1000F894DEBF0FBECDBF8C01DE011196FC0192
:10BC200083E101900D928150E1F766956E83242F98
:10BC300026952F83F8018085958118161CF4961B94
:10BC4000692F01C0691BF8018685468118161CF40E
:10BC5000421B242F01C0241BE62EEE0CEE0C05C067
:10BC60001E1414F4E39401C0EA948E2D992787FDE5
:10BC7000909597FF03C0909581959F4F837090702A
:10BC8000892B71F7F22EFF0CFF0C05C01F1414F462
:10BC9000F39401C0FA948F2D992787FD909597FF13
:10BCA00003C0909581959F4F83709070892B71F799
:10BCB000CE0108966E2DAE014C5F5F4F0E94FF4E85
:10BCC000CE010E966F2DAE014B5F5F4F0E94FF4E6F
:10BCD000CE01019660E00E944A58882311F080E06E
:10BCE0001BC09E2D95959595F8018081890F8083C5
:10BCF0002F2D259525958181820F81838381891B35
:10BD000083838481821B84838281890F82838E81D5
:10BD100085838F81868381E063960FB6F894DEBFBA
:10BD20000FBECDBFCF91DF911F910F91FF90EF908C
:10BD300008952F923F924F925F926F927F928F92CF
:10BD40009F92AF92BF92CF92DF92EF92FF920F93AA
:10BD50001F93DF93CF93CDB7DEB7E0970FB6F8947C
:10BD6000DEBF0FBECDBFD82E262E8091C30D2CE096
:10BD7000829FC00111246091A90D7091AA0D680FD6
:10BD8000791FCE0185964CE050E00E9480435D2CE7
:10BD9000539430E040E0E0E6F1E01FC0842F90E2F1
:10BDA000E0E6F1E0399F9927020E191EE00DF11D22
:10BDB000805F808311242F5F251580F33F5F393129
:10BDC00061F4AA2411E1612E712C6C0E7D1EB7E185
:10BDD0008B2E912C8C0E9D1E36C12D2DEDCF8E01FC
:10BDE000035E1F4F88A599A58A0D911DA3E0880FBA
:10BDF000991FAA95E1F760919B0D70919C0D680FBA
:10BE0000791FC80148E050E00E9480438D8D82FD7B
:10BE100019C189A1D81608F415C18AA1D81608F04D
:10BE200011C1CC24C801302E492E08C10C2D10E0C0
:10BE30008F8D98A1800F911F9C01220F331F280F17
:10BE4000391F220F331F6091280E7091290E620F47
:10BE5000731FC30146E050E00E9480438B89D816CF
:10BE600008F4E8C08C89D81608F0E4C0898987FFF7
:10BE70002AC08091B10D9091B20D892B21F18F8D47
:10BE800098A10196800F911F9C01220F331F280F4C
:10BE9000391F220F331F6091280E7091290E620FF7
:10BEA000731FC40146E050E00E948043E091B10D51
:10BEB000F091B20D81E0B301A401232D342D099539
:10BEC000882309F4B9C0898981FF7BC0BB246AC07B
:10BED000EB2CFF24D801AA0FBB1FAA0FBB1FA00F7A
:10BEE000B11FAE0DBF1DFD01EE0FFF1FE555F34F56
:10BEF00080818A1509F055C0AA0FBB1FA755B34F03
:10BF000013968C918C1509F04CC0A701440F551F56
:10BF1000FA01EE0DFF1DEE0FFF1F9801220F331FD8
:10BF2000C801B5E0880F991FBA95E1F7821B930B02
:10BF3000E80FF91FE755F34F828D938DDD825E8206
:10BF40008F839887808D6D2D681BF701A3E0EE0F1E
:10BF5000FF1FAA95E1F7E40FF51F22E330E0029FEF
:10BF6000C001039F900D129F900D1124E80FF91F3F
:10BF7000E755F34FEA56FF4F20813181E659F040F3
:10BF8000DF01AE56BF4FE257FF4F00818C91089FF3
:10BF9000800111240E5F1F4FCE01059640E00E94E4
:10BFA0003A4DB39400E010E031E0231611F401E0C3
:10BFB00010E0F801E755F34F8081B81608F488CFF8
:10BFC00039C09D894E895A8980FF1BC0D9865A86FF
:10BFD0009B874C87852F90E0880F991FE091AD0DCE
:10BFE000F091AE0DE80FF91F259134918B896D2DDD
:10BFF000681BCE01099640E002E010E00E943A4D35
:10C0000019C0392F13C0A0E6B1E0852F90E2A0E659
:10C01000B1E0399F9927020E191EA00DB11D805F56
:10C020008C9311242F5F251570F33F5F341710F4A4
:10C030002D2DF9CF898987FDC394C3948E8DC816A1
:10C0400008F4F4CEA3948AA5A81608F4C8CEFF2459
:10C050003E010894611C711CAD2CBB24EDE08E2EBA
:10C06000912C8C0E9D1E33C08DA19EA18F0D911D14
:10C07000880F991F880F991F6091260E7091270EC7
:10C08000680F791FC30144E050E00E94804339816A
:10C09000D316E0F0EB81FC812491832F90E0820F96
:10C0A000911DA816B90694F48A813196949131971E
:10C0B000DD865E868F87980F988B6D2D631BC4017C
:10C0C00040E09F0102E010E00E943A4DF3948FA1FE
:10C0D000F81650F220E030E09091C70D8091C30D2A
:10C0E000981711F021E030E0F901E953F24FE280B6
:10C0F000F090A80C7091A70C8BE190E0289FF001C4
:10C10000299FF00D389FF00D1124E051F24FC90125
:10C11000880F991F5C0153E0AA0CBB1C5A95E1F7EC
:10C12000A80EB91E2DEC3DE0A20EB31E60E000E6A5
:10C1300011E049C0808187FF40C085818695869542
:10C140008695D81608F439C0868186958695869599
:10C15000D81608F032C09781492F469546954695E6
:10C1600050855695569556958381813011F43F2D13
:10C1700020C0D5018C9187FF08C0892F90E087707F
:10C180009070892B11F04F5F5F5F372F12C0D8017D
:10C19000832F90E2A0E6B1E0499F9927020E191E75
:10C1A000A00DB11D805F8C9311242F5F251578F3AE
:10C1B0004F5F451710F42D2DF9CF6F5F399626E0AC
:10C1C00030E0A20EB31E6E1508F4B4CFE0960FB6A1
:10C1D000F894DEBF0FBECDBFCF91DF911F910F91BD
:10C1E000FF90EF90DF90CF90BF90AF909F908F9097
:10C1F0007F906F905F904F903F902F9008950F9396
:10C200001F93082F1091B90980912A0E181709F46D
:10C2100073C010932A0E2091AF0D80919D0D2817A9
:10C2200011F120939D0D213079F49091C30D8091EF
:10C23000B00D981710F080E002C0892F8F5F8093B7
:10C24000C30D1092A40D0FC02F3F69F48091C30D50
:10C25000882311F0815002C08091B00D8093C30DEE
:10C2600088EF8093A40D912F969596959695809141
:10C27000C40D981709F440C09093C40D9F31A1F4E8
:10C280002F3F91F48091C30D882311F0815002C09B
:10C290008091B00D8093C30D6FEF0E94BB558091CC
:10C2A000C30D6FEF0E9476578091A40D180F101BDD
:10C2B000812F8695869586956091AF0D0E94995E37
:10C2C0008091C40D8823C1F48091AF0D8130A1F419
:10C2D0009091C30D8091B00D981710F080E002C0CE
:10C2E000892F8F5F8093C30D61E00E94BB558091C1
:10C2F000C30D61E00E94765781E00E9408520E94BF
:10C300003D540E9447551F910F910895EF92FF925F
:10C310000F931F93DF93CF930F92CDB7DEB78C01AE
:10C32000198261E00E944A58E82E82E00E94085279
:10C330000E943851C801BE016F5F7F4F0E943E4F7F
:10C34000F82EF80182859185892311F0248502C099
:10C35000F8012385F80180899785892311F0728976
:10C3600002C0F8017189211129834981442399F17F
:10C37000F8018081840F8083141614F08FEF01C0C0
:10C3800081E08093AF0DF8015281242F332727FDE0
:10C3900030956091260C8091A40C141654F4250F4E
:10C3A000311D90E0860F911D2817390774F4450F51
:10C3B0000AC0250F311D90E0861B91098217930753
:10C3C00024F4450FF801428308C08091B909480F51
:10C3D0004093B90902C01092AF0D772321F0F80104
:10C3E0008181870F8183C8010E94815589810E94C4
:10C3F000FF608F2D8E290F90CF91DF911F910F91AC
:10C40000FF90EF900895EF92FF920F931F93CF93B9
:10C41000DF93182F469F70011124C0E0D0E009C0BF
:10C42000812F8C0F60EE40E021E001E00E94F54A90
:10C430002196CE15DF05A4F3DF91CF911F910F91C7
:10C44000FF90EF9008952F923F924F925F926F92DC
:10C450007F928F929F92AF92BF92CF92DF92EF9294
:10C46000FF920F931F93DF93CF93CDB7DEB7AC97B7
:10C470000FB6F894DEBF0FBECDBF5C01E62E8091F3
:10C48000A40CD5019C91F92EF81A12968C93129750
:10C490009093A20D18968C91189780939D0D1896E5
:10C4A0008C9118978093AF0D18968C91813011F074
:10C4B00088EF01C080E08093A40DE092A30DE0928C
:10C4C000C30DF50190818091A40C981748F4EE20DB
:10C4D00019F00E2D015002C00091B00D1FEF09C0E0
:10C4E0008091B00DE81610F000E002C00E2D0F5F35
:10C4F00011E08E2D612F0E94BB55802F612F0E946D
:10C50000BB558E2D612F0E947657802F612F0E9480
:10C510007657F0922A0EF092B909F694F694F694B2
:10C52000FDA2F092C40D0E949C431FA2FCE0EF9E6E
:10C53000C00111246091A90D7091AA0D680F791F97
:10C54000CE0149964CE050E00E948043D5019C9179
:10C550008091A40C9817D8F4BFA1BB23B1F5EE20AD
:10C5600011F0EA9402C0E090B00DF5018085909141
:10C57000A30D813011F4892F07C0992319F0892F59
:10C58000815002C08091B00D8093C30D03C0FFA104
:10C59000FF2319F04DA055241BC02091B00DE216C9
:10C5A00010F0EE2401C0E394D50118968C9190917F
:10C5B000A30D813039F4921710F080E004C0892F68
:10C5C0008F5F01C0892F8093C30D5DA0F0E24F2ED5
:10C5D000DD24B7C08C8D9D8D8D0D911DE3E0880FFE
:10C5E000991FEA95E1F760919B0D70919C0D680F82
:10C5F000791FCE01419648E050E00E94804389892E
:10C6000082FD9EC0FF2498C08E89851508F493C0D2
:10C610008D89481608F48FC08F898D3108F08BC042
:10C620008B899C898F0D911D9C01220F331F280F30
:10C63000391F220F331F6091280E7091290E620F4F
:10C64000731FCE01059646E050E00E9480438D8125
:10C6500087FF30C08091B10D9091B20D892B51F1BF
:10C66000F3948B899C898F0D911D9C01220F331FA0
:10C67000280F391F220F331F6091280E7091290E49
:10C68000620F731FCE010B9646E050E00E9480437C
:10C69000E091B10DF091B20D81E0BE016B5F7F4F73
:10C6A000AE01455F5F4F9E012F5E3F4F0995882386
:10C6B00009F441C08D8181FD3EC05F81652D551615
:10C6C00008F4652F6F839885442D941508F4492F3D
:10C6D00048877E8180FF15C0872F90E0880F991FC3
:10C6E000E091AD0DF091AE0DE80FF91F2591349159
:10C6F000651BCE01079640E002E010E00E943A4D33
:10C700001AC039855A8513C0E0E6F1E0872F90E220
:10C71000E0E6F1E0399F9927020E191EE00DF11DA8
:10C72000805F808311242F5F241770F33F5F3517DC
:10C7300010F4262FF9CFF3948A89F81608F464CF01
:10C74000D3948E8DD81608F445CFFF2478C0898DF8
:10C750009A8D8F0D911D880F991F880F991F6091D9
:10C76000260E7091270E680F791FCE01019644E0C6
:10C7700050E00E9480434B815C81FA0164914F5FDD
:10C780005F4FFA01F491FEA34150504099813A81E4
:10C79000262F290F251508F451C0491608F44EC05C
:10C7A0003D3108F04BC0852D591608F4892F282EED
:10C7B000291A822F421608F4842D382E391A70E077
:10C7C000662E7724892E9924C32EDD2422C0262F9D
:10C7D00030E0EBA5FCA5E20FF31F3296E40FF51F46
:10C7E000149118A7280D391DE9A5FAA5A0E6B1E016
:10C7F000812F90E2A0E6B1E0E99F9927020E191E71
:10C80000A00DB11D805F8C9311246F5F6315F8F24A
:10C810007F5F2EA1721790F4872F90E0869DD00144
:10C82000879DB00D969DB00D1124BCA7ABA7622DBE
:10C83000FC01EC0DFD1DFAA7E9A7E8CFF3948B8D61
:10C84000F81608F484CFFFA1FF5FFFA3F23009F0D0
:10C850006DCEAC960FB6F894DEBF0FBECDBFCF91B4
:10C86000DF911F910F91FF90EF90DF90CF90BF90DD
:10C87000AF909F908F907F906F905F904F903F9080
:10C880002F900895FB018091880E811110820895E8
:10C890003091640E380F181614F02FEF01C021E00C
:10C8A000622F772767FD709586EF9FEF689F502D69
:10C8B0001124932F3091650EE92F432F950F320FDE
:10C8C000892F851B8A30C0F719C0450F320F9A3067
:10C8D0004CF099E09093660E85E08093650E9093FE
:10C8E000640E0895920F892F821B87FF12C0109249
:10C8F000660E1092650E1092640E0895E093640E19
:10C900008AEF9FEF689F502D11243091660E922F71
:10C91000930F4630D0F63093660E4093650E08951F
:10C920008091390E861729F08091470E826080939E
:10C93000470E80915D0E8F5F80935D0E90915E0E2D
:10C94000891790F010925D0E80915C0E8F5F80933E
:10C950005C0E90915B0E891711F410925C0E809121
:10C96000470E82608093470E0895282F8091410ED4
:10C970009091400E892319F03091430E02C03091FE
:10C98000420E8091390E821729F08091470E826005
:10C990008093470E42FF0FC08091380E882349F4E0
:10C9A0008091500E813029F08091470E83608093F2
:10C9B000470E81E007C043FF07C08091500E8130D1
:10C9C00019F080E18093500E13169CF48091500E64
:10C9D000813079F48091460E80FD03C081608093A0
:10C9E000460E80E18093500E8091470E83608093C5
:10C9F000470E607C91F480913E0E9091380E892B09
:10CA000061F48091500E813041F48091460E80FF98
:10CA100004C08E7F8093460E0BC09091460E90FD11
:10CA20000CC08091380E882341F091609093460E9F
:10CA30008091470E83608093470E332301F58091E8
:10CA4000500E8130E1F480915D0E8F5F80935D0E1A
:10CA500090915E0E891718F110925D0E80915C0E18
:10CA60008F5F80935C0E90915B0E891711F410928A
:10CA70005C0E8091470E82608093470E08958091EE
:10CA80003E0E882361F08091500E803141F483E0A6
:10CA900080935C0E8091470E82608093470E0895CC
:10CAA0009091390E981729F08091470E82608093FB
:10CAB000470E8091450E8430A9F58091380E882369
:10CAC000D9F460737070672B81F080915D0E8F5F79
:10CAD00080935D0E90915E0E891730F110925D0E7D
:10CAE00080915C0E813079F414C080915C0E8823B3
:10CAF000D9F010925C0E10C08C5F893030F48091B8
:10CB00005C0E813089F081E005C080915C0E82303E
:10CB100059F082E080935C0E8091470E8260809392
:10CB2000470E089510925C0E0895EF92FF920F93B6
:10CB30001F93182F062F522F443608F043E6242F58
:10CB400022952F7086E0289FC00111244F70342F4A
:10CB5000380F832F6AE00E94C575F82EF20E832FDE
:10CB60000E94C575E92E57FD19C0252F332727FDD3
:10CB700030958091280190E0412F4F5F28173907A9
:10CB800031F0812F142F602F4DE550E005C0812F2B
:10CB9000142F602F44E050E00E94A643412F4F5FC6
:10CBA000FF2041F0812F142F4F2D50E04E5A5F4F40
:10CBB000602F04C0842F602F40E050E00E94A64305
:10CBC0004E2D50E04E5A5F4F812F602F0E94A6439A
:10CBD0001F910F91FF90EF9008958EE06DE14091CD
:10CBE000AB0E20E00E9495658EE06EE14091AC0EA8
:10CBF00021E00E94956583E16EE14091AD0E22E057
:10CC00000E94956588E16EE14091AE0E23E00E949E
:10CC100095654091BB0E5091BC0E8091B90E9091DC
:10CC2000BA0E480F591F8091BD0E9091BE0E480F4D
:10CC3000591F86E0569547958A95E1F78AE06EE19F
:10CC40002FEF0E949565089540911501552747FDE6
:10CC500050954E5A5F4F83E06DE10E94A64340918C
:10CC60001401552747FD50954E5A5F4F85E06DE101
:10CC70000E94A64340911301552747FD50954E5AF7
:10CC80005F4F86E06DE10E94A64308954091660ED5
:10CC9000552747FD50954E5A5F4F83E06EE10E9445
:10CCA000A6434091650E552747FD50954E5A5F4F5C
:10CCB00085E06EE10E94A6434091640E552747FD32
:10CCC00050954E5A5F4F86E06EE10E94A64308954C
:10CCD000AF92BF92CF92DF92EF92FF920F931F938A
:10CCE000CF93DF9349E8C42E4EE0D42EC3E1D1E0C8
:10CCF0008BE001E03BE0A32EBB24182F1F5FD60181
:10CD0000EC91FF27E7FDF095EC50FF4F4081602F3D
:10CD100050E00E94A643F12EF394D6011196EC91B7
:10CD2000FF27E7FDF095EC50FF4F4081812F602FEA
:10CD300050E00E94A643EF2CE394D6011296EC91AA
:10CD4000FF27E7FDF095EC50FF4F40818F2D602FBE
:10CD500050E00E94A6431D5F8E2D602F40E050E002
:10CD60000E94A643F12EF394EA81FF27E7FDF09598
:10CD7000E65DFE4F4081812F602F50E00E94A64368
:10CD80001E5F409134018F2D602F50E00E94A6431A
:10CD9000E981FF27E7FDF095E65DFE4F4081812F99
:10CDA000602F50E00E94A643E881FF27E7FDF09541
:10CDB000E65DFE4F4081812F8F5F602F50E00E9423
:10CDC000A643BB2029F485E004E025E0A22E0AC09A
:10CDD000B3E0BB1629F481E104E091E1A92E02C081
:10CDE0000E5F8A2DB39424E030E0C20ED31E23964A
:10CDF00037E0B31609F081CFDF91CF911F910F91EA
:10CE0000FF90EF90DF90CF90BF90AF9008951F9369
:10CE1000782F6091380E10913E0E662371F180914B
:10CE20004E0E8F5F80934E0E90914F0E891778F1C2
:10CE300010924E0E862F992787FD9095161684F432
:10CE400022273327281B390B80914D0E90E0442771
:10CE50005527481B590B241735076CF49A010BC052
:10CE600022273327281B390B80914D0E90E0821723
:10CE700093070CF49C01620F0AC086FF04C0609106
:10CE80004A0E619504C087FF02C060914A0E8091EE
:10CE9000450E843009F04AC017FD0EC08091560E31
:10CEA0008F5F8093560E9091570E891728F010923D
:10CEB000560E8091550E181B74FF1DC0212F33276D
:10CEC00027FD30958091510E90E0909581959F4F70
:10CED000821793070CF045C08091530E8F5F8093AB
:10CEE000530E9091540E8917E0F11092530E8091D9
:10CEF000520E181B36C075FF34C0212F332727FD73
:10CF000030958091510E90E02817390754F58091A3
:10CF1000530E8F5F8093530E9091540E891708F132
:10CF20001092530E8091520E180F1BC08830C9F416
:10CF3000E62FFF27E7FDF0954091490E242F30E0C2
:10CF40002E173F0714F4642F09C088279927821BE6
:10CF5000930BE817F90714F4642F61951C300CF457
:10CF60001E5F88E39EE044E35EE00E94FF4E8EE396
:10CF70009EE0612F45E35EE00E94FF4E1F91089501
:10CF80001F93FC016091380E10913E0E112309F0A1
:10CF900041C08091500E8130E9F58E2F807C11F4D4
:10CFA000662341F4E6FF02C0161624F0E7FF30C006
:10CFB00067FF2EC080914E0E8F5F80934E0E909132
:10CFC0004F0E891738F110924E0E862F992787FD44
:10CFD0009095161684F422273327281B390B80914D
:10CFE0004D0E90E044275527481B590B2417350751
:10CFF0006CF49A010BC022273327281B390B809130
:10D000004D0E90E0821793070CF49C01620F02C052
:10D0100010924E0EE6FF0FC0262F332727FD3095C6
:10D020008091490E90E0909581959F4F82179307CC
:10D0300014F42FEF0DC0E7FF2AC0262F332727FD5A
:10D0400030958091490E90E02817390704F521E0CA
:10D0500080914B0E8F5F80934B0E90914C0E8917F1
:10D06000B0F010924B0E112359F48091500E813084
:10D0700039F480914A0E289F802D1124680F09C031
:10D08000662329F480914A0E829F602D112411237A
:10D0900049F48091500E813029F4F0FF03C082E002
:10D0A0008093500E8091500E843019F1853038F401
:10D0B000813009F441C0823009F04AC006C088308E
:10D0C00051F1803109F044C037C01092530E1091D5
:10D0D000550E119581E080935C0E8091460E816023
:10D0E0008093460E8091470E83608093470E84E0C4
:10D0F0000FC0112369F582E080935C0E8091470E8A
:10D1000082608093470E8091110180934F0188E0E7
:10D110008093500E1DC080914F01815080934F012C
:10D120008823B1F483E080935C0E8091470E826087
:10D130008093470E80E1ECCF1092880E8091450ECF
:10D14000813019F480E18093550E8AE080931101BB
:10D150008091500E8830C1F0212F332727FD309564
:10D160008091510E90E02817390774F48091530E86
:10D170008F5F8093530E9091540E891728F0109270
:10D18000530E8091520E180F88E39EE044E35EE058
:10D190000E94FF4E8EE39EE0612F45E35EE00E9419
:10D1A000FF4E1F9108951F93782F6091380E1091B4
:10D1B0003E0E807C11F4662341F476FF02C0161601
:10D1C00024F077FF30C067FF2EC080914E0E8F5F36
:10D1D00080934E0E90914F0E891738F110924E0E9B
:10D1E000862F992787FD9095161684F422273327DA
:10D1F000281B390B80914D0E90E044275527481B82
:10D20000590B241735076CF49A010BC022273327DA
:10D21000281B390B80914D0E90E0821793070CF478
:10D220009C01620F02C010924E0E76FF1CC0262F8A
:10D23000332727FD30958091490E90E09095819598
:10D240009F4F821793074CF580914B0E8F5F809311
:10D250004B0E90914C0E891700F110924B0E80915D
:10D260004A0E681B1AC077FF18C0262F332727FDE8
:10D2700030958091490E90E02817390774F4809119
:10D280004B0E8F5F80934B0E90914C0E891728F0B8
:10D2900010924B0E80914A0E680F8091510E482FCC
:10D2A00050E0812F992787FD90958417950774F496
:10D2B0008091560E8F5F8093560E9091570E89176E
:10D2C00028F01092560E8091550E180F74FF1AC058
:10D2D000212F332727FD309588279927841B950B0D
:10D2E0008217930734F58091530E8F5F8093530E0E
:10D2F0009091540E8917E8F01092530E8091520EBF
:10D30000181B17C075FF15C0812F992787FD9095B1
:10D310008417950774F48091530E8F5F8093530E9A
:10D320009091540E891728F01092530E8091520E4E
:10D33000180F88E39EE044E35EE00E94FF4E8EE318
:10D340009EE0612F45E35EE00E94FF4E1F9108952D
:10D350008091450E823051F0833018F4813041F4D1
:10D3600009C0843089F0883019F410C082E00FC001
:10D3700080E00DC08091460E80FD04C08091380E83
:10D38000882329F081E003C083E001C084E06AE0E3
:10D39000869FB00111246F5D744B88E59EE04AE0E2
:10D3A00050E00E94804308950F931F93082F10911F
:10D3B000450E181711F480E0FEC08091440E609174
:10D3C000590E40915A0E0E9403620093450E0E942E
:10D3D000A869112389F06091590E660F660F660FD8
:10D3E00040915A0E440F440F440F81E39EE00E9487
:10D3F000FE5D882309F4BEC081E08093500E0430A6
:10D40000D1F10830C1F1023009F07DC060913E0ECB
:10D4100069300CF068E08EE39EE045E35EE00E9438
:10D42000FF4E83ED98E69093630E8093620E92E038
:10D4300090934A0E90934D0E10924B0E10924E0EFA
:10D4400028E020934C0E80E180934F0E8CE0809377
:10D45000490E9093520E81E08093550E1092530E18
:10D460001092560E86E08093540E8AE08093570EF9
:10D470002093510E72C0083051F482E08093490E1F
:10D480008CE08093510E00934D0E6CE00AC08CE04E
:10D490008093490E84E08093510E82E080934D0E7C
:10D4A00064E070E080913E0E992787FD9095861785
:10D4B00097070CF4BC018EE39EE045E35EE00E941A
:10D4C000FF4E87E097E69093630E8093620E88E0AC
:10D4D00080934A0E10924B0E10924E0E10924C0EEC
:10D4E0008CE080934F0E81E08093520E8093550E16
:10D4F0001092530E1092560E80E18093540E80E2EB
:10D500008093570E2AC080EC97E69093630E809329
:10D51000620E92E090934A0E90934D0E10924B0E35
:10D5200010924E0E88E080934C0E85E080934F0E53
:10D530002CE02093490E9093520E80E18093550E7B
:10D540001092530E1092560E9093540E9093570EC5
:10D550002093510E8AE0809311018091B20E909138
:10D56000B30E892B29F08091490E880F8093490EC4
:10D5700010E003C01093450E11E00E94A86980914D
:10D58000580E20915C0E829FC00111242091600EE4
:10D590003091610E280F391F00E08091390E8130E3
:10D5A00009F001E08091440E6091590E40915A0EAD
:10D5B0000E94E04C812F1F910F9108958091870E5A
:10D5C000882351F081508093870E882329F48DE2BF
:10D5D0009EE060E00E941D4D8091880E8823C1F07E
:10D5E00081508093880E882349F48091450E8130C4
:10D5F00019F480E18093550E8AE008C08091450EB1
:10D60000813031F480E28093550E80E180931101E6
:10D6100080912B0E90912C0E0097D1F00197909352
:10D620002C0E80932B0E892B49F48091450E81306E
:10D6300019F480E18093550E8AE008C08091450E70
:10D64000813031F480E28093550E80E180931101A6
:10D650008091B20E9091B30E0097E1F001979093F4
:10D66000B30E8093B20E892BA9F46091490E669592
:10D670006093490E8091380E992787FD9095262F4B
:10D6800030E02817390734F488E39EE044E35EE095
:10D690000E94FF4E8091BD0E9091BE0E009731F01A
:10D6A00001979093BE0E8093BD0E38C08091BB0E43
:10D6B0009091BC0E009731F001979093BC0E80932F
:10D6C000BB0E2CC08091B90E9091BA0E892BB9F087
:10D6D0008091450E813039F48091500E813019F4DB
:10D6E00088E00E94D4698091450E8830B9F4809119
:10D6F000B90E9091BA0E009789F001970BC08091F6
:10D70000450E883059F481E00E94D469882331F0B5
:10D7100080E190E09093BA0E8093B90E8091B00EA4
:10D720009091B10E009739F001979093B10E8093CC
:10D73000B00E892B39F48091450E823019F481E0C6
:10D740000E94D4698091B40E9091B50E009749F073
:10D7500001979093B50E8093B40E892B11F410921B
:10D76000B70E08951092B80E1092280C1092270C44
:10D770001092870E1092AF0E1092B70E1092A60E56
:10D7800086E0E9EBFEE0DF011D928A95E9F7109251
:10D79000AB0E1092AC0E1092AD0E1092AE0E8091A8
:10D7A000880E882319F081E08093880E80912B0EDB
:10D7B00090912C0E892B31F081E090E090932C0E0B
:10D7C00080932B0E8091B00E9091B10E892B31F089
:10D7D00081E090E09093B10E8093B00E8091B20EF4
:10D7E0009091B30E892B31F081E090E09093B30ECD
:10D7F0008093B20E8091B40E9091B50E892B31F0CA
:10D8000081E090E09093B50E8093B40E0E94DE6AA2
:10D8100087E69EE06FEF70E040E250E00E948943AF
:10D820000895CF93DF93EC018430910539F1853071
:10D83000910540F48130910589F08230910509F01D
:10D8400062C01CC08930910549F18A30910509F404
:10D850004BC08830910509F056C010C08091B80EB9
:10D86000882361F40E94B26B1092640E1092650ED0
:10D870001092660E1092B60E0E9446664091B80E47
:10D880009E0121503040842F90E082239323821701
:10D890009307C9F54C2B4093B80E35C01416A4F469
:10D8A0008091450E843079F581E00E94D46982E050
:10D8B0008093500E8091270C9091280C90FF23C0EC
:10D8C00080E48093880E1FC08091450E8430D9F08B
:10D8D0008091500E8E70B9F48091B70E882399F420
:10D8E00084E00E94D4690FC014161CF41092A60E96
:10D8F00007C08091A60E882331F481E08093A60EA4
:10D900008FE080931201DF91CF91089581E06EE165
:10D9100043E050E00E94A64381E06DE147E150E022
:10D920000E94A64384E06EE14CE550E00E94A643CD
:10D9300084E06DE14CE550E00E94A6434091150162
:10D94000552747FD50954E5A5F4F83E06DE10E9489
:10D95000A64340911401552747FD50954E5A5F4FFD
:10D9600085E06DE10E94A64340911301552747FDD4
:10D9700050954E5A5F4F86E06DE10E94A64388E0C5
:10D980006DE14BE75CE30E94454B8DE06DE14CE1BE
:10D9900050E00E94A6438CE06EE143E75CE30E9406
:10D9A000454B81E16DE14DE85CE30E94454B86E12A
:10D9B0006DE14CE15EE30E94454B0895DF93CF9308
:10D9C000CDB7DEB7A0970FB6F894DEBF0FBECDBFC0
:10D9D0008EE090E09A838983BE016F5F7F4F0E9443
:10D9E0000B44282F332727FD30952115310511F5DC
:10D9F000A3E1B1E0FE01339685E101900D928150E3
:10DA0000E1F78FE090E09A838983BE016F5F7F4FDB
:10DA10000E940B44282F332727FD3095211531050F
:10DA200049F4A9E8BEE0FE0133968CE101900D9225
:10DA30008150E1F7C901A0960FB6F894DEBF0FBE82
:10DA4000CDBFCF91DF910895DF93CF93CDB7DEB7F0
:10DA5000A0970FB6F894DEBF0FBECDBF8EE090E06A
:10DA60009A838983DE011396E3E1F1E085E1019079
:10DA70000D928150E1F7CE0101960E9466448FE03D
:10DA800090E09A838983DE011396E9E8FEE08CE159
:10DA900001900D928150E1F7CE0101960E946644FB
:10DAA000A0960FB6F894DEBF0FBECDBFCF91DF9129
:10DAB0000895CF93DF9380E090E06AE50E94E2430F
:10DAC00081E090E065E50E94E243C0E4D0E0CE0151
:10DAD0006FEF0E94E243CE0101966FEF0E94E24396
:10DAE000A09688E0C030D80791F7DF91CF910895D4
:10DAF0002F923F924F925F926F927F928F929F925E
:10DB0000AF92BF92CF92DF92EF92FF920F931F934B
:10DB1000DF93CF93CDB7DEB72C970FB6F894DEBF67
:10DB20000FBECDBF0E94F543882311F40E94596DAA
:10DB300009E81EE0C8016DE071E00E9490430C5FAF
:10DB40001F4F2EE0053A1207A9F70E94DE6C892BC1
:10DB500011F00E94246D87EA9EE069E87EE00E9451
:10DB6000904383E29EE40E94634680EB0E94E84675
:10DB700086E890E00E94B44384EA9EE30E949743C3
:10DB800081E00E94F24A83E08093B80981E19CE63B
:10DB900090939F0D80939E0D86E693E79093B20D30
:10DBA0008093B10D82E494E69093A80D8093A70D25
:10DBB0008FE69AE59093A10D8093A00D87E59AE5F5
:10DBC0009093AC0D8093AB0D85E699E59093AE0DE7
:10DBD0008093AD0D83E59BE49093A60D8093A50DF6
:10DBE0008DEC99E59093C60D8093C50D85E396E580
:10DBF0009093270E8093260E8CE29BE59093290E3E
:10DC00008093280E88EC97E690939C0D80939B0D53
:10DC100088E092E79093AA0D8093A90D1092440E8C
:10DC20001092460E82E00E94D46987E69EE06FEF74
:10DC300070E040E250E00E9489438091590E880FC5
:10DC4000880F8093360E80915A0E880F880F80932C
:10DC5000370E84E08093340E1092350E81E080936D
:10DC6000390E80933F0E88ED62EC48ED21EC0E9466
:10DC7000D74C81E39EE065E30E94934C81E39EE0F4
:10DC800065E30E9423621C861B86882411E0A12E76
:10DC9000B12CFF241A862224332401C012010E94D1
:10DCA000B9438823E1F30E94BC4380E00E94C34350
:10DCB0002C0180912901827219F48CE048225524AC
:10DCC00031016094709464207520FF2061F08F2DE5
:10DCD00090E083709070892B29F48EE06FEF41E023
:10DCE0000E94184AFA948091A60E882379F08091B8
:10DCF0001201815080931201882341F48FE08093B8
:10DD000012018BE060E441E00E94184A8091B80E55
:10DD10008F3009F08BC08091BB0E9091BC0E20918A
:10DD2000B90E3091BA0E820F931F2091BD0E309123
:10DD3000BE0E820F931FB6E096958795BA95E1F7D0
:10DD40002091AE0E821B0E9448640E94466620917C
:10DD5000660E9091650E3091640EE3E1F1E000E013
:10DD600010E00987828128176CF0281709F055C048
:10DD7000818198173CF0981709F04FC080813817BF
:10DD80000CF04BC0A2E2CA2EA1E0DA2EF1EAEF2E8F
:10DD9000FEE0FF2EE6E09E2E19C0892D90E0FC01EA
:10DDA000EE0FFF1FE80FF91FED5EFE4FD60183E077
:10DDB0000D9001928150E1F7C7010496B7010E94CE
:10DDC00090439A948DEF9FEFC80ED91E8CEF9FEF72
:10DDD000E80EF91E9985991500F3F801EE0FFF1F63
:10DDE000E00FF11FED5EFE4FA4E6BEE083E00D9074
:10DDF00001928150E1F7000F111F000F111FC801A0
:10DE00008757914F67EA7EE00E9490430E94246604
:10DE10000E94246D48E2F42E07C00F5F1F4F339617
:10DE20000730110509F09DCF0E94B26B10912901B6
:10DE3000113051F58091A50E8F5F8093A50E089447
:10DE4000A108B108A114B10409F02AC284E061E07C
:10DE500041E00E94036281E39EE067E30E94236247
:10DE600080E48093310E28E02093320E8093330EAD
:10DE70008FE0809312011093A60E80E18093290118
:10DE8000A12C33E0B32E0CC2103209F069C0E0912E
:10DE9000A70EFF27E7FDF095EC50FF4F40818DE086
:10DEA00065E050E00E94A643E091A80EFF27E7FD41
:10DEB000F095EC50FF4F40818EE065E050E00E940D
:10DEC000A643E091A90EFF27E7FDF095EC50FF4F28
:10DED00040818FE065E050E00E94A64364FE08C0E8
:10DEE0008C85E82FF0E0E955F14F80818F5F09C004
:10DEF00065FE08C09C85E92FF0E0E955F14F80816F
:10DF0000815080832C85E22FF0E0E955F14F80812C
:10DF1000813414F48AE503C08B3514F081E48083E6
:10DF200066FE0AC08C85882319F492E09C8706C09F
:10DF30008C8581508C8709C067FC03C02DE02B873E
:10DF40000CC08C85823020F01C869DE09B8705C02C
:10DF50002C852F5F2C878DE08B8725E0822EA0C13A
:10DF6000183009F067C18B85682D40E050E00E94B1
:10DF7000A643AA2049F494E0890E24E1281520F450
:10DF800083E18B8792E0892E0894A108B108A1143F
:10DF9000B104A1F582E00E94D46988EA8093310E31
:10DFA00090E29093320E8CE968E70E948E4C84E0F8
:10DFB00061E041E020E23BE400E00E94E04C84E0CC
:10DFC0006CE240E221E001E00E94F54A198220E281
:10DFD0002A838CE18B838FE18C83CE01019660E0F4
:10DFE0000E941D4D81E39EE065E30E94236281E073
:10DFF00080932901A12C82E0B82E52C1A5FE06C053
:10E000008B85682D44E050E00E94A64380E0A8166E
:10E0100085E0B80639F480E890E090932C0E809368
:10E020002B0E19C08091270C9091280C20ECA21681
:10E0300024E0B20631F491609093280C8093270C71
:10E040000AC09E7F9093280C8093270C80E8A81626
:10E0500089E0B80629F090E4A91699E0B90629F4F8
:10E0600081E090E0682A792A04C08EEF9FEF682251
:10E07000792290E0A91692E0B90628F48091B60EB4
:10E08000865F8093B60E20E0A21626E0B20609F461
:10E0900088C081E0A81686E0B80658F590E0A91679
:10E0A00094E0B90609F49BC021E0A21624E0B20670
:10E0B00068F480E0A81682E0B80609F4B7C090E0E2
:10E0C000A91693E0B90609F0EBC0A8C020E8A21693
:10E0D00025E0B20609F473C080ECA81685E0B80606
:10E0E00009F467C090E4A91695E0B90609F0D8C014
:10E0F0006CC020E0A21628E0B206A9F181E0A816C3
:10E1000088E0B80668F490E4A91696E0B90609F428
:10E1100042C020E0A21627E0B20609F0C1C029C023
:10E1200080ECA81689E0B80661F090EEA91699E097
:10E13000B90639F020E0A21629E0B20609F0B0C015
:10E140000EC083E0809328018EE06FEF41E00E94D3
:10E15000184A8091AE0E8B5F8093AE0EA1C085E011
:10E160008093AF0E9DC081E08093280181E890E00C
:10E170001DC01092280181E090E0682A792A82E08F
:10E180000E94D4698091270C9091280C20E930E0FE
:10E19000822793271FC08091270C9091280C8F7E97
:10E1A00019C082E08093280181E490E0682A792AEE
:10E1B00077C08091270C9091280C8F7B0BC08091A9
:10E1C000270C9091280C806805C08091270C9091B5
:10E1D000280C8F779093280C8093270C61C08CE0DB
:10E1E0006FEF41E00E94184A84E180932D0E87E191
:10E1F00080932E0E94E090932F0E87E08093300E44
:10E200008DE29EE060E040E027E23DE302E010E0C6
:10E210000E943A4D80E18093870E42C080E091E0F9
:10E220009093BA0E8093B90E88E001C081E00E94FD
:10E23000D46936C01031A1F50894A108B108A11421
:10E24000B10439F58EE78093310E84E68093320E67
:10E2500080E768E70E948E4C81E39EE066E30E94BF
:10E2600023620E94B26B1092640E1092650E10929F
:10E27000660E1092B60E0E94866C28E0209329014B
:10E2800082E08B8702E0802E1FEFA12E19E0B12ED5
:10E2900007C09FEFA91692E0B90611F40E946866C4
:10E2A00063FE6EC090912901892F897109F44CC0D9
:10E2B00084E062E042E00E94036281E00E94D4694F
:10E2C00028E72093310E88E28093320E8091360E3B
:10E2D000281B822F2093330E60E00E948E4C81E336
:10E2E0009EE064E30E942362B8E02B2E312C2420B0
:10E2F000352088E39EE060E044E35EE00E94FF4E4C
:10E300008EE39EE060E045E35EE00E94FF4E0E94E7
:10E31000866C0E94B26B1092640E1092650E109281
:10E32000660E1092B60E0E9446668091A50E882356
:10E3300009F481E08093A50E83EB9EE40E947E4663
:10E3400082E080932901ABCC903279F49DE09D83EB
:10E3500080E18E8385E08F8386E08887CE010596F5
:10E3600060E00E941D4D81E015C0943021F482E0F0
:10E370008093290105C0923019F424E020932901EB
:10E380008091290162FE31C0803209F487CC81304E
:10E3900021F480E28093290181CC98E79093310E9B
:10E3A00028E22093320E81E39EE068E30E9423621C
:10E3B00088E39EE060E044E35EE00E94FF4E8EE36F
:10E3C0009EE060E045E35EE00E94FF4E81E08093C6
:10E3D000390E0E94B26B0E94A54688E08093290105
:10E3E0001201A1E0AA2EB12C5ACC843009F456CCEB
:10E3F00073FE04C0809128018F5F05C072FE06C0C5
:10E4000080912801815083708093280160FE75C03F
:10E4100080912801813059F1813038F0823009F43F
:10E4200044C0833009F069C052C02091AB0E222352
:10E4300009F463C03091450E832F90E08370907093
:10E44000892B09F45AC021502093AB0E8091B00E55
:10E450009091B10E80509F4F9093B10E8093B00E6B
:10E46000313009F04AC082E00E94D46946C09091E0
:10E47000AC0E992309F441C08091450E8430E9F136
:10E4800091509093AC0E8091B20E9091B30E892B67
:10E4900029F48091490E880F8093490E80E491E021
:10E4A0009093B30E8093B20E28C08091450E8430B5
:10E4B00021F18091AD0E882301F181508093AD0E42
:10E4C00080E891E09093B50E8093B40E16C08091D1
:10E4D000AE0E853090F085508093AE0E8091AC0EDC
:10E4E0008F5F8093AC0E8091AB0E8F5F8093AB0EED
:10E4F0008091AD0E8F5F8093AD0E8091BD0E909197
:10E50000BE0E892BA9F01092280C1092270C88E3DC
:10E510009EE060E044E35EE00E94FF4E8EE39EE0FA
:10E5200060E045E35EE00E94FF4E00E010E045C081
:10E53000810100951095042915298091270C90914F
:10E54000280C0823192304291529062917291093B3
:10E55000280C0093270C8091BB0E9091BC0E892B48
:10E56000E9F0A80140715070440F551F98012078C0
:10E57000307036952795C80180749070880F991F68
:10E58000282B392BC8018F70282B392B0072107063
:10E5900016950795022B132B042B152B1092470E63
:10E5A0009091390E9A87809129018A7031F0E0911B
:10E5B000620EF091630EC801099581E39EE00E940E
:10E5C0008661482F8091450E823051F0833018F4D7
:10E5D0008130D9F411C08430A1F08830B1F411C079
:10E5E0008091BD0E9091BE0E892B79F48091390EE9
:10E5F0006A850E94906409C08A85B8010E94B5644A
:10E6000004C08A85B8010E9450658091470E80FF42
:10E6100002C00E94A8698091470E81FF1BC08091B3
:10E62000580E20915C0E829FC00111242091600E33
:10E630003091610E280F391F00E08091390E813032
:10E6400009F001E08091440E6091590E40915A0EFC
:10E650000E94E04C6091330E8091360E681B409111
:10E66000320E4F5F8091370E481B8091440E2091EF
:10E67000590E00915A0E0E94F54A809129018A7024
:10E6800011F10E94DE6A0E94ED65809129018830B7
:10E6900021F08091B80E8823B1F08091B60E8F5F83
:10E6A0008093B60E8C3378F01092B60E8091AF0E38
:10E6B000882321F081508093AF0E03C081E00E9437
:10E6C00048640E9446660E94AF55E8CA2F923F9266
:10E6D0004F925F927F928F929F92AF92BF92CF9212
:10E6E000DF92EF92FF920F931F93DF93CF9300D0AF
:10E6F00000D0CDB7DEB7A82F7B015A012901FA015E
:10E700008081982F969596959695292E332487701B
:10E71000C82EDD2401E010E0C8010C2C02C0880FD7
:10E72000991F0A94E2F7F101E959F14F70807822BC
:10E73000A130E9F4772009F4F1C1DA0111968C9146
:10E7400011978E3009F0E8C11296EC911297F0E023
:10E75000E959F14F13960C9002C0000F111F0A9453
:10E76000E2F7802F8095908189238083D5C1A230E4
:10E7700099F4772009F4D2C1FA018181893009F036
:10E78000CBC120E08091BD0E9091BE0E892B09F087
:10E7900021E081E02827C3C1772009F4BFC172E0DE
:10E7A000872E912C8E0C9F1CDA0111968C9186304D
:10E7B00009F433C1873088F4823009F496C083307D
:10E7C00028F48823F9F0813039F528C0843009F421
:10E7D00017C1853008F01AC1FEC08A3009F430C173
:10E7E0008B3030F4873009F425C18830A9F494C106
:10E7F0008D3009F46CC18E3009F48EC18C3061F417
:10E8000011E071C18EE06FEF41E00E94184A8091E3
:10E81000AE0E8F5F8093AE0E10E065C18FE06FEF9C
:10E8200041E00E94184AF7018181E82FF0E0EE0FE5
:10E83000FF1FEB59F64A659174914091A50E842F04
:10E8400090E0837090708130910539F182309105AC
:10E850001CF4892B71F02FC08230910519F00397B9
:10E8600051F522C080E091E09093BE0E8093BD0EE2
:10E8700022C02091B90E3091BA0EC90156E096958A
:10E8800087955A95E1F780369105A8F420503F4FBF
:10E890003093BA0E2093B90E0EC080E091E09093B1
:10E8A000BC0E8093BB0E07C08091AE0E882319F07A
:10E8B00081508093AE0E10E06B577C4309F011E05D
:10E8C000842F86958695942F96959695969589276B
:10E8D0008427942F92959F708927879588278795FD
:10E8E0004695842B8093A50EFEC08CE06FEF41E02F
:10E8F0000E94184AC6010196FC0123E0F595E795B0
:10E900002A95E1F7E20DF31DE959F14F87709070F8
:10E9100002C0000F111F8A95E2F7802F8095908129
:10E92000892380838091870E882329F08DE29EE0E1
:10E9300060E00E941D4DF70182819381A481B58121
:10E9400080932D0E90932E0EA0932F0EB093300E29
:10E9500080912E0E8F5F80932E0E80912F0E81500E
:10E9600080932F0E8DE29EE060E040E027E23DE3E1
:10E9700002E010E00E943A4D80E18093870E82E031
:10E98000882E912C8A0C9B1CD20112968D919C9101
:10E990001397BC01660F771F680F791F660F771FEB
:10E9A000625C744AC70146E050E00E948043D70190
:10E9B0001296EC911297F0E0E959F14F81E090E066
:10E9C00013960C9002C0880F991F0A94E2F72081D9
:10E9D000282B208321CFF7018181E82FF0E0EE0F73
:10E9E000FF1FEB59F64A8591949110E083579C43A1
:10E9F00009F011E08091AC0E8F5F8093AC0E73C074
:10EA00008091AD0E8F5F8093AD0E06CF80E891E0D0
:10EA100090932C0E80932B0EFFCE10E0D701119611
:10EA20008C918C3109F011E08091AB0E8F5F809357
:10EA3000AB0E59C08091AF0E8B5F8093AF0EECCEC2
:10EA40008091450E843009F44BC08091B40E9091B2
:10EA5000B50E892B09F444C06091310E70E020910D
:10EA6000360E30E0E091320EF0E04091370E50E08B
:10EA7000CB01821B930BA3E095958795AA95E1F7AF
:10EA80008983260F371F63E0359527956A95E1F74F
:10EA90002A83CF01841B950B23E0959587952A95B2
:10EAA000E1F78B834E0F5F1F03E0559547950A955D
:10EAB000E1F74C83C5010296BE016F5F7F4F0E9454
:10EAC000E24E882369F481E08093B70E25C08091DF
:10EAD000AF0E882329F48091B60E865F8093B60E20
:10EAE00010E088249924F50181818350853028F431
:10EAF0008DE06FEF41E00E94184A8114910471F09B
:10EB0000F101E959F14F7094808178227082C4013B
:10EB1000612F0E941D4D02C021E001C020E0822F24
:10EB20000F900F900F900F90CF91DF911F910F9149
:10EB3000FF90EF90DF90CF90BF90AF909F908F901D
:10EB40007F905F904F903F902F900895629FD001EB
:10EB5000739FF001829FE00DF11D649FE00DF11D98
:10EB6000929FF00D839FF00D749FF00D659FF00D47
:10EB70009927729FB00DE11DF91F639FB00DE11D34
:10EB8000F91FBD01CF0111240895991B79E004C03C
:10EB9000991F961708F0961B881F7A95C9F78095DC
:06EBA0000895F894FFCF78
:10EBA6000100408891D2E4ADB5B6BEBFFF555A45C7
:10EBB600000A0F09090909090909090909090909C1
:10EBC60009090909090909090308525354555657F1
:10EBD60058595A5B5CA7A8A9AAABACADAEAFB0B109
:10EBE600B2B3B4B5B6B7B8B9BABBBCBDBEBFC00840
:00000001FF
